:020000041000EA
:1000000000001020ADD50110E9D50110EBD501108D
:10001000EDD50110EFD50110F1D501100000000061
:10002000000000000000000000000000F3D50110F7
:10003000F5D5011000000000F7D5011019B8001027
:10004000FBD50110FDD5011005C40010A9C3001097
:1000500003D60110C1C10010D5C10010E9C10010C4
:100060000BD601100DD601100FD6011011D60110BC
:1000700013D60110EDBC001085C1001099C100100D
:100080001BD601101DD601101FD6011021D601105C
:1000900023D6011025D6011027D6011029D601102C
:1000A000B5BC0010C3BC0010D1BC001031D601108B
:1000B000C9C20010D7C20010E5C20010F3C2001080
:1000C0003BD601103DD60110ADC1001041D6011044
:1000D00001BD001045D6011047D6011049D60110C8
:1000E0004BD601104DD601104FD6011051D601103C
:1000F00053D6011055D6011057D6011059D601100C
:100100005BD601105DD601105FD6011061D60110DB
:1001100063D6011065D6011067D6011069D60110AB
:100120006BD601106DD60110DFBC001071D6011026
:1001300073D6011075D6011077D6011079D601104B
:100140007BD601107DD601107FD6011081D601101B
:1001500001C300100FC300101DC300102BC30010FB
:1001600039C3001047C3001055C3001063C300100B
:1001700071C300107FC300108DC300109BC300101B
:100180009BD601100348044B834202D0034B03B1BA
:10019000184770478C1F00208C1F002000000000B3
:1001A000054806490B1AD90F01EBA301491002D0EB
:1001B000034B03B1184770478C1F00208C1F002091
:1001C0000000000010B5064C237843B9FFF7DAFFB2
:1001D000044B13B10448AFF300800123237010BD1A
:1001E000901F0020000000008CD8041008B5044BBC
:1001F0001BB104490448AFF30080BDE80840CFE7D5
:1002000000000000941F00208CD8041080B584B03A
:1002100000AF7860124B1B68002B02D1104B114AC3
:100220001A600F4B1B68FB600D4B1A687B68134408
:100230001A460D4B9A4207D91EF082F903460C224A
:100240001A604FF0FF3306E0054B1A687B681344D1
:10025000034A1360FB6818461037BD4680BD00BFD7
:10026000AC1F0020483E012000F00F2080B400AFFA
:100270006FF010031846BD4680BC704780B400AFD5
:100280006FF010031846BD4680BC704780B485B03F
:1002900000AF4FF080439B6803F46063BB60BB68B2
:1002A000B3F5806F02D11A4BFB601EE0BB68B3F55B
:1002B000C06F03D14FF4FA53FB6016E0BB68B3F58F
:1002C000006F02D1134BFB600FE0BB68B3F5206FEA
:1002D00002D1114BFB6008E0104B1B78A12B02D917
:1002E0000F4BFB6001E00F4BFB604FF080439B68BE
:1002F0009B0903F007037B60FA687B6822FA03F32B
:10030000094A136000BF1437BD4680BC704700BF68
:1003100000366E01000E270700127A00B41F00207D
:1003200080F0FA02005A6202B01F002080B400AFD1
:100330004FF080431B6823F440334FF0804243F476
:100340000033136000231846BD4680BC7047000090
:1003500080B500AF04F0FCFE03461A46554B1A70F8
:10036000554B564A9A6062B600BF534BD3F888305B
:10037000514A43F47003C2F88830BFF34F8F00BF77
:10038000BFF36F8F00BF042004F092FDFFF77EFFE4
:100390004FF080431B684FF0804243F400331360FA
:1003A000474B0122C3F8002700BF454BD3F800316B
:1003B00003F48033002BF8D0414BD3F80031404A8E
:1003C00043F00103C2F8003100BF3D4BD3F80031C8
:1003D00003F48033002BF8D0032004F012FD042036
:1003E00004F00FFD052004F00CFD062004F009FDCB
:1003F000072004F006FD082004F003FD092004F0A6
:1004000000FD0A2004F0FDFC0D2004F0FAFC0E2093
:1004100004F0F7FC0F2004F0F4FC102004F0F1FCD1
:10042000112004F0EEFC122004F0EBFC132004F089
:10043000E8FC142004F0E5FC172004F0E2FC1C208A
:1004400004F0DFFC1D2004F0DCFC1E2004F0D9FCCD
:100450001F2004F0D6FC212004F0D3FC222004F05D
:10046000D0FC232004F0CDFC242004F0CAFC27207B
:1004700004F0C7FC282004F0C4FC292004F0C1FCCF
:100480002A2004F0BEFC2B2004F0BBFC2C2004F03E
:10049000B8FC2D2004F0B5FC2E2004F0B2FC2F2077
:1004A00004F0AFFC342004F0ACFC0BF095FC00BF72
:1004B00080BD00BFB41F002000ED00E00000001070
:1004C00000A0024080B483B000AFEFF310833B6024
:1004D0003B687B607B68002B0CBF01230023DBB2F1
:1004E0001A46034B1A6000BF0C37BD4680BC7047EC
:1004F0000000002080B500AFFFF7E4FF054B1B684C
:10050000002B01D072B600BF024B01225A6000BF1F
:1005100080BD00BF0000002080B500AF064B1B6807
:10052000002B01D062B600BF034B00225A60FFF7D8
:10053000C9FF00BF80BD00BF0000002080B485B0AF
:1005400000AF7860064BFB607B689B00FA68134441
:10055000FB60FB6818461437BD4680BC704700BF7F
:1005600020100B4080B489B000AFF860B9607A60A9
:10057000FB687B61BB68FB617B689B08BB617B6838
:1005800003F003037B6005E0FB691A1DFA611A683A
:100590007B691A60BB695A1EBA61002BF4D1FB69F2
:1005A000BB6005E0BB685A1CBA601A78FB681A7019
:1005B0007B685A1E7A60002BF4D100BF00BF24373D
:1005C000BD4680BC704780B489B000AFF860B960A8
:1005D0007A60BB687B61FB68FB617B689B08BB61E1
:1005E0007B6803F003037B6005E0FB691A1DFA6179
:1005F0007A6912681A60BB695A1EBA61002BF4D17D
:10060000FB69FB6006E0FB685A1CFA60BA68127866
:10061000D2B21A707B685A1E7A60002BF3D100BFE9
:1006200000BF2437BD4680BC7047000080B584B051
:1006300000AF78607B68002B05D0102279683948BC
:100640001EF078FA02E0374B00221A60354B9B68A7
:10065000002B08D0334B9B6898470346002B02D0F1
:100660004FF0FF3359E0304B40221A600123FB600A
:1006700006E0FB68184600F033FAFB680133FB60C4
:10068000FB680B2BF5DD294B00221A70284B00224A
:100690005A70274B0022DA80254B00221A81244B06
:1006A0000022DA72224B0022C3F8A024204B40F62D
:1006B0000802C3F860241E4B0022C3F864241C4BBC
:1006C0004FF48072C3F86824194B0022C3F86C24DD
:1006D000174B0122C3F81424154B0122C3F8182428
:1006E000134B0022C3F85C24114B0022C3F84824AA
:1006F0000F4B0222C3F84C240D4B0122C3F83024C7
:100700000B4B0122C3F83C24094B0022C3F81024F0
:10071000074B0122C3F81024002318461037BD46AA
:1007200080BD00BF1C200020E81F002018200020F2
:1007300000100B4080B400AF124B1B68002B08D098
:10074000114B5B78DBB2104A43F02003DBB25370ED
:1007500007E00D4B5B78DBB20B4A23F02003DBB2E2
:100760005370094B5B78DBB2074A43F04003DBB2BE
:100770005370064B00221A7000231846BD4680BCF9
:10078000704700BF1C20002000100B4018200020E4
:1007900080B400AF074B5B78DBB2064A23F040031E
:1007A000DBB25370044B00221A7000231846BD467A
:1007B00080BC704700100B401820002080B483B02C
:1007C00000AF00237B600E4BD3F8A43403F0010389
:1007D000002B03D07B6843F001037B60084B5B7800
:1007E000DBB203F01003002B03D07B6843F002035D
:1007F0007B607B6818460C37BD4680BC704700BFE5
:1008000000100B4080B584B000AFF8600B467A60F2
:10081000FB72FB68002B06D0FB680B2B03D87B68B0
:10082000B3F5007F02D94FF0FF3358E0F86800F0CD
:1008300057F9FFF75FFE2C4BFA68D2B29A73FB7A36
:10084000022B25D0022B41DC002B44D0012B3DD1C3
:10085000254B80229A75244B0222DA75224B7A6846
:1008600092B29A822149FB687A6841F823201E4B94
:100870001B899BB21AB20121FB6801FA03F31BB278
:10088000DB431BB213401AB2174B92B21A8123E01A
:10089000154B40229A74144B2222DA74124B7A6858
:1008A00092B21A821149FB687A6841F823200E4BF4
:1008B000DB889BB21AB20121FB6801FA03F31BB279
:1008C00013431AB2084B92B2DA8005E0FFF724FE18
:1008D0004FF0FF3303E000BFFFF71EFE0023184672
:1008E0001037BD4680BD00BF00100B40E81F002040
:1008F00080B483B000AF7860064A7B6852F823303A
:10090000002B14BF01230023DBB218460C37BD4671
:1009100080BC7047E81F002080B584B000AF7860CD
:100920007868FFF7E5FF0346002B02D14FF0FF3355
:100930004AE0FFF7DFFD264B7A68D2B29A737B68F4
:10094000002B0BD1224B9B7CDBB2214A43F060038E
:10095000DBB293741F4B00221A7017E01C4BDB7C38
:10096000DBB203F02003002B08D0194B9B7CDBB2D9
:10097000174A43F01003DBB2937407E0144B9B7DDE
:10098000DBB2134A43F02003DBB29375124A7B6853
:1009900052F82330FB60104A7B68002142F8231094
:1009A000FB68002B0DD0FB684FF0FF321A61FB682B
:1009B0005B69002B05D0FB685B69FA689269104699
:1009C0009847FFF7A9FD002318461037BD4680BDA4
:1009D00000100B4018200020B81F002080B582B006
:1009E00000AF78607868FFF783FF0346002B02D1E1
:1009F0004FF0FF332FE0FFF77DFD194B7A68D2B23D
:100A00009A737B68002B23D0154BDB7CDBB203F0A1
:100A10002003002B0ED0124B9B7CDBB203F00103B2
:100A2000002B03D00E4B48229A7411E00C4B40224D
:100A30009A740DE00A4B9B7DDBB203F00103002B9F
:100A400003D0074B90229A7502E0054B80229A75DD
:100A5000FFF762FD002318460837BD4680BD00BF82
:100A600000100B4080B485B000AF78601B4B7A68F3
:100A7000D2B29A737B68002B1ED0184BDB7CDBB2A2
:100A800003F02003002B0BD0144B9B7CDBB203F054
:100A90001003002B14BF01230023DBB2FB6016E020
:100AA0000E4B9B7DDBB203F02003002B14BF012310
:100AB0000023DBB2FB600AE0084B9B7CDBB203F057
:100AC0002003002B14BF01230023DBB2FB60FB6873
:100AD00018461437BD4680BC704700BF00100B405D
:100AE00080B584B000AF78607B680B2B02D94FF0E3
:100AF000FF3374E0FFF7FEFC3B4A7B6852F823307B
:100B0000FB60394A7B68002142F823107B68002B88
:100B100062D0364A7B68002142F82310344B7A6851
:100B2000D2B29A73324BDB889BB21AB201217B6836
:100B300001FA03F31BB2DB431BB213401AB22C4B76
:100B400092B2DA802A4B1B899BB21AB201217B68D0
:100B500001FA03F31BB2DB431BB213401AB2244B5E
:100B600092B21A81224B9B7CDBB203F00103002B73
:100B700002D01F4B08229A741D4B10229A741C4BF2
:100B80000222DA741A4B00221A82194B9B7DDBB2C7
:100B900003F00103002B02D0154B10229A75144B61
:100BA00020229A75124B0222DA75114B00229A828A
:100BB000FFF7B2FCFB68002B10D0FB684FF0FF3250
:100BC0001A61FB685B69002B08D0FB685B69FA68F7
:100BD00092691046984701E0FFF79EFC00231846F3
:100BE0001037BD4680BD00BFB81F0020E81F0020A1
:100BF00000100B4080B584B000AF78607B68002B9C
:100C000002D04FF0FF331EE0FFF774FC104B9B7BCC
:100C1000DBB2FB600E4B00229A730E4B1B78012B4C
:100C200007D10B4B9B7CDBB2094A43F04803DBB294
:100C30009374084B00221A70054BFA68D2B29A736B
:100C4000FFF76AFC002318461037BD4680BD00BF81
:100C500000100B401820002080B588B000AF7860ED
:100C60000023FB618FE00122FB6902FA03F37B6141
:100C70007A687B691340002B7FD0474AFB6952F8A2
:100C80002330002B7BD0454BFA69D2B29A73424A8B
:100C9000FB6952F823303B613B699A683B69DB682A
:100CA000D31AFB60FB68002B57D03D4AFB6952F812
:100CB0002330FA689A4205D3394AFB6952F8233047
:100CC000BB6101E0FB68BB61F869FFF737FC3B697A
:100CD0005A683B69DB681344BA691946FFF742FC5E
:100CE0003B69DA68BB691A443B69DA60FB69002B2F
:100CF0002FD1294AFB6952F82330DA682649FB696B
:100D000051F823309B689A421AD1264B00221A7060
:100D1000224B9B7CDBB2214A43F00A03DBB2937483
:100D20001D4AFB69002142F823103B695B69002BD7
:100D300026D03B695B693A699269104698471FE083
:100D4000164B9B7CDBB2154A43F00203DBB2937473
:100D500016E0124B01229A7412E00F4AFB6900213F
:100D600042F823103B695B69002B09D03B695B6942
:100D70003A6992691046984702E000BF00E000BF60
:100D8000FB690133FB61FB690B2B7FF66CAF00BF86
:100D900000BF2037BD4680BDB81F002000100B40AB
:100DA000E81F00201820002090B587B000AF7860C1
:100DB00000237B6114E101227B6902FA03F3FB60EB
:100DC0007A68FB681340002B00F0FC80894A7B693D
:100DD00052F82330002B00F0F780864A7B6952F8E6
:100DE0002330BB60844B7A69D2B29A737B69002B43
:100DF00030D1814B9B7CDBB203F00103002B00F070
:100E0000E5807D4B1B8B9BB2002B10D1794A7B690F
:100E1000002142F82310BB685B69002B00F0D880EA
:100E2000BB685B69BA68926910469847D0E0724B1C
:100E30001B8B9BB23B61BB689A68BB68DB68D31AAB
:100E40003A699A424ED9BB689A68BB68DB68D31A84
:100E50003B6147E0684B9B7DDBB203F00103002B55
:100E600000F0B880644B1B8B9BB2002B28D1614AE9
:100E70007B69002142F823105F4B9B7DDBB25E4A09
:100E800023F00103DBB293755B4B1B899BB21AB253
:100E900001217B6901FA03F31BB2DB431BB2134050
:100EA0001AB2554B92B21A81BB685B69002B00F0F5
:100EB0009380BB685B69BA689269104698478BE07B
:100EC0004D4B1B8B9BB23B61BB689A68BB68DB6870
:100ED000D31A3A699A4205D9BB689A68BB68DB683D
:100EE000D31A3B61BB685A68BB68DB68D418786961
:100EF000FFF724FB03463A6919462046FFF763FBD8
:100F0000BB68DA683B691A44BB68DA607B69002B0E
:100F100026D1BB68DA68BB689B689A4217D1364B0A
:100F20009B7CDBB2344A43F04803DBB29374314A12
:100F30007B69002142F82310BB685B69002B4CD011
:100F4000BB685B69BA6892691046984745E02A4BCE
:100F50009B7CDBB2284A43F04003DBB293743CE055
:100F6000254B9B7DDBB2244A23F00103DBB2937552
:100F7000BB681B7F012B05D0BB68DA68BB689B6828
:100F80009A422AD11B4A7B69002142F823101A4B4E
:100F90001B899BB21AB201217B6901FA03F31BB2D0
:100FA000DB431BB213401AB2134B92B21A81BB68D7
:100FB0005B69002B11D0BB685B69BA689269104607
:100FC00098470AE000BF08E000BF06E000BF04E069
:100FD00000BF02E000BF00E000BF7B6901337B611E
:100FE0007B690B2B7FF6E7AE00BF00BF1C37BD4609
:100FF00090BD00BFB81F002000100B4080B592B01C
:1010000000AF78600023BB63934B9B7BDBB27B63B9
:10101000914B9B7ADBB23B638F4BDB7ADBB2FB629B
:101020003A6BFB6A1340BB628B4B5B889BB27B6263
:10103000894BDB889BB23B627A6A3B6A13407B64D4
:10104000854B9B889BB2FB61834B1B899BB2BB6129
:10105000FA69BB6913403B647F4BD3F898347B61DA
:101060007D4BD3F89C343B617A693B691340FB604C
:10107000794AFB68C2F89834BB6A03F00803002B76
:1010800014BF01230023D9B27A68137861F30003F7
:1010900013707A6813786FF341031370BB6A03F01F
:1010A0000803002B14BF01230023D9B27A681378F8
:1010B00061F382031370BB6A03F00403002B14BFB7
:1010C00001230023D9B27A68137861F3C303137044
:1010D000BB6A03F00103002B14BF01230023D9B224
:1010E0007A68137861F304131370FB6803F002034A
:1010F000002B14BF01230023D9B27A68137861F35F
:1011000045131370FB6803F00103002B14BF012388
:101110000023D9B27A68137861F386131370BB6A1F
:1011200003F00403002B14BF01230023D9B27A6813
:10113000137861F3C71313707A6853786FF3000361
:1011400053707B6C03F00103002B59D0424B0022FB
:101150009A73414B9B7CDBB203F00403002B10D04D
:101160003D4B9B7CDBB23C4A23F00403DBB293741F
:101170007B6C23F001037B64384B00221A7001233F
:10118000BB63354B9B7CDBB203F01003002B13D009
:10119000314B9B7CDBB2304A63F07F03DBB293744C
:1011A0002E4B00221A707B6C23F001037B6400201D
:1011B000FFF796FC0123BB63BB6B002B20D1274BB1
:1011C0001B78002B10D1244B9B7CDBB203F0010376
:1011D000002B09D07A68537843F0010353707B6C7D
:1011E00023F001037B640BE01C4B1B78022B07D11F
:1011F0007B6C23F001037B643B6C43F001033B6495
:101200007B681B7803F00803DBB2002B10D0134B74
:1012100000221A700023FB6306E0FB6B1846FFF701
:101220005FFCFB6B0133FB63FB6B0B2BF5DD0FE00E
:101230007B6C002B02D0786CFFF70EFD3B6C002B13
:1012400002D0386CFFF7B0FD034B7A6BD2B29A73C1
:101250004837BD4680BD00BF00100B40182000205D
:1012600080B483B000AF0346FB71FB79082B02D931
:101270004FF0FF3354E0FB79023B062B4ED801A21E
:1012800052F823F0A1120010B3120010C512001082
:101290000B130010F91200101D130010E7120010BC
:1012A000224BDB7ADBB2214A43F00803DBB2D37274
:1012B00035E01E4BDB7ADBB21C4A43F00403DBB2A1
:1012C000D3722CE0194B5B78DBB2184A43F0010370
:1012D000DBB25370154BDB7ADBB2144A43F00103E7
:1012E000DBB2D3721BE0114BDB889BB20F4A43F099
:1012F00001039BB2D38012E00C4BD3F89C340B4A11
:1013000043F00103C2F89C3409E0084BD3F89C3445
:10131000064A43F00203C2F89C3400E000BF0023F9
:1013200018460C37BD4680BC704700BF00100B400C
:1013300080B483B000AF0346FB71FB79082B02D960
:101340004FF0FF3354E0FB79023B062B4ED801A24D
:1013500052F823F07113001083130010951300103E
:10136000DB130010C9130010ED130010B7130010A9
:10137000224BDB7ADBB2214A23F00803DBB2D372C3
:1013800035E01E4BDB7ADBB21C4A23F00403DBB2F0
:10139000D3722CE0194BDB7ADBB2184A23F001033D
:1013A000DBB2D372154B5B78DBB2144A23F0010336
:1013B000DBB253701BE0114BDB889BB20F4A23F06A
:1013C00001039BB2D38012E00C4BD3F89C340B4A40
:1013D00023F00103C2F89C3409E0084BD3F89C3495
:1013E000064A23F00203C2F89C3400E000BF002349
:1013F00018460C37BD4680BC704700BF00100B403C
:1014000080B483B000AF0346FB71002318460C374D
:10141000BD4680BC7047000080B584B000AF7860E6
:101420003A4BFB60FFF766F8394B00229A737B68F2
:10143000002B06D0364B9B7CDBB203F00103002B64
:1014400004D1FFF769F84FF0FF335BE0FB681B78CE
:10145000DAB27B681A70FB681B78DAB27B685A7064
:10146000FB681B78DBB29AB27B685A80FB681B78FA
:10147000DBB219027B685A888BB213449AB27B683C
:101480005A80FB681B78DBB29AB27B689A80FB6853
:101490001B78DBB219027B689A888BB213449AB22C
:1014A0007B689A80FB681B78DBB29AB27B68DA8033
:1014B000FB681B78DBB219027B68DA888BB21344B5
:1014C0009AB27B68DA807B68DB88002B14D0104BE3
:1014D0009B7CDBB20E4A43F04003DBB293747B6823
:1014E0001B785BB2002B03DA0A4B03221A7006E06A
:1014F000084B02221A7002E0064B01221A70FFF715
:101500000BF8002318461037BD4680BD20100B4055
:1015100000100B401820002080B483B000AF78602A
:101520007B687F2B02D94FF0FF3304E0044B7A68CD
:10153000D2B21A70002318460C37BD4680BC7047E3
:1015400000100B4080B582B000AF78607B681B68EC
:101550000B2B02D94FF0FF331FE07B681B68114A49
:1015600052F823307A689A4202D04FF0FF3314E0E9
:101570007B681B680B4A002142F823107B684FF000
:10158000FF321A617B685B69002B05D07B685B6961
:101590007A68926910469847002318460837BD4676
:1015A00080BD00BFB81F002080B586B000AF786056
:1015B0007B681B683B617B689B687B613B690B2B8D
:1015C00002D94FF0FF3372E03869FFF791F9034613
:1015D000002B02D14FF0FF3369E0FEF78BFF364B53
:1015E0003A69D2B29A73354A3B6952F82330002BDC
:1015F00006D1314B9B7CDBB203F00103002B04D0FE
:10160000FEF78AFF4FF0FF3351E02C493B697A68BF
:1016100041F823207B6800221A610023FB60FB68ED
:10162000002B41D1264A3B6952F823307A699A420D
:1016300004D9234A3B6952F823307B611F4A3B6936
:1016400052F823307A69DA603869FEF777FF7B68F1
:101650005B687A691946FEF785FF3B69002B20D14C
:10166000164A3B6952F82330DA6814493B6951F84D
:1016700023309B689A420BD1124B00221A700E4BFA
:101680009B7CDBB20C4A43F00A03DBB293740BE0A1
:10169000094B9B7CDBB2084A43F00203DBB2937434
:1016A00002E0054B01229A74FEF736FF002318462C
:1016B0001837BD4680BD00BF00100B40B81F00208A
:1016C000E81F00201820002090B587B000AF786098
:1016D0007B681B683B613B690B2B02D94FF0FF33E2
:1016E000ABE0FEF707FF3869FFF702F90346002B6E
:1016F00004D1FEF711FF4FF0FF339EE03869FFF78A
:10170000B1F90346002B04D0FEF706FF4FF0FF337C
:1017100093E04C4A3B6952F82330002B04D0FEF78B
:10172000FBFE4FF0FF3388E07B6800221A617B6884
:101730000022DA6043493B697A6841F82320424B32
:101740003A69D2B29A733B69002B73D00023FB60D5
:10175000FB68002B6ED13C4B9B7DDBB203F0010399
:10176000002B59D0384B1B8B9BB27B617B689A68EE
:101770007B68DB68D31A7A699A4205D97B689A68D4
:101780007B68DB68D31A7B617B685A687B68DB689F
:10179000D4183869FEF7D2FE03467A691946204606
:1017A000FEF711FF7B68DA687B691A447B68DA60B0
:1017B000254B9B7DDBB2244A23F00103DBB29375FA
:1017C0007B681B7F012B05D07B68DA687B689B6890
:1017D0009A4212D1FEF7A0FE1A4A3B69002142F854
:1017E00023107B685B69002B05D07B685B697A6896
:1017F00092691046984700231FE0134B1B899BB248
:101800001AB201213B6901FA03F31BB213431AB266
:101810000D4B92B21A810DE00B4B1B899BB21AB291
:1018200001213B6901FA03F31BB213431AB2064BC1
:1018300092B21A81FEF770FE002318461C37BD468F
:1018400090BD00BFB81F002000100B4080B584B0D1
:1018500000AF0346B9607A60FB73FB7B082B02D8AC
:10186000BB68002B02D14FF0FF330FE0FB7B09492F
:10187000BA6841F83320FB7B064ADB0013447A68E0
:101880005A60FB7B1846FFF7EBFC034618461037FF
:10189000BD4680BD3020002080B584B000AF034637
:1018A000FB714FF0FF33FB60FB79082B02D94FF03F
:1018B000FF3310E0FB791846FFF73AFDF860FB793B
:1018C000074A002142F83310FB79054ADB00134434
:1018D00000225A60FB6818461037BD4680BD00BF25
:1018E0003020002080B582B000AF0346FB71FB7949
:1018F000082B02D94FF0FF3304E0FB791846FFF7BD
:101900007FFD034618460837BD4680BD80B500AF51
:101910005348FFF773FB524B1B7803F02003DBB2F5
:10192000002B0AD04F4B9B6A002B06D04D4B9B6A75
:101930004C4AD26A114605209847494B1B7803F060
:101940004003DBB2002B0AD0464B1B6B002B06D0AA
:10195000444B1B6B434A526B114606209847404B41
:101960001B7803F00803DBB2002B0AD03D4B9B69C8
:10197000002B06D03B4B9B693A4AD26911460320A3
:101980009847374B1B7823F07F03DBB2002B0AD03C
:10199000344B9B6B002B06D0324B9B6B314AD26B86
:1019A0001146072098472E4B1B7803F00103DBB24A
:1019B000002B0AD02B4B1B68002B06D0294B1B6831
:1019C000284A5268114600209847254B1B7803F09F
:1019D0000203DBB2002B0AD0224B9B68002B06D0FF
:1019E000204B9B681F4AD2681146012098471C4B28
:1019F0001B7803F00403DBB2002B0AD0194B1B69E0
:101A0000002B06D0174B1B69164A5269114602205B
:101A10009847134B1B7803F01003DBB2002B0AD05E
:101A2000104B1B6A002B06D00E4B1B6A0D4A526AE4
:101A30001146042098470A4B5B7803F00103DBB2A0
:101A4000002B0AD0074B1B6C002B06D0054B1B6CE0
:101A5000044A526C11460820984700BF80BD00BF61
:101A60002C2000203020002080B582B000AF7860AC
:101A7000104B00221A70104B00221A700F4B0022DC
:101A80001A70102200210E481DF0EEF80D4A0E4982
:101A9000002000F0E9FC7B689A780C4B1A70002259
:101AA0000B49002000F0C0FC034618460837BD462D
:101AB00080BD00BF802000208120002082200020E7
:101AC000C0220020D4220020D02200208320002029
:101AD000A11F001080B483B000AF03463960FB71D2
:101AE000FB79032B02D94FF0FF3305E0FB79054961
:101AF0003A6841F82320002318460C37BD4680BCC5
:101B0000704700BFC022002080B584B000AF78606D
:101B1000574B00221A60574B00221A607B685B8883
:101B2000402B07D87B68DB88402B03D87B685B8918
:101B3000402B02D94FF0FF3395E07B681A784E4B6B
:101B40001A704D4B1B7818467B685B881A4601213A
:101B5000FEF758FEF860FB68002B03D000F0ACF8ED
:101B6000FB6880E07B681A79444B1A70434B1B7802
:101B700018467B68DB881A460221FEF743FEF860B0
:101B8000FB68002B03D000F097F8FB686BE07B68E4
:101B90001A7A3B4B1A703A4B1B7818467B685B8964
:101BA0001A460221FEF72EFEF860FB68002B03D0D8
:101BB00000F082F8FB6856E081223249324800F09A
:101BC00055FB2422002131481DF04EF82B4B1B7889
:101BD0001A462E4B1A602D4B2D4A5A602B4B2D4A1C
:101BE0005A612A4B294A9A61284B01221A7781228D
:101BF00029492A4800F03AFB2422002128481DF0F8
:101C000033F81D4B1B781A46254B1A60244B254A86
:101C10005A60234B40229A60214B234A5A61204B41
:101C20001F4A9A611E4B01221A77242200211F4865
:101C30001DF01AF8124B1B781A461C4B1A601C4BED
:101C40001A781C4B1A71194B1A4A5A60174B0A2200
:101C50009A60164B00225A61144B00229A61134B72
:101C600000221A77002318461037BD4680BD00BFFA
:101C7000782000207C20002080200020812000206F
:101C8000822000200C21002090210020A82000208C
:101C9000CC200020091F0010082200208C220020E8
:101CA000A4210020C8210020E91E00109C22002051
:101CB000832000201000002080B500AF1A48FFF7F5
:101CC00041FC1A4B1B78002B07D0184B1B78184689
:101CD000FEF706FF154B00221A70154B1B78002BE0
:101CE00007D0134B1B781846FEF7FAFE104B002264
:101CF0001A70104B1B78002B07D00E4B1B78184620
:101D0000FEF7EEFE0B4B00221A700B4800F02EFB84
:101D10000A4800F02BFB0A4B00221A60094B0022F4
:101D20001A600023184680BDA421002080200020D6
:101D30008120002082200020902100208C22002081
:101D4000782000207C20002080B400AF024B1B686C
:101D50001846BD4680BC70477820002080B584B00E
:101D600000AF786039600023FB601FE0144B1B68F4
:101D7000002B02D06FF001031DE0124B1B68002BFB
:101D800001D1002317E000F055F807F10B031946C5
:101D90000D4800F0BEFA0346002BE7D17A68FB68D5
:101DA0001344FA7A1A70FB680133FB60FA683B68E7
:101DB0009A42EAD3FB6818461037BD4680BD00BF83
:101DC0007C200020782000208C22002080B584B068
:101DD00000AF786039600023FB6018E07A68FB6828
:101DE00013441B781946114800F05AFA0346002B99
:101DF00006D1FB680133FB603B68013B3B6006E0BA
:101E00000B4B9B68002B02D1094800F07DF83B6822
:101E1000002BE3D1064B9B68002B02D1044800F055
:101E200073F8FB6818461037BD4680BD902100202E
:101E3000A820002080B582B000AF00237B60234B38
:101E40001B68002B34D015E0214B5B681B781946CA
:101E5000204800F025FA0346002B10D101237B60B7
:101E60001B4B5B6801331A4A5360194BDB68013B1B
:101E7000174AD360164BDB68002BE5D100E000BFAA
:101E8000134BDB68002B13D1134B1B78002B0FD0A7
:101E9000124B1B68002B0BD00C4B00221A600C4B12
:101EA00000221A610A4B0E4A5A600948FFF70CFCDF
:101EB0007B68002B06D00B4BDB68002B02D0094B54
:101EC000DB68984700BF0837BD4680BDA0210020D1
:101ED000A42100208C2200208020002078200020D7
:101EE000C8210020C022002080B582B000AF7860F9
:101EF000044B01221A60FFF79DFF00BF0837BD4663
:101F000080BD00BFA021002080B584B000AF786004
:101F10001F4B1B69002B30D11E4B1B78002B2CD084
:101F20001D4800F035FA0346002B26D10023FB6044
:101F300011E007F10B031946174800F0EAF90346D0
:101F4000002B0CD1F97A154AFB6813440A461A7023
:101F5000FB680133FB60FB683F2BEAD900E000BF60
:101F60000B4B0E4A5A60FB68094A9360084B0022EB
:101F7000DA600748FFF718FB06E0054B00229A607D
:101F8000034B00221A6100BF00BF1037BD4680BD61
:101F9000A82000208120002090210020CC200020BB
:101FA00080B584B000AF786039604FF0FF33FB60DC
:101FB0007B681B7803F01F03012B6AD17B689A882A
:101FC0003C4B1B789BB29A4263D17B685B78203B89
:101FD000032B58D801A252F823F000BFED1F0010C8
:101FE000FF1F0010112000106B20001000F0A0F85F
:101FF000F860FB68002B48D10123FB6045E000F04E
:10200000D3F8F860FB68002B41D10123FB603EE070
:102010007B685B8803F00103002B16D02648FFF78E
:10202000C3FA264B00221A60254B264A5A602448E0
:10203000FFF74AFB244B01221A60244B1B68002B3C
:1020400010D0224B1B6898470CE01F4B00221A60EF
:102050001B48FFF777FA1D4B5B68002B02D01B4B28
:102060005B6898470023FB6012E07B685B88002B6D
:1020700003D0174B01221A6002E0154B00221A60B0
:102080000023FB6004E000BF0FE000BF0DE000BFD5
:102090000BE0104B1B68002B07D00E4B1B680E4A41
:1020A0001268114678689847F860FB681846103740
:1020B000BD4680BD832000209C220020A02100205E
:1020C000A4210020C821002078200020C022002068
:1020D0007C200020D0220020D422002080B584B0B3
:1020E00000AF78600023FB607B68BB60BB681B6946
:1020F000002B13D10D4B9B68002B03D00B4B9B681F
:102100009847F860FB68B3F1FF3F03D10020FEF76A
:1021100003FC06E00020FEF76DFD02E00020FEF764
:10212000FBFB00BF1037BD4680BD00BFC0220020B2
:1021300080B500AF242200210D481CF095FD0C4B0A
:1021400000221A600A4B0B4A5A60094B07229A6018
:10215000074B094A5A61064B054A9A61044B002213
:102160001A770348FFF7B0FA0346184680BD00BF50
:102170008420002008000020DD20001080B584B0FD
:1021800000AF78607B68FB60FB681B69002B03D1A4
:102190000020FEF72FFD02E00020FEF7BDFB00BF90
:1021A0001037BD4680BD000080B500AF242200215D
:1021B0000D481CF059FD0C4B00221A600A4B0B4ACB
:1021C0005A60094B07229A60074B094A5A61064B2D
:1021D000054A9A61044B00221A770348FFF7E4F995
:1021E0000346184680BD00BF842000200800002060
:1021F0007D21001080B483B000AFEFF310833B600B
:102200003B687B607B68002B0CBF01230023DBB2A3
:102210001A46034B1A6000BF0C37BD4680BC70479E
:102220001C00002080B500AFFFF7E4FF054B1B68E2
:10223000002B01D072B600BF024B01225A6000BFD2
:1022400080BD00BF1C00002080B500AF064B1B689E
:10225000002B01D062B600BF034B00225A60FFF78B
:10226000C9FF00BF80BD00BF1C00002080B584B046
:1022700000AFF860B9607A60FFF7D4FFFB68002216
:102280009A60FB680022DA60FB68BA685A60FB68F3
:102290007A681A60FFF7D8FF00BF1037BD4680BDCF
:1022A00080B582B000AF78600B46FB707B68DA685F
:1022B0007B689B68013B9A420AD07B689B68002B35
:1022C00009D17B68DA687B681B68013B9A4202D1BE
:1022D0004FF0FF3319E0FFF7A5FF7B685A687B6872
:1022E000DB681344FA781A707B68DB685A1C7B68D9
:1022F000DA607B68DA687B681B689A4202D17B6887
:102300000022DA60FFF7A0FF002318460837BD4619
:1023100080BD80B582B000AF786039607B689A6814
:102320007B68DB689A4202D14FF0FF331AE0FFF777
:1023300079FF7B685A687B689B6813441A783B680E
:102340001A707B689B685A1C7B689A607B689A68E5
:102350007B681B689A4202D17B6800229A60FFF773
:1023600073FF002318460837BD4680BD80B582B094
:1023700000AF7860FFF756FF7B6800229A607B68A9
:102380000022DA60FFF760FF00BF0837BD4680BD5E
:1023900080B483B000AF78607B689A687B68DB6844
:1023A0009A420CBF01230023DBB218460C37BD460E
:1023B00080BC704780B584B000AF78607B68FB60FC
:1023C000FB681B69002B03D10020FEF713FC02E021
:1023D0000020FEF7A1FA24220021F8681CF044FC3A
:1023E00000BF1037BD4680BD80B500AF3822002148
:1023F00009481CF039FC2822002108481CF034FC54
:10240000074B00221A70002206490820FFF71EFA27
:102410000346184680BD00BFD8220020402300207C
:10242000682300201D25001080B485B000AF03464E
:10243000B9607A60FB73FB7B062B02D94FF0FF3348
:102440000BE0FB7B0749BA6841F83320FB7B054A68
:10245000DB0013447A685A60002318461437BD46DF
:1024600080BC7047D822002080B485B000AF0346FE
:10247000B9607A60FB73FB7B062B02D94FF0FF3308
:102480000DE0FB7B084A52F83320BB681A60FB7BE7
:10249000054ADB0013445A687B681A60002318461B
:1024A0001437BD4680BC7047D822002080B483B06A
:1024B00000AF03463960FB711346BB71FB79042BF7
:1024C00002D8BB79052B02D94FF0FF331DE0FB7911
:1024D000032B01D80023BB71FA79BB7913440D4952
:1024E0003A6841F82320FB79012B0DD1094B5B6839
:1024F000DB7903F04003002B06D0074B1B7843F039
:102500000103DAB2044B1A70002318460C37BD469B
:1025100080BC7047402300206823002080B586B02F
:1025200000AF03463960FB7107F10C031846FEF754
:1025300073FF0346002B02DA4FF0FF3350E02A4BC3
:102540005B68002B03D04FF0FF337B613AE03B7BAD
:1025500003F06003402B1FD0402B2FDC002B02D058
:10256000202B07D02AE007F10C03184600F040F8B2
:10257000786127E01D4B1B68002B09D01B4B1B68A3
:102580001A4A516807F10C0210469847786119E021
:102590004FF0FF337B6115E0144B9B68002B09D093
:1025A000124B9B68114AD16807F10C0210469847FC
:1025B000786107E04FF0FF337B6103E04FF0FF33BA
:1025C0007B6100BF7B69002B09DC7B69002B03D199
:1025D0000020FEF70FFB02E00020FEF79DF97B696B
:1025E00018461837BD4680BD1C230020D822002085
:1025F00080B584B000AF78607B685B780C2B54D8D2
:1026000001A252F823F000BF3D260010472600101B
:10261000AB26001051260010AB2600105B260010E0
:1026200069260010732600107B26001085260010F6
:102630008F26001099260010A3260010786800F05D
:102640003DF8F86035E0786800F0B2F8F86030E006
:10265000786800F027F9F8602BE07B685B88184603
:10266000FEF75AFFF86024E0786800F099F9F86006
:102670001FE04FF0FF33FB601BE0786800F098FA32
:10268000F86016E0786800F0CBFAF86011E078683E
:1026900000F0F4FAF8600CE0786800F03DFBF860B8
:1026A00007E04FF0FF33FB6003E04FF0FF33FB60C8
:1026B00000BFFB6818461037BD4680BDB0B584B07A
:1026C00000AF78607B685B88002B0DD17B68DB886E
:1026D000022B09D17B681B7803F01F03002B06D166
:1026E0007B689B88002B02D04FF0FF3353E07B6860
:1026F0001B7803F01F03022B19D17B689B8803F022
:102700000F031846FEF7AEF9F860FB68002B01DAFC
:10271000FB6840E0FB68002BCCBF01230023DBB249
:102720001A461F4B1A701E4B00225A7019E07B6824
:102730001B7803F01F03012B06D1194B00221A70DE
:10274000174B00225A700CE07B681B7803F01F03C4
:10275000002B06D1134B1A78114B1A70104B002224
:102760005A70114A114B14461D460FCD0FC40FCDA0
:102770000FC42B6823600C4B094A5A600A4B022293
:102780009A600948FEF710FFF860FB68002B01D142
:102790000123FB60FB6818461037BD46B0BD00BF83
:1027A00018230020682300201C23002090B9021069
:1027B00080B584B000AF78607B681B785BB2002B7B
:1027C00017DB7B68DB88002B13D17B685B88002BD1
:1027D00005D17B681B7803F01F03022B09D17B68AE
:1027E0005B88012B08D17B681B7803F01F03002B4B
:1027F00002D04FF0FF334CE07B685B88002B10D198
:102800007B689B88002B0CD07B689B8803F00F03B0
:102810001846FEF7E3F8F860FB68002B38DAFB682F
:1028200037E07B685B88012B19D11C4B1B6B002B9D
:1028300012D01A4B1B6B002178689847F860FB6830
:10284000002B01DAFB6824E0154B1B7823F0020310
:10285000DAB2134B1A701BE04FF0FF3319E07B68BC
:102860005B88022B11D10D4B1B6B002B0AD00B4B3D
:102870001B6B002178689847F860FB68002B07DA2B
:10288000FB6806E04FF0FF3303E04FF0FF3300E05A
:10289000002318461037BD4680BD00BFD822002057
:1028A0006823002080B584B000AF78607B68DB8847
:1028B000002B1DD17B685B88002B05D17B681B78C2
:1028C00003F01F03022B13D17B685B88012B05D11A
:1028D0007B681B7803F01F03002B09D17B685B88A2
:1028E000022B08D17B681B7803F01F03002B02D05A
:1028F0004FF0FF334CE07B685B88002B10D17B6886
:102900009B88002B0CD07B689B8803F00F03184634
:10291000FEF702F8F860FB68002B38DAFB6837E056
:102920007B685B88012B19D11B4B9B6A002B12D053
:10293000194B9B6A002178689847F860FB68002B68
:1029400001DAFB6824E0154B1B7843F00203DAB28E
:10295000124B1A701BE04FF0FF3319E07B685B8865
:10296000022B11D10C4B9B6A002B0AD00A4B9B6A9D
:10297000002178689847F860FB68002B07DAFB684D
:1029800006E04FF0FF3303E04FF0FF3300E0002399
:1029900018461037BD4680BDD8220020682300208D
:1029A000B0B586B000AF786000233B610023FB81A7
:1029B0007B685B881B0A9BB2013B062B00F2AC8054
:1029C00001A252F823F000BFE52900101B2A0010D5
:1029D000632A0010192B0010192B0010992A0010DF
:1029E000CF2A00107B681B7803F01F03002B03D154
:1029F0007B689B88002B02D00023FB81A1E0684B01
:102A00001B683B613B69002B02D10023FB8198E0EE
:102A10003B691B789BB2FB8193E07B681B7803F0DA
:102A20001F03002B03D17B689B88002B02D000235F
:102A3000FB8186E05A4B5B683B613B69002B02D10E
:102A40000023FB817DE03B6903331B789BB21B02B3
:102A50009AB23B6902331B789BB213449BB2FB8151
:102A60006FE07B681B7803F01F03002B53D17B685A
:102A70005B88DBB2052B0CDC7B685B88DBB2043344
:102A8000474A52F823303B613B691B789BB2FB817C
:102A900057E00023FB8154E07B681B7803F01F03A1
:102AA000002B03D17B689B88002B02D00023FB8185
:102AB00047E03B4BDB683B613B69002B02D10023C5
:102AC000FB813EE03B691B789BB2FB8139E07B6870
:102AD0001B7803F01F03002B03D17B689B88002B1E
:102AE00002D00023FB812CE02D4B9B683B613B69AE
:102AF000002B02D10023FB8123E03B6903331B78C9
:102B00009BB21B029AB23B6902331B789BB21344FF
:102B10009BB2FB8115E000BF224B1B68002B0DD040
:102B2000204B1B6807F10E0207F1100178689847E7
:102B30003B69002B04D10023FB8101E00023FB81D2
:102B400000BF7B68DA88FB899A4202D27B68DB8807
:102B5000FB81FB89002B03D14FF0FF337B6114E035
:102B6000114A124B14461D460FCD0FC40FCD0FC492
:102B70002B6823603B690C4A5360FB891A460A4B59
:102B80009A600948FEF710FD78617B69002B01D13E
:102B900001237B617B6918461837BD46B0BD00BF75
:102BA00040230020102300201C23002090B9021095
:102BB000B0B584B000AF78607B685B88002B07D12C
:102BC0007B689B88002B03D17B68DB88012B02D0BC
:102BD0004FF0FF3319E00F4A0F4B14461D460FCD3F
:102BE0000FC40FCD0FC42B6823600A4B0B4A5A60E9
:102BF000084B01229A600748FEF7D6FCF860FB6894
:102C0000002B01D10123FB60FB6818461037BD463D
:102C1000B0BD00BF1C23002090B902101423002077
:102C200080B582B000AF78607B689B88002B03D1B1
:102C30007B68DB88002B02D04FF0FF3316E00D4B92
:102C40001B69002B0CD00B4B1B690A4A52691146B9
:102C5000786898470346002B02DA4FF0FF3305E00F
:102C60007B685B88DAB2044B1A7000231846083779
:102C7000BD4680BDD822002014230020B0B584B00A
:102C800000AF78607B685B88002B03D17B68DB88B2
:102C9000012B02D04FF0FF3332E01B4B1B6A002B9D
:102CA00011D0194B1B6A184A526A11467868984726
:102CB000F860FB68002B01DAFB6821E0FB68DAB200
:102CC000124B1A7002E0114B00221A70104A114B7D
:102CD00014461D460FCD0FC40FCD0FC42B682360C3
:102CE0000B4B0A4A5A600A4B01229A600848FEF7C9
:102CF0005BFCF860FB68002B01D10123FB60FB68E3
:102D000018461037BD46B0BDD82200201823002039
:102D10001C23002090B9021080B582B000AF78600B
:102D20007B68DB88002B02D04FF0FF3318E00E4B9E
:102D30009B69002B0CD00C4B9B690B4AD269114646
:102D4000786898470346002B09DA4FF0FF3307E015
:102D50007B685B88002B02D04FF0FF3300E000233C
:102D600018460837BD4680BDD822002080B400AF89
:102D7000034B00221A7000BFBD4680BC704700BFE5
:102D80001423002080B582B000AF78607B68002BF0
:102D900043DB7B680F2B40DC23497A6813469B009A
:102DA00013449B000B441B68002B36D001211F48A5
:102DB00001F0F2FF0346002B02D06FF005032EE076
:102DC00019497A6813469B0013449B000B44002268
:102DD0001A6015497A6813469B0013449B000B4404
:102DE0000C331B6800221A600F497A6813469B0057
:102DF00013449B000B440C3319680B487A68134644
:102E00009B0013449B0003440C331B684A685A60C0
:102E1000064801F0E7FF002301E06FF002031846C7
:102E20000837BD4680BD00BF6C230020AC240020C5
:102E300080B582B000AF78607968044800F018F877
:102E4000034618460837BD4680BD00BF00900240CB
:102E500080B582B000AF78607968044800F034F83B
:102E6000034618460837BD4680BD00BF00900240AB
:102E700080B483B000AF786039603B68B3F1845FA1
:102E800003D33B680C4A934202D96FF002030DE072
:102E90007B6841F234221A647B68084A1A647B68B2
:102EA000074A1A647B68074A1A64002318460C37DD
:102EB000BD4680BC704700BFFF7F8010A35C7F3A97
:102EC000204FE3A1C1B2089680B483B000AF786010
:102ED00039603B68B3F1845F03D33B68074A934290
:102EE00002D96FF0020303E07B68054A1A640023ED
:102EF00018460C37BD4680BC704700BFFF7F80106E
:102F0000EFBEADDE80B485B000AF7860134B1B78A8
:102F1000002B1CD10023FB6013E00023BB600AE000
:102F20000F49FB685A01BB681344002241F8232073
:102F3000BB680133BB60BB681F2BF1DDFB6801334D
:102F4000FB60FB68032BE8DD044B01221A700023B1
:102F500018461437BD4680BC704700BFB02800201B
:102F6000B024002080B586B000AF78607B68002B6D
:102F700010D07B68012B0BD07B68022B06D07B68BE
:102F8000032B01D1204B06E0002304E01F4B02E09D
:102F90001F4B00E01F4BFB60F86800F071F978618F
:102FA0007969F86800F078F900233B6123E07B69D8
:102FB00003F00103002B18D017497B685A013B69C5
:102FC000134451F82330002B0FD013497B685A016A
:102FD0003B69134451F8233010487A6851013A692B
:102FE0000A4450F82220104698473B6901333B6160
:102FF0007B695B087B617B69002BD8D100BF00BF78
:103000001837BD4680BD00BF00B0004000A00040A2
:103010000090004000800040B0240020B026002036
:1030200080B582B000AF78607B68002B03D10020B0
:1030300001F011FF17E07B68012B03D1012001F0A3
:103040000AFF10E07B68022B03D1022001F003FF8E
:1030500009E07B68032B03D1262001F0FCFE02E08F
:103060006FF0020303E07868FFF74CFF0346184651
:103070000837BD4680BD000080B584B000AF7860E1
:103080007B681B68FB607B68997A7B685B681A4683
:10309000F86800F019F9B860BB68002B01D0BB6874
:1030A000B3E07B68197A7B685B681A46F86800F0C1
:1030B000A7F9B860BB68002B01D0BB68A5E07B68AE
:1030C0005B7A042B00F28F8001A252F823F000BF3C
:1030D000E53000101B3100104D3100107F31001021
:1030E000B3310010FB681A6E7B685B68DB431A40E3
:1030F000FB681A66FB685A6E7B685B68DB431A40A4
:10310000FB685A66FB68D3F8B8207B685B68DB43D2
:103110001A40FB68C3F8B82068E0FB681A6E7B6849
:103120005B681A43FB681A66FB685A6E7B685B68CB
:10313000DB431A40FB685A66FB68D3F8B8207B680B
:103140005B681A43FB68C3F8B8204FE0FB681A6E4F
:103150007B685B68DB431A40FB681A66FB685A6E43
:103160007B685B681A43FB685A66FB68D3F8B82033
:103170007B685B681A43FB68C3F8B82036E0FB68DD
:103180001A6E7B685B681A43FB681A66FB685A6EA6
:103190007B685B68DB431A40FB685A66FB68D3F8C0
:1031A000B8207B685B68DB431A40FB68C3F8B82033
:1031B0001CE0FB681A6E7B685B68DB431A40FB68A7
:1031C0001A66FB685A6E7B685B681A43FB685A662E
:1031D000FB68D3F8B8207B685B68DB431A40FB6868
:1031E000C3F8B82002E06FF002030EE07B681B7AA0
:1031F000002B01D1002308E07B68D97A7B685B68EB
:103200001A46F86800F072F8034618461037BD46B3
:1032100080BD00BF80B582B000AF7860396039688A
:10322000786800F075F8034618460837BD4680BD3B
:1032300080B582B000AF786039603968786800F096
:1032400075F800BF0837BD4680BD80B582B000AFBD
:10325000786039603968786800F075F800BF083721
:10326000BD4680BD80B582B000AF786039603968F6
:10327000786800F075F8034618460837BD4680BDEB
:1032800080B582B000AF7860786800F084F80346BB
:1032900018460837BD4680BD80B582B000AF786063
:1032A00039603968786800F069F800BF0837BD46B2
:1032B00080BD80B582B000AF78607868FFF752FEBD
:1032C00000BF0837BD4680BD80B584B000AFF86050
:1032D0000B467A60FB72FB7A7A681946F86800F050
:1032E00065F8034618461037BD4680BD80B584B0EA
:1032F00000AFF8600B467A60FB72FB7A7A68194679
:10330000F86800F0E3F8034618461037BD4680BD64
:1033100080B483B000AF786039607B685A6A3B68DC
:10332000134018460C37BD4680BC704780B483B04C
:1033300000AF786039607B683A68DA6100BF0C37AB
:10334000BD4680BC704780B483B000AF7860396000
:103350007B683A681A6200BF0C37BD4680BC704774
:1033600080B483B000AF786039607B689A693B684D
:10337000134018460C37BD4680BC704780B483B0FC
:1033800000AF786039607B683A689A6400BF0C3798
:10339000BD4680BC704780B483B000AF78607B6866
:1033A0001B6C18460C37BD4680BC704780B485B096
:1033B00000AFF8600B467A60FB72FB7A002B02D0FC
:1033C000012B0AD012E0FB68D3F8C0207B68DB43F6
:1033D0001A40FB68C3F8C0200BE0FB68D3F8C0209C
:1033E0007B681A43FB68C3F8C02002E06FF0020359
:1033F00000E0002318461437BD4680BC704700002B
:1034000080B485B000AFF8600B467A60FB72FB6851
:103410001A6B7B681A43FB681A63FB687A685A6008
:10342000FB7A032B48D801A252F823F03D34001058
:103430005F340010813400109D340010FB687A68FE
:103440005A61FB687A685A60FB687A681A67FB6899
:103450007A68DA67FB687A68C3F888202FE0FB682F
:103460007A681A61FB687A685A60FB687A681A673A
:10347000FB687A68DA67FB687A68C3F888201EE020
:10348000FB687A68C3F88820FB687A68DA67FB68AB
:103490007A681A67FB687A689A6010E0FB687A6855
:1034A000C3F88820FB687A68DA67FB687A68DA66AE
:1034B000FB687A689A6002E06FF0020300E0002384
:1034C00018461437BD4680BC704700BF80B485B035
:1034D00000AFF8600B467A60FB72FB7A032B53D87F
:1034E00001A252F823F000BFF93400101F3500107C
:1034F0004335001067350010FB68D3F8B0207B68B7
:10350000DB431A40FB68C3F8B020FB68D3F8B42053
:103510007B68DB431A40FB68C3F8B42046E0FB68D5
:10352000D3F8B0207B681A43FB68C3F8B020FB686F
:10353000D3F8B4207B68DB431A40FB68C3F8B4209F
:1035400034E0FB68D3F8B0207B68DB431A40FB68AB
:10355000C3F8B020FB68D3F8B4207B681A43FB683B
:10356000C3F8B42022E0FB68D3F8B0207B681A438C
:10357000FB68C3F8B020FB68D3F8B4207B681A431B
:10358000FB68C3F8B42011E0FB68D3F8B0207B6877
:10359000DB431A40FB68C3F8B020FB68D3F8B420C3
:1035A0007B68DB431A40FB68C3F8B420002318464D
:1035B0001437BD4680BC704780B582B000AF7860DC
:1035C000786800F031F8034618460837BD4680BDDC
:1035D00080B584B000AFF860B9607A607A68B96885
:1035E000F86800F03EF8034618461037BD4680BD27
:1035F00080B584B000AFF860B9607A607A68B96865
:10360000F86800F058F8034618461037BD4680BDEC
:1036100080B582B000AF78600821786800F0A6FB22
:1036200000BF0837BD4680BD80B483B000AF78606E
:103630007B68002B02D14FF0FF330DE07B681B6BE2
:1036400043F004027B681A6300BF7B681B6B03F0C6
:103650000403002BF9D1002318460C37BD4680BC6B
:10366000704780B487B000AFF860B9607A6000231B
:103670007B61FB68002B02D0BB68002B0BD14FF0A5
:10368000FF3313E0FB68D96A7B695A1C7A61BA6818
:103690001344CAB21A707A687B699A4205D9FB68EA
:1036A0005B6803F00203002BECD07B6918461C37E3
:1036B000BD4680BC704780B487B000AFF860B96089
:1036C0007A6000237B61FB68002B02D0BB68002B73
:1036D0000CD14FF0FF3314E07B695A1C7A61BA6851
:1036E00013441B78DBB21A46FB68DA627A687B699E
:1036F0009A4205D9FB685B6803F01003002BEBD0FE
:103700007B6918461C37BD4680BC704780B483B0C7
:1037100000AF78607B68DB6943F080027B68DA6128
:1037200000BF7B68DB6903F08003002BF9D100BF89
:1037300000BF0C37BD4680BC704780B483B000AF7B
:1037400078607B685B6A43F080027B685A6200BFE6
:103750007B685B6A03F08003002BF9D100BF00BFD8
:103760000C37BD4680BC704780B485B000AFF860B0
:10377000B9607A60FB68BA689A60FB687A681A6117
:1037800000BF1437BD4680BC7047000080B584B0D0
:1037900000AF786039607B680E4A934208D07B683E
:1037A0000D4A934201D1012303E04FF0FF3300E0C3
:1037B00000230A4A52F82330FB60FB68DB69002BC8
:1037C00004D0FB68DB693968F868984700BF103798
:1037D000BD4680BD00D0014000E00140B42800207B
:1037E00080B483B000AF78607B680022DA607B68C9
:1037F00000225A617B689A687B689A607B681A69C4
:103800007B681A617B680B4A934208D07B680A4A3E
:10381000934201D1012303E04FF0FF3300E0002386
:10382000064A002142F8231000BF0C37BD4680BC79
:10383000704700BF00D0014000E00140B4280020E4
:1038400080B586B000AF7860904A7B6852F823302C
:103850007B618F4A7B6852F823303B617B68002B89
:1038600006D07B68012B01D18A4B02E0002300E0E7
:10387000894BFB60894A7B6852F82330BB60FB6848
:103880009B6803F4FE43002B19D0FB689A68FB6821
:103890009A60FB681A69FB681A61FB680022DA60AB
:1038A000FB6800225A61F868FFF786FE6FF0080196
:1038B000F868FFF76BFFF868FFF792FFE2E0BB687C
:1038C000DB687A699A4243D2FB689B6803F0200365
:1038D000002B13D0BB689A687B69D118BB68DA6883
:1038E0007B69D31A1A46F868FFF782FE03461A4628
:1038F0007B6913447B61FB6820229A60BB68DB68AC
:103900007A699A4206D2FB68DB6843F02002FB68C2
:10391000DA6005E0FB68DB6823F02002FB68DA6010
:10392000BB68DB687A699A4212D1BB685B69002B7D
:103930000ED0FB681B6B43F00202FB681A63FB6846
:1039400001229A60FB68DB6843F00102FB68DA60E1
:10395000BB685B693A699A4219D2FB689B6803F0BD
:103960001103002B13D0BB681A693B69D118BB68DF
:103970005A693B69D31A1A46F868FFF729FE0346CD
:103980001A463B6913443B61FB6810229A60BB688E
:10399000DB687A699A423AD1BB685B693A699A42B4
:1039A00035D0FB689B6803F00103002B2FD0FB6828
:1039B00001229A603B69002B06D1BB685B685B0003
:1039C00043F00102FB68DA62BB685A693B69D31AAB
:1039D000B3F5807F03D9FB6800221A6205E0BB685B
:1039E0005A693B69D21AFB681A62BB685B693A691B
:1039F0009A4206D2FB68DB6843F01102FB68DA608A
:103A000005E0FB68DB6823F01102FB68DA60BB6845
:103A1000DB687A699A422BD1BB685B693A699A4242
:103A200026D1FB680022DA60FB6800225A61FB683D
:103A30009A68FB689A60FB681A69FB681A61BB6840
:103A40009B69002B06D0FB681B6B43F00202FB68EE
:103A50001A6305E0FB681B6B43F00402FB681A6302
:103A60000021F868FFF792FEF868FFF7B9FE09E059
:103A700006497B687A6941F8232005497B683A69E1
:103A800041F823201837BD4680BD00BFBC28002068
:103A9000C428002000E0014000D00140B4280020EC
:103AA00080B586B000AFF860B9607A603B60FB68B3
:103AB0009B687B613B6800221A607B6903F4FE43CC
:103AC000002B30D03B686FF008021A60BB68002BF7
:103AD00004D0BB683A680421F868984707226FF061
:103AE0007F41F868FFF740FEF868FFF726FEF868A8
:103AF000FFF70CFE7B6800221A607B68043300220B
:103B00001A60FB68964A934208D0FB68954A934234
:103B100001D1012303E04FF0FF3300E00023924A7C
:103B2000002142F823107B681B6803F01003002B70
:103B300006D17B6804331B6803F00103002B20D0FF
:103B40007B6903F01003002B0AD0BB68002B04D064
:103B5000BB6800220221F8689847FB6810229A602F
:103B6000FB681B6903F00103002B0AD0BB68002B24
:103B700004D0BB6800220621F8689847FB68012240
:103B80001A617B681A6848F220031340002B06D1A3
:103B90007B6804331B6803F00203002B4DD07B6964
:103BA00003F02003002B0AD0BB68002B04D0BB68B5
:103BB00000220321F8689847FB6820229A60FB687E
:103BC0001B6903F00203002B0AD0BB68002B04D052
:103BD000BB6800220521F8689847FB6802221A6139
:103BE0007B6903F40043002B27D03B6800221A6056
:103BF000BB68002B04D0BB683A680421F86898477A
:103C0000FB684FF400429A607B6800221A607B6870
:103C1000043300221A60FB68514A934208D0FB68C3
:103C2000504A934201D1012303E04FF0FF3300E0FB
:103C300000234D4A002142F823107B681B6803F0E3
:103C40000103002B37D07B6903F04003002B27D002
:103C50003B6800221A60BB68002B04D0BB683A683E
:103C60000421F8689847FB6840229A607B6800222C
:103C70001A607B68043300221A60FB68384A93425A
:103C800008D0FB68374A934201D1012303E04FF08B
:103C9000FF3300E00023344A002142F823100AE0F9
:103CA0007B6903F00103002B05D0FB6801229A60B9
:103CB0007B6808221A607B681B6803F00803002BEE
:103CC0004AD07B6903F00803002B45D07B6903F0E1
:103CD0004003002B07D07B6903F00103002B02D1C6
:103CE000FB6840229A60FB681B6803F40063002BAA
:103CF0001BD0BB68002B04D0BB6800220121F868F0
:103D00009847FB684FF480029A60FB6808229A602B
:103D1000FB684FF400429A607B684FF621721A608C
:103D20007B68043302221A6016E0BB68002B04D0C3
:103D3000BB6800220021F8689847FB684FF4000236
:103D40009A60FB6808229A607B6847F611721A60D5
:103D50007B68043301221A6000BF1837BD4680BD5E
:103D600000D0014000E00140B428002080B588B0B8
:103D700000AF786039607B681C4A934208D07B684A
:103D80001B4A934201D1012303E04FF0FF3300E0CF
:103D90000023FB61FB69002B23DB7B681B6803F0BE
:103DA0000203002B03D0F869FFF74AFD1AE0114A1D
:103DB000FB6952F82330BB617B68DB68FB607B6882
:103DC0005B693B6107F1140307F10C02B96978687C
:103DD000FFF766FEFA687B68DA603A697B685A61C9
:103DE00000E000BF2037BD4680BD00BF00D00140CD
:103DF00000E00140B428002080B582B000AF7860B8
:103E00007968044800F042F8034618460837BD4672
:103E100080BD00BF0060004080B582B000AF786018
:103E20007968044800F057F8034618460837BD463D
:103E300080BD00BF0060004080B500AF024800F0C8
:103E400070F80346184680BD0060004080B582B01F
:103E500000AF78607968044800F070F803461846AF
:103E60000837BD4680BD00BF0060004080B400AF91
:103E700000BF054B1B6903F00803002BF9D100BFFD
:103E800000BFBD4680BC70470060004080B582B076
:103E900000AF786039603B6803F026033B603B6805
:103EA000002B02D16FF0020311E0FFF7DFFF7B6808
:103EB0001A693B681A437B681A613B6823F0200348
:103EC0003B603B68002B01D0FFF7D0FF0023184672
:103ED0000837BD4680BD80B582B000AF78603960DC
:103EE0003B6803F026033B603B68002B02D16FF078
:103EF000020312E0FFF7BAFF7B681A693B68DB43F5
:103F00001A407B681A613B6823F020033B603B68E2
:103F1000002B01D0FFF7AAFF002318460837BD4643
:103F200080BD80B483B000AF78607B681B6903F00C
:103F3000D00318460C37BD4680BC704780B483B0B0
:103F400000AF786039607B681A693B6803F0D00382
:103F5000DB431A407B681A61002318460C37BD46C4
:103F600080BC704780B586B002AFF860B9607A60F7
:103F70003B603B68042B02DD6FF0020369E0374BC6
:103F80001B685B08FA699A4202D96FF0020360E08D
:103F9000FB68334A934214D0FB68324A93420ED0F6
:103FA000FB68314A934208D0FB68304A934201D102
:103FB000032307E04FF0FF3304E0022302E0012374
:103FC00000E00023032B36D801A252F823F000BFF3
:103FD000E13F0010FB3F00100F4000102340001095
:103FE0000D2001F08BF8062000F035FF2048FFF788
:103FF00043F82048FFF740F820E00E2001F07EF85B
:10400000072000F028FF1C48FFF736F816E00F20C5
:1040100001F074F8082000F01EFF1848FFF72CF894
:104020000CE0292001F06AF82E2000F014FF14485B
:10403000FFF722F802E06FF002030AE0FB69019348
:10404000BB6900933B687A68B968F86800F026F9A4
:10405000034618461037BD4680BD00BFB01F002084
:1040600000600440007004400080044000E00B4009
:10407000FCB9021008BA021014BA021050BA0210A9
:104080008CBA021080B582B000AF7860786800F01A
:10409000FDF97B681E4A934214D07B681D4A934207
:1040A0000ED07B681C4A934208D07B681B4A93421F
:1040B00001D1032307E04FF0FF3304E0022302E0C5
:1040C000012300E00023032B1AD801A252F823F0A9
:1040D000E1400010E9400010F1400010F9400010EC
:1040E000062000F0B8FE0EE0072000F0B4FE0AE063
:1040F000082000F0B0FE06E02E2000F0ACFE02E04A
:104100006FF0020300E0002318460837BD4680BD6B
:1041100000600440007004400080044000E00B4058
:1041200080B483B000AF78607B68174A934210D0A8
:104130007B68164A93420CD07B68154A934208D09C
:104140007B68144A934204D1134B1B6823F001038C
:1041500015E07B680C4A93420BD07B680B4A934274
:1041600007D07B680A4A934203D07B68094A93428E
:1041700003D1094B1B685B0801E06FF0020318468E
:104180000C37BD4680BC704700600440007004409E
:104190000080044000E00B40B01F002080B582B0DA
:1041A00000AF786039603968786800F035FA034606
:1041B00018460837BD4680BD80B582B000AF786034
:1041C00039603968786800F08FFA03461846083776
:1041D000BD4680BD80B582B000AF7860786800F0E1
:1041E000FBFA034618460837BD4680BD80B582B04D
:1041F00000AF78600B46FB70FB781946786800F0DA
:1042000001FB034618460837BD4680BD80B582B025
:1042100000AF78600B46FB70FB781946786800F0B9
:104220002BFB034618460837BD4680BD80B584B0D9
:1042300000AFF860B9607A607A68B968F86800F031
:104240006BFB034618461037BD4680BD80B582B073
:1042500000AF7860786800F0C1FB03461846083765
:10426000BD4680BD80B584B000AFF860B9607A60AB
:104270007A68B968F86800F0BFFB03461846103743
:10428000BD4680BD80B582B000AF7860786800F030
:1042900011FC034618460837BD4680BD80B586B080
:1042A00000AFF860B9607A603B60FB68714A934286
:1042B00014D0FB68704A93420ED0FB686F4A934259
:1042C00008D0FB686E4A934201D1032307E04FF008
:1042D000FF3304E0022302E0012300E000237B61BE
:1042E0007B69002B02DA6FF00203BEE065497A6950
:1042F00013469B001344DB000B4400221A60614903
:104300007A6913469B001344DB000B4408330022F8
:104310001A605C497A6913469B001344DB000B4426
:104320000C3301221A6057497A6913469B001344E3
:10433000DB000B44103300221A6052497A6913469D
:104340009B001344DB000B441C3300221A604D49D0
:104350007A6913469B001344DB000B442033002290
:104360001A6048497A6913469B001344DB000B44EA
:1043700014336FF001021A6042497A6913469B00B8
:104380001344DB000B4418336FF001021A603D49FF
:104390007A6913469B001344DB000B442733012248
:1043A0001A70FB6801225A60FB68374A1A61BB68C1
:1043B000002B06D0FB685B6843F00202FB685A6082
:1043C00005E0FB685B6823F00202FB685A60796ACB
:1043D000F868FFF7E3FE3B6AFF2B02D96FF0020398
:1043E00043E0FB68DA683B6A1B041A43FB68DA6047
:1043F000FB681A6AFB681A6222497A6913469B00B5
:104400001344DB000B4427331B78002B23D03B687D
:10441000012B05D1FB685B6843F48032FB685A606E
:104420003B68022B05D1FB685B6843F44032FB68B4
:104430005A603B68032B05D1FB685B6843F4E022BC
:10444000FB685A603B68042B05D1FB685B6843F44A
:104450007022FB685A607B68002B05D0FB68DB6824
:1044600043F40052FB68DA60002318461837BD4653
:1044700080BD00BF00600440007004400080044024
:1044800000E00B40CC2800200101010080B584B081
:1044900000AF78607B685B4A934214D07B685A4ACD
:1044A00093420ED07B68594A934208D07B68584AA1
:1044B000934201D1032307E04FF0FF3304E00223CE
:1044C00002E0012300E00023FB607B6800225A62C7
:1044D0007B681A6A7B681A627B685B6823F001025A
:1044E0007B685A607B68DB6923F040127B68DA6185
:1044F0004849FA6813469B001344DB000B441B68D1
:10450000002B2AD04349FA6813469B001344DB0072
:104510000B441B68BB60FA6813469B001344DB0026
:104520003C4A1344184600F05DFC3A49FA681346C9
:104530009B001344DB000B441B685B6A002B0CD010
:104540003449FA6813469B001344DB000B441B6894
:104550005B6A6FF00E01B86898477B6800225A606A
:104560007B6800229A607B680022DA607B68002208
:104570001A612849FA6813469B001344DB000B4478
:1045800014331B68002B16DB2249FA6813469B0084
:104590001344DB000B4414331B681846FEF7F2FB90
:1045A0001C49FA6813469B001344DB000B44143388
:1045B0006FF001021A601749FA6813469B00134412
:1045C000DB000B4418331B68002B16DB1149FA681B
:1045D00013469B001344DB000B4418331B6818463A
:1045E000FEF7D0FB0B49FA6813469B001344DB002F
:1045F0000B4418336FF001021A600023184610377D
:10460000BD4680BD0060044000700440008004404E
:1046100000E00B40CC28002080B586B000AF786069
:104620003960304B1B685B083A689A4202D96FF0D8
:10463000020353E07868FFF773FD0346BB60BA6876
:104640003B68B2FBF3F3BB60BB685B087B61BB6894
:104650005B083B610023FB60BB6803F00103002B98
:1046600010D07B6901337B610CE07B69DA0F134466
:104670005B107B613B69DA0F13445B103B61FB68A5
:104680000133FB607B690F2B02DDFB68072BECDD40
:10469000FB68082B03D10F233B610F237B617B68F1
:1046A0005B6923F0FF023B69DBB21A437B685A6106
:1046B0007B685B6923F47F427B691B029BB21A43D0
:1046C0007B685A617B685B6923F47022FB681B047A
:1046D00003F470231A437B685A6100231846183785
:1046E000BD4680BDB01F002080B485B000AF7860AB
:1046F00039603B68012B02D03B68102B02DD6FF064
:1047000002035AE07B682F4A934214D07B682E4AFA
:1047100093420ED07B682D4A934208D07B682C4A86
:10472000934201D1032307E04FF0FF3304E002235B
:1047300002E0012300E00023FB607B681B6B03F0B9
:104740000103002B37D12349FA6813469B00134419
:10475000DB000B440C331B68012B2CD17B685B689E
:1047600023F001027B685A6039681A48FA681346D8
:104770009B001344DB000344083319603B680F2B94
:104780000BDC7B68DB6823F470623B681B0203F47C
:1047900070631A437B68DA6005E07B68DB6823F4AA
:1047A00070627B68DA607B685B6843F001027B685B
:1047B0005A60002301E06FF0060318461437BD4627
:1047C00080BC7047006004400070044000800440DA
:1047D00000E00B40CC28002080B483B000AF7860AC
:1047E0007B68DB6803F47063002B01D1102304E0C5
:1047F0007B68DB681B0A03F00F0318460C37BD46C5
:1048000080BC704780B483B000AF78600B46FB700B
:104810007B68DB6823F430427B68DA60FB78032B2B
:1048200024D801A252F823F039480010474800105C
:10483000514800105F4800107B68DB6843F4004279
:104840007B68DA6012E07B68DA687B68DA600DE02A
:104850007B68DB6843F480527B68DA6006E07B6843
:10486000DB6843F400527B68DA6000BF002318461F
:104870000C37BD4680BC704780B483B000AF786011
:104880000B46FB70FB78032B3ED801A252F823F0B5
:10489000A1480010BB480010D5480010EF48001098
:1048A0007B68DB6823F001027B68DA607B68DB6889
:1048B00023F002027B68DA6027E07B68DB6843F064
:1048C00001027B68DA607B68DB6823F002027B68A8
:1048D000DA601AE07B68DB6823F001027B68DA604B
:1048E0007B68DB6843F002027B68DA600DE07B687E
:1048F000DB6843F001027B68DA607B68DB6843F0C9
:1049000002027B68DA6000E000BF002318460C3723
:10491000BD4680BC704700BF80B588B000AFF8606E
:10492000B9607A60BB68002B02D07B68002B01D194
:1049300000234FE0F868FFF789FCB861F868FFF7DB
:1049400049FC03467B617A68BB699A4201D9BB691D
:104950007B607B69082B03D97B6823F001037B60B4
:104960000023FB6132E07B69082B23D97B68032B92
:104970000CD9BA68FB691344FA6812681A607B683C
:10498000043B7B60FB690433FB610FE07B68012B18
:104990000CD9BA68FB691344FA68128892B21A807B
:1049A0007B68023B7B60FB690233FB617B68012B08
:1049B0000CD10EE0FB695A1CFA61BA681344FA681C
:1049C0001278D2B21A707B68013B7B607B68002B47
:1049D000C9D1FB6918462037BD4680BD80B483B07D
:1049E00000AF78607B68DB691B0E03F03F0318465D
:1049F0000C37BD4680BC704780B588B000AFF8600A
:104A0000B9607A60BB68002B02D07B68002B01D1B3
:104A100000234BE0F868FFF735FCB861F868FFF752
:104A2000D9FB03467B617A68BB699A4201D9BB69AD
:104A30007B607B69082B03D97B6823F001037B60D3
:104A40000023FB612EE07B69082B20D97B68032BB8
:104A50000CD9FB68B968FA690A4412681A607B6865
:104A6000043B7B60FB690433FB611BE07B68012B2B
:104A700018D9FB68B968FA690A44128892B21A8098
:104A80007B68023B7B60FB690233FB610AE0FB69E8
:104A90005A1CFA61BA6813441A78FB681A707B686A
:104AA000013B7B607B68002BCDD1FB69184620372A
:104AB000BD4680BD80B483B000AF78607B68DB69A1
:104AC0001B0A03F03F03C3F1200318460C37BD4611
:104AD00080BC704780B500AF0F4B1B6803F4803378
:104AE000002B16D00D4B1B68002B05DD0B4B1B68F4
:104AF000013B0A4A13600CE000F0F6F8084B1B6813
:104B0000002B06D0064B1B6800209847044B002260
:104B10001A6000BF80BD00BF10E000E0240000204C
:104B2000742900202DE9B04386B000AF7860364983
:104B3000896879613449096821F48031334801601A
:104B40003149096801F00101002911D12E496FF0A6
:104B50007F4048602C496FF07F4088602A490520DB
:104B600008606FF07F4179614FF08071396103E037
:104B700025494968013139617968002088468146B4
:104B80002349096800200A46034602FB09F008FB96
:104B900003F10144A8FB02454B191D461D4A4FF085
:104BA00000032046294619F003FB02460B46134634
:104BB000FB60FA683B69B2FBF3F31A46164B1A60C6
:104BC000FB683A69B3FBF2F2396901FB02F29B1A06
:104BD000BB60BA687B699A420CD30F4B1B680133E8
:104BE0000D4A13607A69BB68D21A3B6913440B4AB9
:104BF000136004E07A69BB68D31A084A136000BFE7
:104C00001837BD46BDE8B08310E000E070290020F1
:104C1000B01F002040420F00240000206C2900201B
:104C200080B582B000AF78603960104A3B6813608D
:104C30000F4B1B68002B02DD6FF0050312E07B6851
:104C4000002B01D100230DE07868FFF76BFF084BC4
:104C50001B68002B05DD074B1B68064A43F0020367
:104C60001360002318460837BD4680BD7429002014
:104C70002400002010E000E080B500AF164B1B6858
:104C8000002B0CDA154B1B68002B06D0134B1B684E
:104C900000209847114B00221A6000231AE00E4BA7
:104CA0001B68002B14D10E4B9A680E4B1B689A425E
:104CB0000ED800F019F8094B1B68002B06D0074BE3
:104CC0001B6800209847054B00221A60002301E072
:104CD0006FF00503184680BD2400002074290020D1
:104CE00010E000E06C29002080B500AF0A4B1B6883
:104CF000002B07D0084B1B686FF00F009847064B3E
:104D000000221A60054A064B1B681360054B4FF0E2
:104D1000FF321A6000BF80BD7429002010E000E05F
:104D2000702900202400002080B582B000AF786098
:104D3000164B1B68002B02DD6FF0050321E07B683A
:104D4000002B01D100231CE07868FFF7EBFE0AE09E
:104D50000F4B1B6803F48033002B04D00B4B1B68F4
:104D6000013B0A4A1360094B1B68002BF0DC00BFB3
:104D7000074B9A68074B1B689A42F9D8FFF7B4FFB4
:104D8000002318460837BD4680BD00BF2400002020
:104D900010E000E06C29002080B489B000AF78609A
:104DA00039607B68FB61FB6953E8003FBB61BB690D
:104DB000002B02D06FF005030FE03B687B617B683E
:104DC0003B6139697A6941E80023FB60FB68002B8D
:104DD000E7D1BFF35F8F00BF002318462437BD46DD
:104DE00080BC704780B483B000AF7860BFF35F8F42
:104DF00000BF7B6800221A6000BF0C37BD4680BC34
:104E0000704780B483B000AF0346FB71FB791F2B62
:104E10000FD9FB79203BFB714FF080439B6CFA79F3
:104E2000012101FA02F211464FF080420B439364D4
:104E30000BE04FF080435B6AFA79012101FA02F23C
:104E400011464FF080420B435362002318460C3743
:104E5000BD4680BC704780B483B000AF0346FB7191
:104E6000FB791F2B10D9FB79203BFB714FF080435E
:104E70009B6CFA79012101FA02F2D24311464FF0FC
:104E800080420B4093640CE04FF080435B6AFA79F8
:104E9000012101FA02F2D24311464FF080420B4049
:104EA0005362002318460C37BD4680BC7047000093
:104EB00080B584B000AF0346FB714FF080439B6820
:104EC00003F46063FB60FB79062B00F2968001A27D
:104ED00052F823F0F14E0010FB4F0010C54F0010A8
:104EE000274F0010514F00108B4F0010C54F00107E
:104EF0004FF080439B684FF0804243F480239360DF
:104F00004FF0806000F0DAF80346002B02D06FF01B
:104F10000903CFE04FF080439B684FF0804223F4B9
:104F2000606393606CE04FF0005000F0C7F80346F8
:104F3000002B02D06FF00903BCE04FF080439B6868
:104F400023F460634FF0804243F4C063936057E002
:104F50004FF080439B684FF0804243F400239360FE
:104F60004FF0006000F0AAF80346002B02D06FF06B
:104F700009039FE04FF080439B6823F460634FF088
:104F8000804243F4006393603AE04FF080439B68B3
:104F90004FF0804243F4801393604FF0805000F054
:104FA0008DF80346002B02D06FF0090382E04FF02A
:104FB00080439B6823F460634FF0804243F4206396
:104FC00093601DE04FF080439B684FF0804243F4B4
:104FD000003393604FF0007000F070F80346002B30
:104FE00002D06FF0090365E04FF080439B684FF0FB
:104FF000804223F46063936002E06FF0020359E0A3
:105000004FF4005000F05AF80346002B0ED04FF03A
:1050100080439B6823F46062FB6803F460634FF095
:10502000804113438B606FF0090343E0FB79062B4B
:105030003DD801A252F823F055500010AF50001097
:105040009D50001067500010795000108B500010D8
:105050009D5000104FF080439B684FF0804223F436
:10506000D013936023E04FF080439B684FF0804261
:1050700023F4F01393601AE04FF080439B684FF0E5
:10508000804223F4B013936011E04FF080439B689B
:105090004FF0804223F46023936008E04FF0804398
:1050A0009B684FF0804223F4E013936000BFFBF74E
:1050B000EDF8002318461037BD4680BD80B582B09C
:1050C00000AF786000214FF47A70FFF7A9FD4FF030
:1050D00080439A687B681340002B03D0FFF704FEDF
:1050E000002307E0FFF7C8FD034613F1060FEED0DB
:1050F0006FF0090318460837BD4680BD80B483B001
:1051000000AF0346FB71FB791F2B0FD9FB79203BC6
:10511000FB71FB7901229A404FF080435A6400BF33
:105120004FF080435B6C002BFAD10BE0FB7901223E
:105130009A404FF080435A6000BF4FF080435B6855
:10514000002BFAD1002318460C37BD4680BC7047AF
:1051500080B584B000AF3B460D21184600F01CF826
:105160003B789E2B94BF01230023DAB23B7803F0F7
:105170000F03092BCCBF01230023DBB21343DBB2A7
:10518000002B04D04FF080431B6DDBB200E03B7876
:1051900018461037BD4680BD80B588B000AF786036
:1051A00039603B680D2B02D06FF0020386E07B680C
:1051B000002B02D14FF0FF3380E04FF08450FDF719
:1051C00037FE4FF084531B68BB603E4B1B68FB608F
:1051D0003D4B1B683B613D4B1B687B613C4B1B6837
:1051E000BB613C4B1B68FB614FF08450FDF730FE08
:1051F000BB68DB0BDAB27B681A70BB68DA0D7B68C0
:105200000133D2B21A70BB68DA0F7B680233D2B2B4
:105210001A707B6802331978FB68DBB25B00DAB284
:105220007B6802330A43D2B21A70FB68DA097B68E2
:105230000333D2B21A70FB68DA0B7B680433D2B244
:105240001A70FB68DA0D7B680533D2B21A703B69BD
:10525000DA0B7B680633D2B21A703B69DA0D7B68D1
:105260000733D2B21A703B69DA0F7B680833D2B2C7
:105270001A707B68083319787B69DBB25B00DAB29D
:105280007B6808330A43D2B21A707B69DA097B68FB
:105290000933D2B21A707B69DA0B7B680A33D2B257
:1052A0001A707B69DA0D7B680B33D2B21A70BB6956
:1052B000DA0B7B680C33D2B21A7000231846203701
:1052C000BD4680BD04008010080080100C008010D6
:1052D000100080101400801080B500AF0320FFF78D
:1052E00090FD0023184680BD80B582B000AF786085
:1052F000786800F004F800BF0837BD4680BD80B470
:1053000083B000AF78607B680122DA6000BF0C37A1
:10531000BD4680BC704780B582B000AF786000BFEA
:10532000786800F019FA0346002BF9D0786800F08D
:10533000C7F9034618460837BD4680BD80B582B020
:1053400000AF78600B46FB7000BF786800F036FA5B
:105350000346002BF9D0FB781946786800F0BCF9B9
:10536000034618460837BD4680BD000080B584B0AE
:1053700000AF78603960786800F084F8F860FB6806
:10538000002B01D0FB6869E07B68364A93420ED05F
:105390007B68354A934208D07B68344A934201D1F6
:1053A000022305E04FF0FF3302E0012300E0002379
:1053B000022B14D0022B19DC002B02D0012B07D0BA
:1053C00014E02B48FDF758FE0920FFF744FD10E0DC
:1053D0002848FDF751FE0A20FFF73DFD09E0264869
:1053E000FDF74AFE2120FFF736FD02E06FF00203D1
:1053F00034E07B681B4A93420ED07B681A4A934282
:1054000008D07B68194A934201D1022305E04FF08E
:10541000FF3302E0012300E00023184A002142F894
:1054200023107B680F4A93420ED07B680E4A93424A
:1054300008D07B680D4A934201D1022305E04FF06A
:10544000FF3302E0012300E000230D4A002142F86F
:1054500023103968786800F09DFA03461846103723
:10546000BD4680BD002004400030044000400440A0
:10547000B4B90210CCB90210E4B9021078290020A6
:105480008429002080B582B000AF78607B681C4A18
:1054900093420ED07B681B4A934208D07B681A4A1D
:1054A000934201D1022305E04FF0FF3302E00123D4
:1054B00000E00023022B14D0022B19DC002B02D0B9
:1054C000012B07D014E00B20FFF718FE0920FFF78F
:1054D00098FC10E00C20FFF711FE0A20FFF791FC6A
:1054E00009E01C20FFF70AFE2120FFF78AFC02E0FA
:1054F0006FF0020300E0002318460837BD4680BD68
:1055000000200440003004400040044080B582B0D8
:1055100000AF786039603968786800F0D1FA0346E6
:1055200018460837BD4680BD80B582B000AF7860B0
:10553000786800F099FB034618460837BD4680BDE1
:1055400080B582B000AF786039603968786800F063
:105550000DFC034618460837BD4680BD80B582B0B5
:1055600000AF78600B46FB70FB781946786800F056
:105570001FFC034618460837BD4680BD80B582B083
:1055800000AF78600B46FB70FB781946786800F036
:1055900033FC034618460837BD4680BD80B584B04D
:1055A00000AFF8600B467A60FB72FB681A4A9342C0
:1055B0000ED0FB68194A934208D0FB68184A934200
:1055C00001D1022305E04FF0FF3302E0012300E0A8
:1055D0000023022B0ED0022B10DC002B02D0012B5B
:1055E00004D00BE00F48FDF747FD0AE00E48FDF739
:1055F00043FD06E00D48FDF73FFD02E06FF00203BA
:1056000006E0FB7A7A681946F86800F0CDFC03469C
:1056100018461037BD4680BD0020044000300440CD
:1056200000400440C0B90210D8B90210F0B902100D
:1056300080B582B000AF78607B680B4A93420AD095
:105640007B680A4A934206D07B68094A934202D09B
:105650006FF0020303E07868FFF75DFE034618462B
:105660000837BD4680BD00BF002004400030044024
:105670000040044080B582B000AF78600B46FB70FC
:105680007B680C4A93420AD07B680B4A934206D04F
:105690007B680A4A934202D06FF0020305E0FB7870
:1056A00019467868FFF74AFE034618460837BD4694
:1056B00080BD00BF00200440003004400040044092
:1056C00080B582B000AF7860786800F0BEFC034619
:1056D00018460837BD4680BD80B582B000AF7860FF
:1056E0000B46FB70FB781946786800F0C2FC034655
:1056F00018460837BD4680BD80B584B000AFF8605D
:10570000B9607A607A68B968F86800F0CAFC034644
:1057100018461037BD4680BD80B584B000AFF86034
:10572000B9607A607A68B968F86800F0E5FC034609
:1057300018461037BD4680BD80B584B000AFF86014
:10574000B9607A607A68B968F86800F0FFFC0346CF
:1057500018461037BD4680BD80B582B000AF786076
:105760007B680B4A93420AD07B680A4A934206D070
:105770007B68094A934202D06FF0020303E0786825
:1057800000F009FD034618460837BD4680BD00BF3E
:1057900000200440003004400040044080B584B044
:1057A00000AFF860B9607A607A68B968F86800F0AC
:1057B00000FD034618461037BD4680BD80B582B057
:1057C00000AF78607B680B4A93420AD07B680A4A34
:1057D000934206D07B68094A934202D06FF00203DD
:1057E00003E0786800F00AFD034618460837BD4616
:1057F00080BD00BF00200440003004400040044051
:1058000080B582B000AF786039603968786800F0A0
:1058100007FD034618460837BD4680BD80B582B0F7
:1058200000AF786039603968786800F017FD03468A
:1058300018460837BD4680BD80B582B000AF78609D
:105840007B680B4A93420AD07B680A4A934206D08F
:105850007B68094A934202D06FF0020303E0786844
:1058600000F01DFD034618460837BD4680BD00BF49
:1058700000200440003004400040044080B582B065
:1058800000AF786039603968786800F013FD00BFB8
:105890000837BD4680BD80B582B000AF7860396002
:1058A0003968786800F014FD00BF0837BD4680BD38
:1058B00080B582B000AF786039603968786800F0F0
:1058C00018FD00BF0837BD4680BD000080B582B01E
:1058D00000AF78607B680B4A93420AD07B680A4A23
:1058E000934206D07B68094A934202D06FF00203CC
:1058F00003E0786800F00FFD034618460837BD4600
:1059000080BD00BF0020044000300440004004403F
:1059100080B582B000AF7860786800F007FD03467C
:1059200018460837BD4680BD80B582B000AF7860AC
:1059300039603968786800F039FE03461846083740
:10594000BD4680BD80B582B000AF786039603968EF
:10595000786800F0EDFD034618460837BD4680BD67
:1059600080B582B000AF786039603968786800F03F
:10597000A1FD034618460837BD4680BD80B582B0FC
:1059800000AF7860786800F053FE00BF0837BD466E
:1059900080BD000080B584B000AF7860396001211F
:1059A0007868FFF72DFFF860FB68002B01D0FB68DB
:1059B0007AE002217868FFF731FFF860FB68002B7E
:1059C00001D0FB6870E008217868FFF7B9FDF86046
:1059D000FB68002B01D0FB6866E000217868FFF7C8
:1059E000CDFDF860FB68002B01D0FB685CE0002176
:1059F0007868FFF7B3FDF860FB68002B01D0FB6807
:105A000052E07B681B6843F001027B681A603968CA
:105A10007868FFF77BFD7B68254A93420ED07B6850
:105A2000244A934208D07B68234A934201D102233F
:105A300005E04FF0FF3302E0012300E00023BB60EC
:105A40001E49BA6813469B0013449B000B440C3359
:105A50004FF0FF321A601949BA6813469B0013448D
:105A60009B000B4408334FF0FF321A601349BA68A9
:105A700013469B0013449B000B4400221A600F49FD
:105A8000BA6813469B0013449B000B440433002266
:105A90001A600A49BA6813469B0013449B000B44E2
:105AA000103300221A70002318461037BD4680BDFF
:105AB000002004400030044000400440A829002099
:105AC00090B587B000AF786039607B681B6803F4DD
:105AD0000043002B03D04FF4E1037B6103E0614BF3
:105AE0001B685B087B61786918F0B2F80446386877
:105AF00018F0AAF803461946204618F0B1F90346F3
:105B0000BB6008233B6117E0386918F0A1F8034631
:105B10001946B86818F0A4F903464FF07E511846AC
:105B200018F088FA0346002B03D03B695B103B61F9
:105B300005E03B695B003B613B69802BE4DD3B6931
:105B4000802B01DD80233B613B69072B02DC6FF07A
:105B5000020383E0386918F07BF803461946B868F9
:105B600018F07EF90346BB60B86818F08BFA03465C
:105B7000184618F06DF803461946B86817F0B2FFDA
:105B800003464FF08641184618F0B6F8034618460B
:105B900018F078FA0346FB60FB68032B03DDFB6813
:105BA000033BFB6002E0FB680333FB603B69802B37
:105BB00021D03B69802B21DC3B69402B18D03B690D
:105BC000402B1BDC3B69202B0FD03B69202B15DCC5
:105BD0003B69082B03D03B69102B03D00EE0042354
:105BE0003B610EE003233B610BE002233B6108E0D5
:105BF00001233B6105E000233B6102E06FF00703F6
:105C00002CE03B691B043B617B685B6923F44032F9
:105C10003B6903F440331A437B685A617B685B69D4
:105C200023F47F6424F00F04B86818F02BFA0346BD
:105C3000C3F30B0344EA03027B685A617B689B69E8
:105C400023F47F6323F00F03FA68C2F30B021A43B5
:105C50007B689A617868FFF767FC034618461C3733
:105C6000BD4690BDB01F002080B586B000AF786003
:105C700000237B614FF00003FB604FF000033B61AA
:105C80007B681B6803F40043002B03D04FF4E1034F
:105C90007B6103E0324B1B685B087B617B685B695F
:105CA000C3F30B03184617F0CFFF03461946F868F5
:105CB00017F01AFF0346FB607B689B69C3F30B0375
:105CC000184617F0C1FF03463B612649386918F0B2
:105CD000CFF90346002B0DD02349386918F0B4F9E9
:105CE0000346002B06D01F49386917F0FBFE034618
:105CF0003B6105E01B49386917F0F6FE03463B613E
:105D00004FF08641386918F0ABF803461946F86839
:105D100017F0EAFE0346FB607B685B6903F44033DF
:105D2000C3F10703012202FA03F3184617F090FFAC
:105D300003461946F86817F0DFFF0346FB607869F1
:105D400017F086FF0346F968184618F089F80346ED
:105D5000184618F097F9034618461837BD4680BD17
:105D6000B01F0020000040400000C04080B483B05D
:105D700000AF786039603B68042B02DD3B68082B7C
:105D800002DD6FF002030EE03B68053B1B023B6047
:105D90007B681B6823F440723B6803F440731A432A
:105DA0007B681A60002318460C37BD4680BC7047DC
:105DB00080B483B000AF78600B46FB70FB78002B9B
:105DC00002D0012B07D00DE07B681B6823F48062B2
:105DD0007B681A6009E07B681B6843F480627B681B
:105DE0001A6002E06FF0020300E0002318460C374F
:105DF000BD4680BC7047000080B483B000AF7860BF
:105E00000B46FB70FB780C2B00F2C58001A252F808
:105E100023F000BF495E0010575E0010A35E001023
:105E2000F75E00104B5F0010575E00107D5E0010A3
:105E3000A35E0010CD5E0010F75E0010215F001021
:105E40004B5F0010715F00107B681B6823F002023B
:105E50007B681A60A2E07B681B6843F002027B68E3
:105E60001A607B681B6823F00C027B681A607B68F1
:105E70001B6823F010027B681A608FE07B681B6848
:105E800043F002027B681A607B681B6823F00C02F7
:105E90007B681A607B681B6843F010027B681A609D
:105EA0007CE07B681B6843F002027B681A607B68B9
:105EB0001B6823F00C0343F004027B681A607B68C4
:105EC0001B6823F010027B681A6067E07B681B6820
:105ED00043F002027B681A607B681B6823F00C03A6
:105EE00043F004027B681A607B681B6843F0100271
:105EF0007B681A6052E07B681B6843F002027B6893
:105F00001A607B681B6823F00C0343F008027B686F
:105F10001A607B681B6823F010027B681A603DE002
:105F20007B681B6843F002027B681A607B681B6811
:105F300023F00C0343F008027B681A607B681B683F
:105F400043F010027B681A6028E07B681B6843F00E
:105F500002027B681A607B681B6843F00C027B6856
:105F60001A607B681B6823F010027B681A6015E0DA
:105F70007B681B6843F002027B681A607B681B68C1
:105F800043F00C027B681A607B681B6843F01002C8
:105F90007B681A6002E06FF0020300E000231846FD
:105FA0000C37BD4680BC704780B485B000AFF86048
:105FB0000B467A60FB72FB7A022B1AD0022B25DC8F
:105FC000002B02D0012B07D020E0FB681B6823F4D4
:105FD0000062FB681A601CE0FB681B6843F4006207
:105FE000FB681A60FB681B6823F48052FB681A6028
:105FF0000FE0FB681B6843F40062FB681A60FB68F3
:106000001B6843F48052FB681A6002E06FF00203E1
:1060100016E07B68002B02DD7B68202B02DD6FF031
:1060200002030DE07B681B047B60FB685B6823F464
:106030007C127B6803F47C131A43FB685A600023CC
:1060400018461437BD4680BC704780B483B000AF9B
:1060500078607B689B6803F01003002B02D06FF020
:106060000C0301E07B68DB6918460C37BD4680BC39
:10607000704780B483B000AF78600B46FB707B68DC
:106080009B6803F08003002B02D06FF00B0303E04A
:10609000FA787B68DA61002318460C37BD4680BC6D
:1060A000704780B586B000AFF860B9607A600023B1
:1060B0007B6114E0F868FFF7BBFA38613B69002B9D
:1060C00004DA7B687A691A603B6911E07B69BA6817
:1060D00013443A69D2B21A707B6901337B617B68E1
:1060E0001B687A699A42E5DB7B687A691A6000234B
:1060F00018461837BD4680BD80B586B000AFF86041
:10610000B9607A6000237B6113E07B69BA6813444D
:106110001B781946F868FFF7ADFA38613B69002B28
:1061200004D07B687A691A603B690BE07B690133B4
:106130007B617B681B687A699A42E6DB7B687A69D7
:106140001A60002318461837BD4680BD80B487B05A
:1061500000AFF860B9607A6000237B610FE0FB68F4
:106160009B6803F01003002B0ED1FB68D969BA6855
:106170007B691344CAB21A707B6901337B617A6907
:106180007B689A42EBD300E000BF7B6918461C375E
:10619000BD4680BC704780B483B000AF78607B6838
:1061A0009B681B0A03F03F0318460C37BD4680BCB2
:1061B000704780B487B000AFF860B9607A600023A0
:1061C0007B610FE0FB689B6803F08003002B0ED11E
:1061D000BA687B6913441B781A46FB68DA617B69ED
:1061E00001337B617A697B689A42EBD300E000BFA0
:1061F0007B6918461C37BD4680BC704780B485B0AB
:1062000000AF78607B689B681B0C03F03F03FB606A
:10621000FB68C3F1200318461437BD4680BC7047A5
:1062200080B483B000AF786039603B68002B02D047
:106230003B68202B02D96FF002030AE07B685B68A1
:1062400023F03F023B6803F03F031A437B685A6028
:10625000002318460C37BD4680BC704780B483B01D
:1062600000AF786039603B68002B02D03B68202B80
:1062700002D96FF002030DE03B681B023B607B68B4
:106280005B6823F47C523B6803F47C531A437B68BD
:106290005A60002318460C37BD4680BC704780B456
:1062A00083B000AF78607B681B6918460C37BD4629
:1062B00080BC704780B483B000AF786039607B6881
:1062C0003A681A61002318460C37BD4680BC7047F7
:1062D00080B483B000AF786039607B68DA683B686F
:1062E0001A437B68DA60002318460C37BD4680BC31
:1062F000704780B483B000AF786039607B68DA683B
:106300003B68DB431A407B68DA60002318460C3791
:10631000BD4680BC704780B483B000AF78607B68B6
:106320009B6818460C37BD4680BC704780B586B068
:1063300000AF78607B681B68594A934210D07B6835
:106340001B68584A934209D07B681B68564A93429F
:1063500001D1022305E04FF0FF3302E0012300E00A
:1063600000237B617B68DB68002B3ED04F4A7B6952
:1063700052F82330002B02D06FF006038CE07B68CC
:106380005B68002B02D16FF0020385E07B6800227E
:106390005A6146497B697A6841F823207B681B680B
:1063A00040211846FFF777FA7B681B681846FFF70D
:1063B00005FA38617B68DA687B685B69D31A3A69E9
:1063C000934228BF13463B617B6818687B685A6814
:1063D0007B685B6913443A691946FFF7DFF90246A7
:1063E0007B685B691A447B685A617B681B69002B78
:1063F00051D02F4A7B6952F82330002B02D06FF026
:10640000060349E07B689B68002B09D17B681B6809
:106410004FF0FF311846FFF74BFA6FF002033BE0F5
:106420007B6800229A6122497B697A6841F82320BF
:106430007B681B680B211846FFF72DFA7B681B68E9
:1064400010211846FFF727FA7B681B681846FFF7EC
:1064500083F9F8607B681A697B689B69D31AFA68CC
:10646000934228BF1346FB607B6818687B689A6874
:106470007B689B691344FA681946FFF75DF9024689
:106480007B689B691A447B689A617B681B68102152
:106490001846FFF7F3F9002318461837BD4680BDAC
:1064A00000200440003004400040044090290020B7
:1064B0009C29002080B584B000AF786039607B688B
:1064C000174A93420ED07B68164A934208D07B68E5
:1064D000154A934201D1022305E04FF0FF3302E059
:1064E000012300E00023FB60104AFB6852F82330D0
:1064F000002B02D16FF006030EE00C4AFB6852F845
:106500002330BB60BB68DB69002B04D0BB68DB6950
:106510003968B8689847002318461037BD4680BDD3
:106520000020044000300440004004409C2900202A
:1065300080B584B000AF786039607B68174A9342B9
:106540000ED07B68164A934208D07B68154A934266
:1065500001D1022305E04FF0FF3302E0012300E008
:106560000023FB60104AFB6852F82330002B02D155
:106570006FF006030EE00C4AFB6852F82330BB6054
:10658000BB68DB69002B04D0BB68DB693968B8687D
:106590009847002318461037BD4680BD00200440B0
:1065A00000300440004004409029002080B584B0B1
:1065B00000AF786039607B68184A93420ED07B68E0
:1065C000174A934208D07B68164A934201D10223AE
:1065D00005E04FF0FF3302E0012300E00023BB6041
:1065E00039687868FFF7AEF9F860FB68002B01D0D6
:1065F000FB680FE00C4ABB6852F823200B49BB68CC
:1066000051F823309A4204D039687868FFF7A8F926
:10661000F860FB6818461037BD4680BD0020044076
:106620000030044000400440902900209C290020B4
:1066300080B588B000AF78607B68904A93420ED0F6
:106640007B688F4A934208D07B688E4A934201D17F
:10665000022305E04FF0FF3302E0012300E00023B6
:10666000FB617868FFF7E8F8B8617B68DA68BB69B6
:10667000134003F00B03002B15D05B217868FFF764
:1066800017F96FF008017868FFF74EF97E4AFB6949
:10669000002142F823107D4AFB69002142F82310B3
:1066A0006FF00303E6E0794AFB6952F823307B611F
:1066B000BB6903F04003002B2DD07B69002B2AD04F
:1066C0007B69DB68002B26D07B691B681846FFF7C7
:1066D00075F838617B69DA687B695B69D31A3A6956
:1066E000934228BF13463B617B6918687B695A68EF
:1066F0007B695B6913443A691946FFF74FF8024614
:106700007B695B691A447B695A617B691B6840211C
:106710001846FFF7B3F85C4AFB6952F823307B61F7
:10672000BB6903F01003002B2DD07B69002B2AD00E
:106730007B691B69002B26D07B691B681846FFF715
:106740000BF8F8607B691A697B699B69D31AFA6850
:10675000934228BF1346FB607B6918687B699A687F
:106760007B699B691344FA681946FEF7E5FF024608
:106770007B699B691A447B699A617B691B6810215C
:106780001846FFF77BF8404AFB6952F823203F493F
:10679000FB6951F823309A4227D17B69002B22D024
:1067A0007B699A697B691B699A421CD17B695A692A
:1067B0007B69DB689A4216D15B217868FFF778F82D
:1067C000314AFB69002142F82310304AFB6900215D
:1067D00042F823107B69DB69002B04D07B69DB69FD
:1067E000002178699847002344E0284AFB6952F861
:1067F00023307B617B69002B19D07B695A697B69E7
:10680000DB689A4213D140217868FFF751F81F4A9C
:10681000FB69002142F823107B69DB69002B04D05F
:106820007B69DB69002178699847002322E0164ADA
:10683000FB6952F823307B617B69002B19D07B699F
:106840009A697B691B699A4213D11B217868FFF70B
:106850002FF80D4AFB69002142F823107B69DB69A0
:10686000002B04D07B69DB690021786998470023FD
:1068700000E0002318462037BD4680BD00200440BC
:1068800000300440004004409C2900209029002052
:1068900080B5B2B000AF012387F8843002233B6794
:1068A0001A237B67002387F87830504BFB6707F18A
:1068B0008403C7F8803007F1700207F18C0311469A
:1068C000184604F00DF9C7F8C400D7F8C430002BFF
:1068D00002D0D7F8C43084E0012387F86C3003235A
:1068E000BB650523FB65002387F860303F4B7B6663
:1068F00007F16C03BB6603237B640423BB640023A2
:1069000087F84C30394B3B6507F16C037B6507F129
:10691000300300221A605A609A60DA601A6101231B
:106920003B63012387F8353007F110032022002153
:10693000184618F099F92E4B7B6103237B762D4B7B
:10694000FB6107F13003BB6207F158037B6007F17D
:106950004403BB6007F11003FB6007F188003B1D97
:106960000ECB04F07EFEC7F8C400D7F8C430002B6D
:1069700002D0D7F8C43034E007F190031E4918461E
:1069800018F080FDD7F88C300121184604F054F936
:10699000C7F8C400D7F8C430002B02D0D7F8C430F1
:1069A0001FE0D7F8883007F190021146184604F02E
:1069B000CBFCC7F8C400D7F8C430002B02D0D7F8FE
:1069C000C4300EE0D7F88C300021184604F034F9BA
:1069D000C7F8C400D7F8C430002B02D0D7F8C430B1
:1069E000FFE71846C837BD4680BD00BFC8C90210C2
:1069F00040420F006CCA02103CBB021080B588B048
:106A000000AF0023FB6100F041FCF861FB69002B43
:106A100001D0FB6998E000F0F5FBF861FB69002B01
:106A200001D0FB6990E0FB69002B0ED10023BB6114
:106A300007F1180319464FF4906000F097FAF861D7
:106A4000FB69002B01D00B23FB61414BBB6107F1BC
:106A500018031946602000F035FAF861FB69002B35
:106A600002D00523FB6113E04FF40063BB61BB69F7
:106A700043F00203BB6107F11803194640F281405D
:106A800000F074FAF861FB69002B01D00623FB616A
:106A9000FB69002B0FD14FF44063BB6107F1180372
:106AA000194640F2AF4000F061FAF861FB69002B33
:106AB00001D00723FB61FB69002B10D10023BB61D0
:106AC000BB69BB6107F11803194640F29A4000F018
:106AD0004DFAF861FB69002B01D00923FB61FB69CA
:106AE000002B07D100F094F8F861FB69002B01D06E
:106AF0000C23FB61FB69002B07D100F064F8F861FF
:106B0000FB69002B01D00A23FB61FB69002B0ED12E
:106B10000123BB6107F1180319464FF4906000F0A0
:106B200025FAF861FB69002B01D00B23FB613B1DAB
:106B30001A46012140F2A44000F0E8FABB88194649
:106B4000044818F0F7F8FB6918462037BD4680BDA9
:106B5000800002005CBB021080B584B000AF00234F
:106B6000FB604FF41803BB60FB68002B0DD10023C2
:106B70007B603B1D19464FF4906000F0F7F9F86018
:106B8000FB68002B01D00B23FB6007F108031946BB
:106B900040F2024000F096F9F860FB68002B0DD13E
:106BA00001237B603B1D19464FF4906000F0DEF935
:106BB000F860FB68002B01D00B23FB60FB681846D4
:106BC0001037BD4680BD80B582B000AF00237B602A
:106BD00000233B603B46194640F2054000F072F945
:106BE00078607B68002B0ED14FF408033B603B4676
:106BF000194640F2054000F065F978607B68002B8B
:106C000001D00A237B607B6818460837BD4680BDEB
:106C100080B582B000AF00237B6000237B807B883F
:106C200023F010039BB27B80BB1C19464FF4946089
:106C300000F09CF978607B68002B0ED14FF49E53D6
:106C40007B80BB1C19464FF4946000F08FF978608C
:106C50007B68002B01D00C237B607B68002B0CD160
:106C6000BB1C1A4601214FF4946000F04FFA786083
:106C70007B68002B01D00C237B607B68002B10D13C
:106C80007B8843F010039BB27B80BB1C19464FF4FA
:106C9000946000F06BF978607B68002B01D00C23C6
:106CA0007B607B6818460837BD4680BD80B586B0DE
:106CB00000AF78600B467B8000237B610023FB6084
:106CC00000233B6107F10C031A4601214FF41B70AE
:106CD00000F0A0F978617B69002B17D1FB68002BCD
:106CE00003D140F601033B6102E040F601433B6102
:106CF0003B699BB279887A68184600F007FA786198
:106D00007B69002B04D00D237B6101E00D237B61A7
:106D10007B6918461837BD4680BD80B584B000AF8A
:106D200078600B467B800023FB6000237B810FE0B3
:106D30007B8903F26B2398B27B899B007A681344AA
:106D40001A46012100F066F9F8607B8901337B81E6
:106D50007A897B889A42EBD3FB68002B01D0102301
:106D6000FB60FB6818461037BD4680BD80B584B017
:106D700000AF78600B467B800023FB607B887A68DD
:106D8000194640F2326000F045F9F860FB68002BCC
:106D900001D00F23FB60FB6818461037BD4680BD4D
:106DA00080B584B000AF78600B467B800023FB6029
:106DB0007B887A68194640F2366000F02BF9F8605B
:106DC000FB68002B01D00E23FB60FB6818461037D0
:106DD000BD4680BD80B584B000AF78600B467B8037
:106DE00013463B800023FB6000237B813B88002B04
:106DF00003D140F282437B8102E04FF491637B81B7
:106E000000233B810FE07A893B89134498B23B8988
:106E10005B007A6813441A46012100F077F9F860A4
:106E20003B8901333B813A897B889A42EBD3FB68EB
:106E3000002B01D01123FB60FB6818461037BD46BC
:106E400080BD80B584B000AF78600023FB60002374
:106E5000BB607A68012140F2034000F0DBF8F86083
:106E60007B681B68BB60BB6803F40073002B07D012
:106E700007F10803194640F2034000F023F8F860D8
:106E8000FB68002B01D01323FB60FB68184610370A
:106E9000BD4680BD80B584B000AF78600023FB6044
:106EA0007A68012140F26A2000F0B4F8F860FB68CB
:106EB000002B01D01223FB60FB6818461037BD463B
:106EC00080BD000080B5ADF5616D00AF024607F5ED
:106ED0006163A3F56163196007F56163A3F60A6353
:106EE0001A800023C7F80C3E07F56163A3F60A6316
:106EF0001B881B099BB2DAB207F56163A3F608632E
:106F00001A7007F56163A3F60A631B881B01DAB2E6
:106F100007F56163A3F608635A7007F56163A3F58B
:106F200061630422042118680CF0A1FA07F561637B
:106F3000A3F561631B681B681A4607F56163A3F636
:106F40000863C3F80220084B1B6807F108010622FA
:106F5000184604F09FF8C7F80C0ED7F80C3E1846F8
:106F600007F56167BD4680BDE429002080B5ADF519
:106F7000616D00AF024607F56163A3F561631960B7
:106F800007F56163A3F60A631A800023C7F80C3E75
:106F900007F56163A3F60A631B881B099BB2DAB28B
:106FA00007F56163A3F608631A7007F56163A3F63A
:106FB0000A631B881B01DAB207F56163A3F6086355
:106FC0005A7007F56163A3F5616302220221186814
:106FD0000CF04DFA07F56163A3F561631B681B882C
:106FE0009AB207F56163A3F608635A80084B1B68E1
:106FF00007F108010422184604F04CF8C7F80C0EFB
:10700000D7F80C3E184607F56167BD4680BD00BF46
:10701000E429002080B5ADF5616D00AF07F561632F
:10702000A3F561631A6007F56163A3F60A6302467C
:107030001A8007F56163A3F60C630A461A800023E1
:10704000C7F80C3E07F56163A3F60A631B881B09AA
:107050009BB2DAB207F56163A3F608631A7007F50D
:107060006163A3F60A631B881B01DBB20833DAB243
:1070700007F56163A3F608635A7007F56163A3F629
:107080000C631B889A0007F108030233002118469D
:1070900017F0EAFD1C4B186807F56163A3F60C6353
:1070A0001B889B009BB202339AB207F10803194672
:1070B00003F0F0FFC7F80C0E07F56163A3F60C634D
:1070C0001B889B001A4607F10803991C07F56163AA
:1070D000A3F56163186817F02DFD07F56163A3F64A
:1070E0000C631B889B00194607F56163A3F5616378
:1070F000042218680CF0BBF9D7F80C3E184607F5C7
:107100006167BD4680BD00BFE429002080B5ADF5B4
:10711000616D00AF07F56163A3F561631A6007F560
:107120006163A3F60A6302461A8007F56163A3F65A
:107130000C630A461A800023C7F80C3E07F561630A
:10714000A3F60A631B881B099BB2DAB207F56163D9
:10715000A3F608631A7007F56163A3F60A631B8838
:107160001B01DBB20833DAB207F56163A3F60863EB
:107170005A7007F56163A3F60C631B885A0007F188
:10718000080302330021184617F06EFD1C4B1868E7
:1071900007F56163A3F60C631B8801339BB25B00A8
:1071A0009AB207F10803194603F074FFC7F80C0EF2
:1071B00007F56163A3F60C631B885B001A4607F1B1
:1071C0000803991C07F56163A3F56163186817F05C
:1071D000B1FC07F56163A3F60C631B885B001946DD
:1071E00007F56163A3F56163022218680CF03FF9AB
:1071F000D7F80C3E184607F56167BD4680BD00BF55
:10720000E429002080B582B000AF00237B603B46BC
:107210001D49184603F064FC78607B68002B22D17E
:107220003B680121184603F0E1FC78607B68002B85
:107230001BD13B680021184603F0FEFC78607B6898
:10724000002B14D1642004F004FB3B680121184694
:1072500003F0F2FC78607B68002B0AD1642004F014
:10726000F8FA7B680BE000BF04E000BF02E000BF5B
:1072700000E000BF3B68184603F096FC7B681846A8
:107280000837BD4680BD00BF0805002080B500AFAF
:107290000349044803F004FE0346184680BD00BFBE
:1072A000E8040020E429002080B584B000AF7860B5
:1072B0000023FB600023BB607B6800221A607A68B1
:1072C000012140F20240FFF7A5FEF8607B681B68D1
:1072D000BB60FB68002B01D01423FB60FB68002B14
:1072E00010D1BB6843F40023BB6007F108031946C3
:1072F00040F20240FFF7E6FDF860FB68002B01D08A
:107300001423FB60FB6818461037BD4680BD80B56E
:1073100084B000AF78600023FB600EE007F1080343
:107320001846FFF7C1FFF860FB68142B02D0FB681A
:10733000002B02D17B68013B7B607B68002BEDD189
:1073400000BF00BF1037BD4680BD80B584B000AF20
:107350000346FB800B46BB8013467B800023FB600B
:1073600000237B81BB881B01BB807B88DB017B808A
:10737000FB88322B02D10023FB8008E0FB883C2BEA
:1073800003D14FF48073FB8001E004232EE007F16A
:107390000A031A46012140F29240FFF7B7FEF86057
:1073A000FB68002B01D00823FB60FB68002B1CD17D
:1073B0007B8923F4F8739BB27B817A89FB88134322
:1073C0009AB2BB8813439AB27B8813439BB27B81EA
:1073D00007F10A03194640F29240FFF7C7FDF86033
:1073E000FB68002B01D00823FB60FB6818461037B0
:1073F000BD4680BD80B584B000AF0346FB8000234E
:10740000FB6000237B81FB88002B02D10023FB80E3
:107410000DE0FB88012B02D10A23FB8007E0FB88EB
:10742000022B02D11423FB8001E01E23FB80FB888A
:107430007B8107F10A03194640F29A40FFF796FD57
:10744000F860FB68002B01D00923FB60FB6818463D
:107450001037BD4680BD80B485B000AFF860B9601C
:107460007A60BB680133BB60FA68BB6822FA03F339
:10747000FB60FB68002B0BD17B684FF0FF321A607A
:1074800000230EE0BB680133BB60FB685B08FB6058
:10749000FB6803F00103002BF4D07B68BA681A6024
:1074A000012318461437BD4680BC70470000000019
:1074B00080B58AB002AFF860B9607A603B60FB6863
:1074C000002B02D16FF0120327E2FB683B61BB6A1D
:1074D000222B00F32082BB6A0A3B172B00F20782A3
:1074E00001A252F823F000BF497500106F7500101B
:1074F00095750010EF780010BB750010E175001055
:10750000077600102D760010537600107976001063
:107510009F760010C5760010EB76001011770010F2
:1075200037770010EF7800105D7700107D7700103E
:10753000CD770010ED7700105178001069780010B9
:10754000B9780010D7780010AB4B03F56043D3F83F
:107550009C39184616F01AFA02460B46CDE900236C
:10756000A64A7968B86817F02DFF0346D5E1A24B0B
:1075700003F56043D3F89439184616F007FA02462B
:107580000B46CDE900239D4A7968B86817F01AFFC9
:107590000346C2E1984B03F56043D3F89839184687
:1075A00016F0F4F902460B46CDE90023934A7968B8
:1075B000B86817F007FF0346AFE18F4B03F5604350
:1075C000D3F86839184616F0E1F902460B46CDE9C2
:1075D00000238A4A7968B86817F0F4FE03469CE1F4
:1075E000854B03F56043D3F86C39184616F0CEF995
:1075F00002460B46CDE90023804A7968B86817F047
:10760000E1FE034689E17C4B03F56043D3F8703912
:10761000184616F0BBF902460B46CDE90023774A1F
:107620007968B86817F0CEFE034676E1724B03F531
:107630006043D3F87439184616F0A8F902460B4691
:10764000CDE900236D4A7968B86817F0BBFE0346A0
:1076500063E1694B03F56043D3F87839184616F0B7
:1076600095F902460B46CDE90023644A7968B8686B
:1076700017F0A8FE034650E15F4B03F56043D3F8D3
:107680007C39184616F082F902460B46CDE90023F4
:107690005A4A7968B86817F095FE03463DE1564BA3
:1076A00003F56043D3F88039184616F06FF90246A7
:1076B0000B46CDE90023514A7968B86817F082FE7D
:1076C00003462AE14C4B03F56043D3F8843918464E
:1076D00016F05CF902460B46CDE90023474A79686B
:1076E000B86817F06FFE034617E1434B03F560439C
:1076F000D3F88C39184616F049F902460B46CDE905
:1077000000233E4A7968B86817F05CFE034604E13E
:10771000394B03F56043D3F89039184616F036F923
:1077200002460B46CDE90023344A7968B86817F061
:1077300049FE0346F1E0304B03F56043D3F8883946
:10774000184616F023F902460B46CDE900232B4AD2
:107750007968B86817F036FE0346DEE0264B03F57D
:10776000604393F8F43C1A46254B53F822301A46EE
:107770007968B86817F026FE0346CEE0BB680022A1
:107780001A700023FB6119E01D4AFB6952F823308F
:107790001946B86817F032FFFB69042B0BD0B868A4
:1077A00018F02EF903461A46BB68134415491A46C9
:1077B0000B461B881380FB690133FB61FB69042BBB
:1077C000E2D9B86818F01CF90346A6E00A4B03F5A5
:1077D000604393F8EC3C1A460B4B53F822301A46A0
:1077E0007968B86817F0EEFD034696E0BB680022A2
:1077F0001A700023BB6123E0F03F002008BC021098
:1078000094BF021010BC0210A8BF0210484ABB6906
:1078100052F823301946B86817F0F0FEBB69032B05
:107820000BD0B86818F0ECF803461A46BB6813444E
:1078300040491A460B461B881380BB690133BB6164
:10784000BB69032BE2D9B86818F0DAF8034664E0A4
:10785000394B03F56043D3F85039384A7968B86832
:1078600017F0B0FD034658E0BB6800221A700023F1
:107870007B6119E0324A7B6952F823301946B868B7
:1078800017F0BCFE7B69012B0BD0B86818F0B8F874
:1078900003461A46BB68134426491A460B461B8802
:1078A00013807B6901337B617B69012BE2D9B86866
:1078B00018F0A6F8034630E0224B1B78DBB2002B11
:1078C00001D0214B00E0214B214A7968B86817F0BC
:1078D00079FD034621E014A3D3E90023CDE9002379
:1078E0001C4A7968B86817F06DFD034615E03A69DF
:1078F000BB6A02339B0013445B68184616F046F8D7
:1079000002460B46CDE90023134A7968B86817F0A0
:1079100059FD034601E06FF0150318462037BD46B8
:1079200080BD00BFAFF30080000000A09999014026
:10793000A8BF021010BC0210F03F002014BC0210BF
:10794000B8BF02101C05002018BC02101CBC02109D
:1079500020BC021024BC021008BC021090B5ADF689
:107960002C6D00AF07F62864A4F61C64206007F6AF
:107970002860A0F56260016007F62861A1F6246125
:107980000A6007F62862A2F62862136007F62863E9
:10799000A3F56263186816F093FD02460B46104685
:1079A000194616F04BF80346C7F8183E07F6286349
:1079B000A3F61C631B68002B02D16FF0120388E151
:1079C00007F62863A3F61C631B68C7F8143ED7F8B4
:1079D000383E222B00F37B81C04B01221A70D7F86E
:1079E000383E0A3B162B00F2628101A252F823F0C6
:1079F0004D7A00105F7A0010717A0010AF7C001091
:107A0000837A0010957A0010A77A0010B97A0010D6
:107A1000CB7A0010DD7A0010EF7A0010017B0010A5
:107A2000137B0010257B0010377B0010AF7C00100B
:107A3000497B0010AF7C0010A57B0010AF7C0010CC
:107A4000017C0010AF7C0010617C0010A44B03F59A
:107A500060431A46D7F8183EC2F89C3931E1A04B72
:107A600003F560431A46D7F8183EC2F8943928E166
:107A70009B4B03F560431A46D7F8183EC2F8983975
:107A80001FE1974B03F560431A46D7F8183EC2F83A
:107A9000683916E1924B03F560431A46D7F8183E51
:107AA000C2F86C390DE18E4B03F560431A46D7F8E6
:107AB000183EC2F8703904E1894B03F560431A4659
:107AC000D7F8183EC2F87439FBE0854B03F56043E4
:107AD0001A46D7F8183EC2F87839F2E0804B03F521
:107AE00060431A46D7F8183EC2F87C39E9E07C4B6F
:107AF00003F560431A46D7F8183EC2F88039E0E033
:107B0000774B03F560431A46D7F8183EC2F884391C
:107B1000D7E0734B03F560431A46D7F8183EC2F816
:107B20008C39CEE06E4B03F560431A46D7F8183E09
:107B3000C2F89039C5E06A4B03F560431A46D7F89E
:107B4000183EC2F88839BCE00023C7F8243E22E082
:107B5000644AD7F8243E52F8232007F62863A3F599
:107B600062631146186817F06FFD0346002B0DD1B4
:107B7000D7F8243EDAB25A4B03F5604383F8F42C6D
:107B800007F62863A3F624631B68A2E0D7F8243E17
:107B90000133C7F8243ED7F8243E042BD8D96FF020
:107BA000150396E00023C7F8203E22E04E4AD7F89E
:107BB000203E52F8232007F62863A3F5626311469E
:107BC000186817F041FD0346002B0DD1D7F8203E71
:107BD000DAB2434B03F5604383F8EC2C07F62863D5
:107BE000A3F624631B6874E0D7F8203E0133C7F87E
:107BF000203ED7F8203E032BD8D96FF0150368E05C
:107C00000023C7F81C3E24E0384AD7F81C3E52F83F
:107C1000232007F62863A3F562631146186817F05E
:107C200013FD0346002B0FD1D7F8180E16F050FAAB
:107C300003462B4A02F56042C2F8503907F6286322
:107C4000A3F624631B6844E0D7F81C3E0133C7F851
:107C50001C3ED7F81C3E012BD6D96FF0150338E037
:107C60001E4B00221A7007F62863A3F562632049B1
:107C7000186817F0E9FC0346002B03D11D4B0122C5
:107C80001A7014E01B4B00221A70154B03F5604369
:107C9000D3F8043D07F110014FF4606218460AF072
:107CA0004BFEC7F8100ED7F8103E002BEDD0D7F8DA
:107CB000142ED7F8383E02339B001344D7F8182E01
:107CC0005A6007F62863A3F624631B6801E06FF08F
:107CD0001503184607F62C67BD4690BDE83F002007
:107CE000F03F002094BF0210A8BF0210B8BF0210DE
:107CF00018BC02101C05002080B59EB002AFF860D1
:107D0000B9607A603B60FB68002B03D16FF012030F
:107D100001F034B9FB68FB61BB6F162B03DD6FF01C
:107D2000150301F02BB93B68DB780D2B00F01B84A9
:107D30000D2B01F32181002B04D0012B00F0588280
:107D400001F01AB9BB6F162B00F23B8201A252F868
:107D500023F000BFB17D0010037E0010717E001083
:107D60003D7F00100B8000103D8000104F80001000
:107D7000C3810010CD8000101F810010C38100104E
:107D8000C3810010C3810010C3810010C3810010A3
:107D9000C3810010C3810010C3810010C381001093
:107DA000C3810010C38100107181001099810010FF
:107DB000BB4B03F56043D3F8F82C3B68B3F90030B4
:107DC0001946DC2301FB03F3134403F58C731B6892
:107DD000B34A02F56042D2F894291146184601F0E0
:107DE0003BFA0346184615F0D1FD02460B46CDE995
:107DF0000023AC4A7968B86817F0E4FA034601F04A
:107E0000BDB83B68B3F90030022B20D0022B2FDC29
:107E1000002B02D0012B09D02AE00023A24A796866
:107E2000B86817F0CFFA034601F0A8B89C4B03F5E9
:107E30005043B3F8B839184601F0F2F903469A4AAC
:107E40007968B86817F0BEFA034601F097B8944B0A
:107E500003F55043B3F8BC39184601F0E1F9034685
:107E6000914A7968B86817F0ADFA034601F086B810
:107E7000BB6800221A7007F110004FF000028B4B14
:107E8000CDE900234FF000024FF00003884917F0BE
:107E9000F9FA07F110031946B86817F0AFFBB86894
:107EA00017F0AEFD03461A46BB68134481491A46D3
:107EB0000B461B8813800023FB6636E0784B03F5E6
:107EC0006043D3F8F83C3A68B2F9002011466E22BC
:107ED00002FB01F1FA6E0A44943233F8123018466C
:107EE00001F0E0F90346184615F050FD02460B4636
:107EF00007F11000704917F0C5FA07F11003194691
:107F0000B86817F07BFBFB6E312B0BD0B86817F00D
:107F100077FD03461A46BB68134466491A460B466A
:107F20001B881380FB6E0133FB66FB6E302BC5DDB7
:107F3000B86817F065FD034601F020B8BB68002261
:107F40001A7007F110004FF00002584BCDE90023E2
:107F50004FF000024FF00003554917F093FA07F174
:107F600010031946B86817F049FBB86817F048FDC8
:107F700003461A46BB6813444E491A460B461B88F3
:107F800013800023BB6637E0454B03F56043D3F80D
:107F9000F82C3B68B3F9003019466E2303FB01F15E
:107FA000BB6E0B44C4335B0013449B88184601F03E
:107FB00079F90346184615F0E9FC02460B4607F12D
:107FC00010003D4917F05EFA07F110031946B86832
:107FD00017F014FBBB6E312B0BD0B86817F010FDF7
:107FE00003461A46BB68134432491A460B461B889F
:107FF0001380BB6E0133BB66BB6E302BC4DDB8682B
:1080000017F0FEFC034600F0B9BF254B03F56043B3
:10801000D3F894392949184615F022FF034618462B
:1080200015F0B4FC02460B46CDE90023244A7968DA
:10803000B86817F0C7F9034600F0A0BF0023214A33
:108040007968B86817F0BEF9034600F097BF144B83
:1080500003F56043D3F8F82C3B68B3F900301946B8
:10806000DC2301FB03F3134403F5F8731B88184664
:1080700015F0EAFD03461449184615F0F1FE0346D3
:10808000184615F083FC02460B46CDE900230A4A48
:108090007968B86817F096F9034600F06FBF00BF23
:1080A000F03F002008BC02102CBC02100000594018
:1080B00030BC021010BC021038BC021000288E46E2
:1080C0003CBC021014BC02100000C842B94B03F5BE
:1080D0006043D3F8F82C3B68B3F900301946DC2331
:1080E00001FB03F3134403F58E731B68B14A02F5D9
:1080F0006042D2F894291146184601F0ADF80346C3
:10810000184615F043FC02460B46CDE90023AA4A67
:108110007968B86817F056F9034600F02FBFA54BF1
:1081200003F56043D3F8F82C3B68B3F900301946E7
:10813000DC2301FB03F3134403F590731B689D4A92
:1081400002F56042D2F894291146184601F084F8ED
:108150000346184615F01AFC02460B46CDE90023EB
:10816000954A7968B86817F02DF9034600F006BF04
:10817000904B03F56043D3F8F83C3A68B2F900201D
:1081800002F2D24233F822308C4A7968B86817F08C
:1081900019F9034600F0F2BE864B03F56043D3F8AD
:1081A000F82C3B68B3F9003003F2D2439B00134430
:1081B0005B88824A7968B86817F004F9034600F0D2
:1081C000DDBE3B68B3F900301A46F96913465B001F
:1081D0001344DB009B1ABA6F1344263351F8233043
:1081E000774A7968B86817F0EDF8034600F0C6BE24
:1081F000BB6F062B00F2A08101A252F823F000BF52
:108200001D8200106F820010E5820010D5830010DF
:10821000A5840010D7840010E9840010654B03F595
:108220006043D3F8F82C3B68B3F900301946D023EB
:1082300001FB03F3134403F56B731B685D4A02F5FE
:108240006042D2F898291146184601F005F8034615
:10825000184615F09BFB02460B46CDE90023564A13
:108260007968B86817F0AEF8034600F087BE3B683F
:10827000B3F90030022B20D0022B2FDC002B02D0D0
:10828000012B09D02AE000234C4A7968B86817F01E
:1082900099F8034600F072BE464B03F55043B3F81D
:1082A000BE39184600F0BCFF0346444A7968B868F6
:1082B00017F088F8034600F061BE3E4B03F55043CB
:1082C000B3F8C239184600F0ABFF03463B4A796861
:1082D000B86817F077F8034600F050BE6FF015034A
:1082E00000F04CBEBB6800221A7007F110004FF07E
:1082F0000002344BCDE900234FF000024FF00003A1
:10830000314917F0BFF807F110031946B86817F0A4
:1083100075F9B86817F074FB03461A46BB68134436
:108320002A491A460B461B88138000237B6638E0D7
:10833000204B03F56043D3F8F82C3B68B3F90030C9
:108340001946682303FB01F17B6E0B4403F5EA73C6
:108350005B0013441B89184600F0A4FF034618462F
:1083600015F014FB02460B4607F11000184917F0F0
:1083700089F807F110031946B86817F03FF97B6ECA
:10838000312B0BD0B86817F03BFB03461A46BB688D
:1083900013440E491A460B461B8813807B6E01332B
:1083A0007B667B6E302BC3DDB86817F029FB034674
:1083B00000F0E4BDF03F002008BC02102CBC02100D
:1083C00014BC02100000594030BC021010BC021056
:1083D00038BC0210BB6800221A7007F110004FF081
:1083E0000002BC4BCDE900234FF000024FF0000328
:1083F000B94917F047F807F110031946B86817F0A4
:10840000FDF8B86817F0FCFA03461A46BB68134437
:10841000B2491A460B461B88138000233B6638E09E
:10842000AF4B03F56043D3F8F82C3B68B3F9003049
:108430001946682303FB01F13B6E0B4403F50273FD
:108440005B0013449B88184600F02CFF0346184637
:1084500015F09CFA02460B4607F11000A14917F0EF
:1084600011F807F110031946B86817F0C7F83B6E0A
:10847000312B0BD0B86817F0C3FA03461A46BB6815
:10848000134496491A460B461B8813803B6E0133F2
:108490003B663B6E302BC3DDB86817F0B1FA03467C
:1084A00000F06CBD8E4B03F56043D3F898398E49CC
:1084B000184615F0D5FC0346184615F067FA024633
:1084C0000B46CDE90023894A7968B86816F07AFF2F
:1084D000034600F053BD0023854A7968B86816F05A
:1084E00071FF034600F04ABD7D4B03F56043D3F8AE
:1084F000F82C3B68B3F900301946D02301FB03F395
:10850000134403F58F631B88184615F09DFB034643
:108510007849184615F0A4FC0346184615F036FABB
:1085200002460B46CDE900236E4A7968B86816F01A
:1085300049FF034600F022BD3B68B3F90030DA1C66
:10854000F96913465B001344DB009B1ABA6F1344AE
:10855000263351F82330664A7968B86816F032FF3E
:10856000034600F00BBD3B68B3F90030032B00F26B
:10857000008501A252F823F089850010258800109B
:10858000A58A0010B18D0010BB6F0D3B042B00F2CB
:10859000468101A252F823F0AD850010CB85001072
:1085A0004F860010018700107F8700104C4B03F5A9
:1085B0006043D3F8F83C93F828304F4A7968B8689C
:1085C00016F000FF034600F0D9BCBB6800221A7009
:1085D0000023FB6532E0FB6D012B0EDC404B03F505
:1085E0006043D3F8F81CFA6D13465B001344DB00BC
:1085F0000B443033D3E9002303E04FF000024FF087
:10860000000307F110003D4916F03CFF07F110038D
:108610001946B86816F0F2FFFB6D052B0BD0B86851
:1086200017F0EEF903461A46BB6813442B491A4665
:108630000B461B881380FB6D0133FB65FB6D052B1F
:10864000C9DDB86817F0DCF9034600F097BCBB68D9
:1086500000221A700023BB6532E0BB6D012B0EDCDB
:108660001F4B03F56043D3F8F81CBA6D13465B004B
:108670001344DB000B443833D3E9002303E04FF00D
:1086800000024FF0000307F110001C4916F0FAFE3B
:1086900007F110031946B86816F0B0FFBB6D052B43
:1086A0000BD0B86817F0ACF903461A46BB68134400
:1086B0000A491A460B461B881380BB6D0133BB6504
:1086C000BB6D052BC9DDB86817F09AF9034600F0B9
:1086D00055BC00BF0000594030BC021010BC021055
:1086E000F03F002038BC021000288E463CBC02102F
:1086F00014BC02100000C84244BC02104CBC021062
:10870000BB6800221A7000237B6530E07B6D012B73
:108710000EDCB84B03F56043D3F8F81C7B6D5A1C94
:1087200013465B001344DB000B4428331B6800E056
:10873000002307F110001A46AF4916F0A3FE07F117
:1087400010031946B86816F059FF7B6D052B0BD046
:10875000B86817F055F903461A46BB681344A74991
:108760001A460B461B8813807B6D01337B657B6D3E
:10877000052BCBDDB86817F043F90346FEE3BB6871
:1087800000221A7000233B6541E03B6D012B1DDC8C
:10879000984B03F56043D3F8F81C3B6D5A1C134605
:1087A0005B001344DB000B442C331B68914A02F539
:1087B0006042D2F894291146184600F04DFD034658
:1087C000184615F0E3F802460B4603E04FF00002AE
:1087D0004FF0000307F11000894916F053FE07F12E
:1087E00010031946B86816F009FF3B6D052B0BD036
:1087F000B86817F005F903461A46BB6813447F4969
:108800001A460B461B8813803B6D01333B653B6D5D
:10881000052BBADDB86817F0F3F80346AEE36FF046
:108820001503ABE3BB6F0D3B052B00F2388101A2B2
:1088300052F823F04D88001069880010EB88001072
:108840006D8900109F8A0010E9890010694B03F5BB
:108850006043D3F8F83C93F829306A4A7968B868DD
:1088600016F0B0FD034689E3BB6800221A700023AE
:10887000FB6432E0FB6C012B0EDC5E4B03F56043C6
:10888000D3F8F81CFA6C13465B001344DB000B446E
:108890006033D3E9002303E04FF000024FF0000300
:1088A00007F11000584916F0EDFD07F110031946C5
:1088B000B86816F0A3FEFB6C052B0BD0B86817F058
:1088C0009FF803461A46BB6813444C491A460B46A8
:1088D0001B881380FB6C0133FB64FB6C052BC9DD2B
:1088E000B86817F08DF8034648E3BB6800221A7099
:1088F0000023BB6432E0BB6C012B0EDC3D4B03F567
:108900006043D3F8F81CBA6C13465B001344DB00D9
:108910000B446833D3E9002303E04FF000024FF02B
:10892000000307F11000384916F0ACFD07F1100301
:108930001946B86816F062FEBB6C052B0BD0B86800
:1089400017F05EF803461A46BB6813442B491A46D3
:108950000B461B881380BB6C0133BB64BB6C052BBF
:10896000C9DDB86817F04CF8034607E3BB6800227E
:108970001A7000237B642FE07B6C012B0DDC1D4BF8
:1089800003F56043D3F8F81C7A6C13465B0013447C
:10899000DB000B4470331B6800E0002307F110007C
:1089A0001A46154916F06EFD07F110031946B8680E
:1089B00016F024FE7B6C052B0BD0B86817F020F85E
:1089C00003461A46BB6813440C491A460B461B88DB
:1089D00013807B6C01337B647B6C052BCCDDB8682A
:1089E00017F00EF80346C9E2BB6800221A70002394
:1089F0003B644CE0F03F002054BC021010BC02105D
:108A00003CBC021044BC02104CBC02103B6C012B5D
:108A10001CDCA54B03F56043D3F8F81C3A6C1346F5
:108A20005B001344DB000B4474331B689E4A02F561
:108A30006042D2F894291146184600F00DFC034616
:108A4000184614F0A3FF02460B4603E04FF0000265
:108A50004FF0000307F11000944916F013FD07F1E1
:108A600010031946B86816F0C9FD3B6C052B0BD0F6
:108A7000B86816F0C5FF03461A46BB6813448C4914
:108A80001A460B461B8813803B6C01333B643B6CDE
:108A9000052BBBDDB86816F0B3FF03466EE26FF03E
:108AA00015036BE2BB6F0D3B072B00F27E8101A229
:108AB00052F823F0D58A0010F18A00106D8B001057
:108AC000EB8B0010AB8D0010AB8D0010618C001093
:108AD000138D0010744B03F56043D3F8F83C93F802
:108AE0002A30744A7968B86816F06CFC034645E28F
:108AF000BB6800221A700023FB632FE0FB6B012B85
:108B00000BDC694B03F56043D3F8F82CFB6B0633A1
:108B10005B011344D3E9002303E04FF000024FF060
:108B2000000307F11000644916F0ACFC07F11003D4
:108B30001946B86816F062FDFB6B052B0BD0B868C0
:108B400016F05EFF03461A46BB68134458491A469E
:108B50000B461B881380FB6B0133FB63FB6B052B00
:108B6000CCDDB86816F04CFF034607E2BB68002274
:108B70001A700023BB6330E0BB6B012B0CDC4A4B4B
:108B800003F56043D3F8F82CBB6B05335B0113444A
:108B90002833D3E9002303E04FF000024FF0000335
:108BA00007F11000444916F06DFC07F11003194657
:108BB000B86816F023FDBB6B052B0BD0B86816F018
:108BC0001FFF03461A46BB68134439491A460B4631
:108BD0001B881380BB6B0133BB63BB6B052BCBDDE9
:108BE000B86816F00DFF0346C8E1BB6800221A7092
:108BF00000237B632CE07B6B012B0ADC2A4B03F503
:108C00006043D3F8F82C7B6B5B011344D0331B68B3
:108C100000E0002307F110001A46284916F032FC44
:108C200007F110031946B86816F0E8FC7B6B052BBA
:108C30000BD0B86816F0E4FE03461A46BB6813442E
:108C40001B491A460B461B8813807B6B01337B63E1
:108C50007B6B052BCFDDB86816F0D2FE03468DE1A5
:108C6000BB6800221A7000233B634AE03B6B012B78
:108C700026DC0D4B03F56043D3F8F82C3B6B5B010E
:108C80001344D4331B68084A02F56042D2F8942991
:108C90001146184600F0E0FA0346184614F076FE36
:108CA00002460B4610E000BFF03F00203CBC021023
:108CB00010BC021044BC02104CBC021054BC021088
:108CC0004FF000024FF0000307F11000AD4916F01D
:108CD000D9FB07F110031946B86816F08FFC3B6BFF
:108CE000052B0BD0B86816F08BFE03461A46BB68FE
:108CF0001344A5491A460B461B8813803B6B01336E
:108D00003B633B6B052BB1DDB86816F079FE03467B
:108D100034E1BB6800221A700023FB623DE0FB6A6D
:108D2000012B19DC994B03F56043D3F8F82CFB6A4F
:108D30005B011344D8331B68944A02F56042D2F8B1
:108D400094291146184600F087FA0346184614F095
:108D50001DFE02460B4603E04FF000024FF00003F9
:108D600007F11000874916F08DFB07F11003194633
:108D7000B86816F043FCFB6A052B0BD0B86816F0F8
:108D80003FFE03461A46BB6813447F491A460B460A
:108D90001B881380FB6A0133FB62FB6A052BBEDD77
:108DA000B86816F02DFE0346E8E06FF01503E5E025
:108DB000BB6F0D3B032B00F2D98001A252F823F0C8
:108DC000D18D0010ED8D00106F8E0010F18E00100F
:108DD0006E4B03F56043D3F8F83C93F82B306C4AA4
:108DE0007968B86816F0EEFA0346C7E0BB6800225F
:108DF0001A700023BB6232E0BB6A012B0EDC634BAE
:108E000003F56043D3F8F81CBA6A13465B001344B9
:108E1000DB000B449033D3E9002303E04FF0000262
:108E20004FF0000307F110005A4916F02BFB07F131
:108E300010031946B86816F0E1FBBB6A052B0BD08E
:108E4000B86816F0DDFD03461A46BB6813444E4968
:108E50001A460B461B881380BB6A0133BB62BB6A90
:108E6000052BC9DDB86816F0CBFD034686E0BB686C
:108E700000221A7000237B6232E07B6A012B0EDC39
:108E8000424B03F56043D3F8F81C7A6A13465B0043
:108E90001344DB000B449833D3E9002303E04FF085
:108EA00000024FF0000307F110003A4916F0EAFA09
:108EB00007F110031946B86816F0A0FB7B6A052B72
:108EC0000BD0B86816F09CFD03461A46BB681344E5
:108ED0002D491A460B461B8813807B6A01337B623F
:108EE0007B6A052BC9DDB86816F08AFD034645E0AC
:108EF000BB6800221A7000233B622FE03B6A012B03
:108F00000DDC224B03F56043D3F8F81C3A6A134694
:108F10005B001344DB000B44A0331B6800E000231C
:108F200007F110001A461C4916F0ACFA07F11003BD
:108F30001946B86816F062FB3B6A052B0BD0B8687F
:108F400016F05EFD03461A46BB6813440E491A46E6
:108F50000B461B8813803B6A01333B623B6A052B3F
:108F6000CCDDB86816F04CFD034607E06FF0150342
:108F700004E06FF0150301E06FF015031846703739
:108F8000BD4680BD3CBC021010BC0210F03F00206A
:108F900044BC02104CBC021054BC021080B483B01C
:108FA00000AF78607B68002B02D16FF0120316E0EF
:108FB0000D4B03F56043D3F8043D002B07D17B68CC
:108FC0005B685B69084A02F56042C2F8043D7B6851
:108FD0005B685A687B685B689B68B2FBF3F3184672
:108FE0000C37BD4680BC7047F03F002080B592B082
:108FF00000AF786000237B644FF0FF33BB637B6876
:10900000002B02D16FF0150351E07B681B683B64B5
:109010003B6CD3F89434002B23D17B685B6807F159
:109020000C021146184606F01BFF03463FE03B6C5E
:10903000D3F894243B6CD3F89034B96B01FB03F361
:109040009B001344FB631C4B1B689B00FA6B1A4488
:109050007B6C591C796412689B0048333B4443F88D
:109060003C2C3B6CD3F88C34B96B07F138021846B2
:10907000FEF7F1F90346002BD9D13B6CD3F89034BD
:109080005A1E0D4B1B689A4203D10B4B00221A60EB
:1090900004E0094B1B680133074A13607B685B6877
:1090A00007F10C021146184606F0DAFE0346184690
:1090B0004837BD4680BD00BFEC3F002080B584B07E
:1090C00000AF0023FB60504BBB60504B7B60504BAC
:1090D0003B607B680C331846FEF7E6F8F860FB68E7
:1090E000002B40D17B68DB6803F40023002B3AD0CF
:1090F0007B68143303211846FDF738FEF860FB68DF
:10910000002B07D17B682033002203211846FDF78E
:1091100061FEF860FB68002B07D17B6826330122D3
:1091200003211846FDF756FEF860FB68002B06D1B8
:109130007B68103301211846FDF7EFFDF860FB68EE
:10914000002B05D17B6808331846FDF77AFEF860DE
:10915000FB68002B07D17B6800221A707B685B6874
:109160005A1C7B685A60FB68002B2DD17B68DB683A
:1091700003F40003002B27D04FF4E0612548FDF7EE
:1091800095FDF860BB6800221A70BB685B685A1CCA
:10919000BB685A60204B03F56043D3F8043D002BB5
:1091A00012D01E4B1B78DBB283F00103DBB2002B25
:1091B0000AD0194B03F56043D3F8043D4FF46062C5
:1091C0001449184609F0A7FBFB68002B17D17B68F0
:1091D000DB6803F48013002B11D03B6808330721B0
:1091E0001846FDF7DDFDF860FB68002B07D13B68F2
:1091F00000221A703B685B685A1C3B685A60FB6827
:1092000018461037BD4680BDE41901208819012099
:10921000C0190120EC190120F03F00201C0500209E
:1092200080B584B000AF0346FB80FB88184614F07D
:109230000BFD03460749184614F05EFD0346184629
:1092400014F046FF0346FB81FB8918461037BD46E4
:1092500080BD00BF0000903C80B584B000AF786056
:1092600039600E4BFB60786814F0EEFC03463968F9
:10927000184614F041FD03460949184614F0F0FD64
:109280000346BB60F968B86814F0EAFD0346BB60AA
:10929000BB6818461037BD4680BD00BFEE04B53F21
:1092A000E30A494C80B584B000AF0346FB80FB88DD
:1092B000184614F0C9FC03460E49184614F0D0FDB8
:1092C0000346FB604FF00001F86814F0C7FE034648
:1092D000002B08D00749F86814F0B6FE0346002BAF
:1092E00001D0FB6801E04FF0000318461037BD467F
:1092F00080BD00BF0000C84280B584B000AF786078
:109300000749786814F0F8FC0346184614F0E0FEAC
:109310000346FB81FB8918461037BD4680BD00BF60
:109320000000C84280B584B000AF78600749786813
:1093300014F0E2FC0346184614F0CAFE0346FB6034
:10934000FB6818461037BD4680BD00BF00007A4458
:1093500080B584B000AF78604FF08E41786814F02B
:10936000CBFC0346184614F0B3FE0346FB81FB8991
:1093700018461037BD4680BD80B584B000AF786018
:109380000749786814F0B8FC0346184614F0A0FEAC
:109390000346FB60FB6818461037BD4680BD00BF22
:1093A00000007A4480B582B000AF00237B60114892
:1093B00000F02AFD104B03F56043002283F8032DD3
:1093C0000D4B00229A600C4B03F550431A460023C4
:1093D000C2F89C39084B03F550431A460023C2F8E3
:1093E000D439054800F0C0F878607B681846083723
:1093F000BD4680BDF0270120F03F002080B588B039
:1094000000AF0346FB710023FB61424BBB610023AD
:10941000FB60414B7B61414B3B613E4B00229A60BC
:109420003C4B0022DA603B4B00221A61394B03F5BA
:109430005043012283F8D029364B03F550430122D3
:1094400083F89829334B03F55043012283F8F4291C
:10945000304B03F550431A460023C2F89C392D4B7C
:1094600003F550431A460023C2F8F839294B03F597
:1094700050431A460023C2F8D439264B03F5604303
:10948000002283F8032D234B00221A70214AFB7916
:109490005370204B00229A8007F10C031846FDF709
:1094A000F9FCF861FB69002B2ED1FB687A699A42BE
:1094B00003D0FB683A699A4226D1B86900F080F877
:1094C000F861144B00229A60FB69002B11D1FDF763
:1094D00043FBF861FB69002B0DD10E4B03F5604394
:1094E000D3F850391846FDF712FF0D4B00221A70C1
:1094F00001E00123FB61FB69002B05D1054B03F55E
:109500006043012283F8032DFB6918462037BD46CE
:1095100080BD00BFF03F002061B409081C875409DA
:10952000F82C012080B500AF0C4B1B78DBB2002B70
:109530000ED00B4815F0FEFB0020FFF75FFF074B36
:1095400000221A70074B03F56043012283F8032DB4
:1095500000F014F90023184680BD00BFE83F00204A
:1095600058C00210F03F002080B58AB002AF78608A
:10957000104BFB614AF21013BB610F4B7B6143F64A
:1095800034033B61002301933B6900937B69BA6913
:10959000F9690A4809F0B4FF0346FB73FB7B1946DF
:1095A000786800F00BFCB860BB6818462037BD46F1
:1095B00080BD00BF0440002014E1002050190120AC
:1095C00080B588B000AF78600023FB610023FB7694
:1095D000664B7B61664B3B613B6903F2ED43FB608D
:1095E0003B69D3F89C31BB60624B03F55043D3F821
:1095F0006039012118460AF067F80346FB76FB7EC6
:10960000002B15D15B4B03F56043D3F850399BB267
:10961000584A02F5604292F8F42C91B2554A02F58C
:10962000604292F8012892B21846FDF78EFEF8616A
:10963000FB69002B07D13B6993F8DC349BB21846D9
:10964000FDF7D8FEF861FB69002B40F08A803B698A
:1096500093F8DC247B691A724749B86814F04CFB14
:109660000346184614F034FD02467B695A603B6994
:10967000D3F85031322B03D17B6900221A7002E0FB
:109680007B6901221A703B6993F8EC247B699A7616
:10969000384B03F550431A46FB68C2F880393869E5
:1096A00000F07EFA3B69D3F888311846FFF724FEB4
:1096B00003461A467B691A853B69D3F88C311846F4
:1096C000FFF730FE02467B695A623B69D3F890315E
:1096D0001846FFF751FE02467B69DA623B69D3F810
:1096E0005431002B03D17B69012283F820203B6990
:1096F0009A787B6983F821201E4B03F55043D3F8F9
:1097000060391A49184609F037FF0346FB76FB7E9D
:10971000002B20D13B69D3F85431002B1BD07B693F
:109720001A783B6903F59C631946104600F0F6F879
:10973000F861FB69002B0ED10E4B03F55043D3F8B3
:1097400060093B6903F59C617B691B781A4609F047
:1097500095FF0346FB76FB7E1946786800F02EFBEA
:10976000F861FB6918462037BD4680BD54190120B9
:10977000F0270120F03F0020E30A494C80B588B073
:1097800000AF0023FB610023BB765E4B7B615E4B29
:109790003B615E4BFB605E4B03F55043D3F8603991
:1097A000BB600023FB76FFF789FCF8618EE07B69E4
:1097B0001B78002B2CD15349B86809F0E9FE034609
:1097C000BB76BB7E1946524800F05EFAF861FB6931
:1097D000002B40F0868001214D4800F001FCBB7E4B
:1097E00019464B4800F05EFC494B9B680133484AE0
:1097F0009360BB7E1946464800F0E0FAF861FB69C9
:10980000002B70D14349B86809F020FF0346BB76AE
:109810003F4B03F5604393F8033D012B02D1032333
:10982000FB6169E0FB681B7883F00103DBB2002B6E
:109830000ED03649B86809F0D9FE0346BB76BB7E28
:109840001946334800F0BAFAF861FB69002B4CD195
:109850003B691B78002B13D12F4B1B78DBB2002BFD
:109860000ED02949B86809F09FFE0346BB76BB7E3F
:109870001946274800F0A2FAF861FB69002B36D19F
:109880003B1D1946B86809F0CFFE0346BB76BB7E88
:1098900019461F4800F092FAF861FB69002B28D1A5
:1098A0007B68002B0ED01B49B86809F0CFFE034639
:1098B000BB76BB7E1946164800F080FAF861FB695A
:1098C000002B18D10323FB610123FB76FB7E83F081
:1098D0000103DBB2002B0FD0FB69002B3FF467AF15
:1098E0000AE000BF08E000BF06E000BF04E000BFE0
:1098F00002E000BF00E000BFFB6918462037BD460C
:1099000080BD00BF88190120C0190120E419012081
:10991000F03F0020E82C01201C05002080B588B015
:1099200000AF03463960FB710023FB610023BB617C
:109930009A4BFB60FB79002B71D1FB68B3F8443183
:109940003B61FB68B3F846317B61FB68B3F8443197
:10995000002B2FD00023BB6113E0FB68BA6968328B
:1099600053F822301846FFF7F3FC03461946FA680D
:10997000BB693C335B0013440A469A80BB690133E0
:10998000BB61FB68B3F844311A46BB699342E4D328
:10999000FB68B3F844213B685A80FB68B3F8443154
:1099A000C3F133039AB23B681A80FB6803F17C026F
:1099B0003B689A60FB68B3F84631002B00F09F804B
:1099C0000023BB6111E0FB68BA699A3253F8223078
:1099D0001846FFF7BDFC03461946FB68BA697032AA
:1099E00023F81210BB690133BB61FB68B3F8463141
:1099F0001A46BB699342E6D3FB68B3F846213B683D
:109A00005A80FB68B3F84631C3F133039AB23B681E
:109A10001A80FB6803F1E0023B685A606FE0FB6864
:109A2000B3F848313B61FB68B3F84A317B61FB68AE
:109A3000B3F84831002B2FD00023BB6113E0FB6843
:109A4000BA69CC3253F822301846FFF781FC03463E
:109A50001946FA68BB693C335B0013440A469A8096
:109A6000BB690133BB61FB68B3F848311A46BB6977
:109A70009342E4D3FB68B3F848213B685A80FB6803
:109A8000B3F84831C3F133039AB23B681A80FB68DC
:109A900003F17C023B689A60FB68B3F84A31002B03
:109AA0002DD00023BB6111E0FB68BA69FE3253F888
:109AB00022301846FFF74CFC03461946FB68BA698A
:109AC000703223F81210BB690133BB61FB68B3F835
:109AD0004A311A46BB699342E6D3FB68B3F84A2180
:109AE0003B685A80FB68B3F84A31C3F133039AB23A
:109AF0003B681A80FB6803F1E0023B685A607A69B0
:109B00003B699A4240D07B69002B15D10023BB6191
:109B10000DE0FA68BB693C335B0013449988FB682D
:109B2000BA69703223F81210BB690133BB61BA699C
:109B30003B699A42EDD32CE03B69002B16D1002300
:109B4000BB610EE0FB68BA69703233F81210FA6834
:109B5000BB693C335B0013440A469A80BB690133FE
:109B6000BB61BA697B699A42ECD312E03A697B69BE
:109B70009A4204D23B699AB23B685A8009E07B69F9
:109B80009AB23B685A8004E07B69002B01D1012323
:109B9000FB61FB6918462037BD4680BDF0270120D8
:109BA00080B58AB000AF7860364B7B627B68D3F8B3
:109BB00080311846FFF7A0FB03467B847B68D3F80F
:109BC00084311846FFF798FB03463B847A8C3B8C24
:109BD000D31AFB837B6A7A8C1A837B6AFA8BDA82CC
:109BE0007B68D3F868311846FFF786FB0346BB83D2
:109BF0007B68D3F86C311846FFF77EFB03467B8306
:109C00007A8BBB8B13443B837B68D3F87031184647
:109C1000FFF772FB0346FB827B68D3F8743118466A
:109C2000FFF76AFB0346BB82FA8ABB8AD31A7B82A0
:109C30007B68D3F878311846FFF75EFB03463B821A
:109C40007B68D3F87C311846FFF756FB0346FB814F
:109C5000FA893B8A1344BB817B6A3A8B9A817B6A7F
:109C6000BA8B5A817B6AFA8A1A827B6A7A8ADA818B
:109C70007B6ABA899A827B6A3A8A5A8200BF2837FD
:109C8000BD4680BD5419012080B586B000AF786014
:109C90000B46FB7000237B61464B03F5604393F852
:109CA000033D012B40F08180424B03F56043D3F824
:109CB0005829404BDB689A4230D93F4B00221A703A
:109CC000FB78042B22D14FF47A73FB60394B0022CE
:109CD000DA60384B1B690133364A1361354B1B6917
:109CE000FA689A420FD2334B03F560431A460023B9
:109CF000C2F84C392F4B03F56043002283F8032D43
:109D000002237B6145E003237B6142E0294BDB6852
:109D10000133284AD36003237B613AE064237B82CA
:109D2000244B03F5604393F8003883F00103DBB262
:109D3000002B02D0204B01221A701F4B1B78DBB284
:109D4000002B04D11B4B9B887A8A9A4219D200239C
:109D50007B74184B03F56043022283F8032D154BE7
:109D600003F55043D3F860397A7C1146184609F060
:109D7000ABFC104B00229A600021786800F030F9AB
:109D800001E003237B610B4B9B8801339AB2094BA3
:109D90009A80084B03F55043012283F8D029054BE4
:109DA00003F55043012283F8F4297B6918461837DC
:109DB000BD4680BDF03F0020F82C012080B584B066
:109DC00000AF78600B46FB700023FB60FB78002B34
:109DD00012D007F10B02FB781146184609F0DCFCA3
:109DE000FB7A022B08D10423FB60064B03F560438A
:109DF0001A460023C2F84C39FB6818461037BD4696
:109E000080BD00BFF03F002080B485B000AF786017
:109E10000223FB600AE0FB68023BFA68D1B27A6871
:109E200013440A46DA70FB680133FB60FB68322B8F
:109E3000F1DD0123FB600BE0FB68013BFA68D1B266
:109E40007A6813440A4683F83520FB680133FB60C7
:109E5000FB68322BF0DD7B68322283F867207B6859
:109E6000322283F868200023FB600CE0504AFB6834
:109E700052F823107B68FA6802F5987243F82210B2
:109E8000FB680133FB60FB68062BEFDD7B6800227B
:109E9000C3F858217B68474AC3F894217B68464A37
:109EA000C3F898217B680022C3F84C217B683222DA
:109EB000C3F850217B68414AC3F89C217B684FF06E
:109EC0008042C3F86C217B683D4AC3F868217B68F7
:109ED0004FF08042C3F874217B683A4AC3F870217E
:109EE0007B684FF08042C3F87C217B68364AC3F818
:109EF00078217B68354AC3F880217B68344AC3F8EF
:109F000084217B682722A3F8E2247B680222A3F83D
:109F1000E0247B680122C3F854217B680022A3F867
:109F200044217B680022A3F846217B680022A3F825
:109F300048217B680022A3F84A217B68254AC3F8A0
:109F400088217B68244AC3F88C217B68234AC3F8A4
:109F500090217B68002283F8ED247B68012283F83E
:109F6000EE247B68022283F8EF247B68002283F8CA
:109F7000F0247B68012283F8F1247B68022283F8B5
:109F8000F2247B68032283F8F3247B6801221A7091
:109F90007B6800225A707B6800229A707B680022DE
:109FA00083F8F42400BF1437BD4680BC704700BF5F
:109FB0007C0D002000407A44000093434B59A63E9C
:109FC0000000B4420000DC420000A0400000C0409D
:109FD000000040409A99993E0000A5430000F042DD
:109FE000B0B58CB002AF78600B46FB70002387F8E9
:109FF00027302A4B03F55043D3F86039FB61142313
:10A000007B8301237B7600233B624FF000024FF0FD
:10A010000003C7E90423224B1B78DBB2002B37D0A7
:10A020001F4B00221A70FB78002B1ED007F108038B
:10A030001946F86909F0A0FBD7E90223D7E9040122
:10A04000841A61EB0305B4F57A7F75F1000318DB20
:10A050007B8B7A7E01920093D7E90423F86909F09B
:10A0600047FB034687F827300BE07B8B7A7E019213
:10A070000093D7E90423F86909F03AFB034687F80F
:10A08000273097F8273019460448FFF797FE3862C3
:10A090003B6A18462837BD46B0BD00BFF03F0020E0
:10A0A000F82C012090B589B002AF78600B46FB70A8
:10A0B0000123FB750023BB82134B5B78002B1ED062
:10A0C000FB78152B02D0FB78192B18D10E4B03F51A
:10A0D00069436033D3E90023C7E902230A4B002216
:10A0E0005A70094B03F55043D3F86049D7E902236E
:10A0F000B98AF87D01900091204609F0F9FA00BF75
:10A100001C37BD4690BD00BFF03F002080B586B033
:10A1100000AF786039604FF49361012008F0CEF908
:10A120000346BB60BB68002B02D16FF00B0341E01C
:10A130003B68D3F88424BB68C3F894243B68D3F805
:10A140008024BB68C3F8902400237B6118E00023BF
:10A150003B610FE0B9687A6913465B001344DB008A
:10A160009B1A3A6913442633002241F823203B69A5
:10A1700001333B613B69162BECDD7B6901337B616D
:10A180007B690A2BE3DD0023FB600CE03B68FA6887
:10A1900053F82220B968FB6802339B000B445A60D5
:10A1A000FB680133FB60FB68222BEFDD7B68BA683C
:10A1B0001A60002318461837BD4680BD80B582B0AE
:10A1C00000AF78607B68002B02D16FF0150303E0CD
:10A1D000786808F081F9002318460837BD4680BD2D
:10A1E00080B485B000AF786039607B68002B02D105
:10A1F0006FF0120306E07B68FB60FB683A68C3F807
:10A200008C24002318461437BD4680BC704780B4A8
:10A2100085B000AF78607B68002B02D16FF012032D
:10A2200006E07B68FB60FB680022C3F88C240023F7
:10A2300018461437BD4680BC70470000F0B5ABB07F
:10A240000EAF07F1200340220021184614F00CFD48
:10A25000554A07F1180392E8030083E80300534BC3
:10A2600003F560431A460023C2F8043D4FF4B05290
:10A2700000214F4814F0F8FC0023FB66FCF708FBB4
:10A28000F866FB6E002B7CD107F16803494918463C
:10A2900000F032FFF866FB6E002B74D1BB6E1846DF
:10A2A00004F0D8F8FCF7AAFBF866FB6E002B03D08D
:10A2B000414814F03FFD69E0FFF774F8F866FB6E63
:10A2C000002B03D03D4814F035FD5FE007F1640337
:10A2D0003B491846FFF71AFFF866FB6E002B03D0C8
:10A2E000384814F027FD51E00020FFF787F8F866A2
:10A2F000FB6E002B04D0F96E334814F01BFD45E0D3
:10A30000324814F017FD324B3B607B6E7B60314B63
:10A31000BB6007F11803FB6000233B6100237B61F6
:10A320003B46BB620123FB622B4B07F138041D4601
:10A330000FCD0FC495E8070084E80700274BBB65E5
:10A3400007F160066D4607F12C040FCC0FC50FCC4A
:10A350000FC50FCC0FC523682B6007F120030ECB70
:10A36000304606F026FDF866FB6E002B0DD13B6EE5
:10A37000184606F055FEF8663B6E184606F07FFE5E
:10A3800004E000BF02E000BF00E000BF7B6E1846A3
:10A39000FFF714FFBB6E184600F0F2FEFB6E184686
:10A3A0007437BD46F0BD00BFC0C10210F03F0020B1
:10A3B000E8290020CC04002020C1021034C1021082
:10A3C0004400002054C1021074C10210A4C1021044
:10A3D000BCC10210440D002028000020259500106B
:10A3E00080B582B000AF6FF015037B60FFF726FFEA
:10A3F00078607B6818460837BD4680BD80B588B058
:10A4000000AF78607B68FB61FB695B689B6807F164
:10A4100010021146184608F005FEB861BB69002B12
:10A4200008D0FB691A68FB695B681946104600F0A2
:10A43000CAFA3FE0FB695B689B6807F114021146AA
:10A44000184608F06AFDFB695B689B6807F10C021F
:10A450001146184608F069FC3B691B69002B06D0C1
:10A460003B691B69386979693A6952699847FB68A1
:10A47000002B0ED1FB691B681A69FB695B68DB68FE
:10A480001946104600F0C5FCFB695B6801221A7191
:10A4900010E0FB691B68DB681B69FA69526879691F
:10A4A00010469847FB691A68FB695B6819461046B5
:10A4B00000F04DFA2037BD4680BD80B586B000AFB4
:10A4C000786039603B68002B03D03B689B68002BA9
:10A4D00002D16FF015037FE03B689B681B68002B7F
:10A4E00002D16FF0570377E007F10803184608F030
:10A4F0006BFFBB68184608F070FF3B689B681B68E1
:10A5000039687868984778617B69002B5ED17B68F1
:10A510001B681C33184608F057FF7B681B683A68B5
:10A520009268DA6000233B6122E07B681B689968CF
:10A530003A691346DB009B1ADB000B440833002208
:10A540000121184608F082FB78617B69002B1FD13E
:10A550007B681B6899683A691346DB009B1ADB002D
:10A560000B443033184608F02FFF3B6901333B6141
:10A570003B685B683A699A42D7D37B681B689A69E3
:10A5800001329A61BB68184608F030FF002323E0CF
:10A5900000BF0023FB600FE07B681B6899683A6985
:10A5A0001346DB009B1ADB000B449B68184608F03F
:10A5B00091FBFB680133FB60FA683B699A42EBD37D
:10A5C0007B681B68184600F00BF800E000BFBB6812
:10A5D000184608F00BFF7B6918461837BD4680BD4A
:10A5E00090B585B000AF78607B68002B02D16FF02A
:10A5F000150365E07B689B69002B01D100235FE0B8
:10A600000023FB6041E07B689B689B68184608F06C
:10A6100061FBB860BB68002B01D0BB6850E07B6871
:10A620009968FA681346DB009B1ADB000B441B6B2E
:10A63000184608F0E4FE7B681B69002B22D07B687B
:10A640009968FA681346DB009B1ADB000B44DB6950
:10A65000002B17D07B6818697B689968FA681346E5
:10A66000DB009B1ADB000B44DC687B689968FA68A6
:10A670001346DB009B1ADB000B4410331A462146BD
:10A6800000F081FBFB680133FB607B685B68FA6864
:10A690009A42B8D37B68DB69184608F0B0FE7B6845
:10A6A000DB685B6878689847B860BB68002B01D0AE
:10A6B000BB6805E07B689B695A1E7B689A61002332
:10A6C00018461437BD4690BD80B584B000AF7860A1
:10A6D00039607B68002B03D07B68DB68002B02D1DC
:10A6E0006FF015032AE07B68DB689B68002B02D1C2
:10A6F0006FF0570322E07B68DB69184608F06DFEB7
:10A700007B68DB689B6807F1080211467868984708
:10A71000F860FB68002B0AD17B689968BA68134619
:10A72000DB009B1ADB00CA183B681A6000E000BF20
:10A730007B68DB69184608F059FEFB68184610373D
:10A74000BD4680BD80B584B000AF786039607B685D
:10A75000002B06D07B68DB68002B02D03B68002B07
:10A7600002D16FF015031BE07B68DB68DB68002B10
:10A7700002D16FF0570313E03B681B6B184608F0DB
:10A780002CFE7B68DB68DB683A68126811467868E3
:10A790009847F8603B681B6B184608F027FEFB687B
:10A7A00018461037BD4680BD80B588B000AFF86050
:10A7B000B9607A603B60FB68002B08D0BB68002B57
:10A7C00005D07B68002B02D03B68002B02D16FF0D4
:10A7D000150399E03B681B6B184608F0FEFD00234B
:10A7E000FB610FE03B689868FA691346DB0013448D
:10A7F0009B001A46BB681344194608F0E6FAFB6949
:10A800000133FB61FA697B689A42EBD3FB681B69F1
:10A81000002B57D03B6810337B613B6803F120026B
:10A820007B695A603B681B681A467B69DA60BB68C3
:10A830001A7F7B695A723B68FA681A623B683A6809
:10A840005A62BB681B7B012B02DC002B03DA0AE097
:10A85000022B04D007E07B690A221A7207E07B69A9
:10A8600008221A7203E06FF01503BB6134E0FB6845
:10A87000DB681B69B96838689847B861BB69002B09
:10A8800027D1FB681B6A002B04D0FB681A6A7B691E
:10A890001A6002E07B691E4A1A60FB6818693B680F
:10A8A000DB687A69194600F04AFAB861BB69002B87
:10A8B00011D1FB6818693B68D968BB689B691A4667
:10A8C00000F0C9FA3B681B6B184608F08FFD0023A7
:10A8D0001AE000BF00E000BF0023FB610AE03B6814
:10A8E0009B6807F110021146184608F09BFBFB69B4
:10A8F0000133FB61FA697B689A42F0D33B681B6BBA
:10A90000184608F073FDBB6918462037BD4680BD68
:10A91000FDA3001080B582B000AF78607B681B6B30
:10A92000184608F05AFD7B68002B02D16FF0150322
:10A9300009E07B68002283F834207B681B6B184693
:10A9400008F054FD002318460837BD4680BD80B589
:10A9500084B000AF786039607B68002B06D07B68DC
:10A96000DB68002B02D03B68002B02D16FF015038F
:10A9700025E07B68DB685B69002B02D16FF0570331
:10A980001DE03B681B6B184608F027FD7B681B69C0
:10A99000002B07D07B681A693B68DB6819461046B4
:10A9A00000F015FA7B68DB685B693968786898475E
:10A9B000F8603B681B6B184608F018FDFB681846EA
:10A9C0001037BD4680BD80B584B000AF7860396077
:10A9D0007B68002B06D07B68DB68002B02D03B68CD
:10A9E000002B02D16FF0150331E07B68DB689B69B7
:10A9F000002B02D16FF0570329E03B681B6B184610
:10AA000008F0EBFC7B681B69002B07D07B681A6998
:10AA10003B68DB681946104600F0FBF93B689B6811
:10AA200007F108021146184608F0FCFAF860FB68C6
:10AA3000002BF3D07B68DB689B693968786898479E
:10AA4000F8603B681B6B184608F0D0FCFB681846A2
:10AA50001037BD4680BD80B483B000AF78603960E8
:10AA60003B68002B01D1012301E03B681B791846AC
:10AA70000C37BD4680BC704780B584B000AF7860AD
:10AA800039607B68002B06D07B68DB68002B02D026
:10AA90003B68002B01D101231EE07B68DB681B6A49
:10AAA000002B01D1012317E03B681B6B184608F00F
:10AAB00094FC7B68DB681B6A3968786898470346B2
:10AAC000FB603B681B6B184608F090FCFB68002B92
:10AAD00014BF01230023DBB218461037BD4680BDEA
:10AAE00080B584B000AF786039603B68002B03D03C
:10AAF0003B68DB68002B02D16FF0150319E03B685F
:10AB0000DB681B68002B02D16FF0570311E03B6834
:10AB1000DB681B68396878689847F860FB68002B29
:10AB200001D0FB6805E07B681B683A68D268DA6090
:10AB3000002318461037BD4680BD80B584B000AFF5
:10AB4000786039603B68002B04D03B685B68B3F1E8
:10AB5000FF3F04D17B6800221A60002320E03B689D
:10AB6000DB68002B02D16FF0150319E03B68DB684E
:10AB70005B68002B02D16FF0570311E03B68DB6884
:10AB80005B68396878689847F860FB68002B01D0EB
:10AB9000FB6805E07B681B683A68D268DA600023CE
:10ABA00018461037BD4680BD80B582B000AF7860D2
:10ABB0007B68002B15D07B68DB68002B02D16FF01F
:10ABC00015030FE07B68DB689B68002B02D16FF0F8
:10ABD000570307E07B68DB689B6878689847034603
:10ABE00000E0002318460837BD4680BD80B582B01E
:10ABF00000AF78600B46FB707B68002B17D07B683A
:10AC0000DB68002B02D16FF0150311E07B68DB6875
:10AC10001B69002B02D16FF0570309E07B68DB68EA
:10AC20001B69FA78114678689847034600E00023CC
:10AC300018460837BD4680BD80B582B000AF786049
:10AC40000B46FB707B68002B17D07B68DB68002B02
:10AC500002D16FF0150311E07B68DB689B69002B64
:10AC600002D16FF0570309E07B68DB689B69FA78D3
:10AC7000114678689847034600E0002318460837D5
:10AC8000BD4680BD80B584B000AF786039603B6858
:10AC9000002B03D03B685B68002B02D16FF01503DB
:10ACA0001EE03B685B681B68002B02D16FF0570306
:10ACB00016E03B685B681B68396878689847F860FD
:10ACC000FB68002B01D0FB680AE07B681B689A6870
:10ACD00001329A607B681B683A6852685A600023A8
:10ACE00018461037BD4680BD80B582B000AF786091
:10ACF0007B68002B03D07B685B68002B02D16FF070
:10AD0000150318E07B685B685B6A002B02D16FF06B
:10AD1000570310E07B689B685A1E7B689A607B68CB
:10AD20009B68002B01D0002305E07B685B685B6AB1
:10AD300078689847034618460837BD4680BD80B5F9
:10AD400084B000AFF860B9607A60FB68002B03D074
:10AD5000FB685B68002B02D16FF015030FE0FB6806
:10AD60005B685B68002B02D16FF0570307E0FB685C
:10AD70005B685B687A68B968F86898470346184664
:10AD80001037BD4680BD80B584B000AFF860B960B3
:10AD90007A60FB68002B03D0FB685B68002B02D154
:10ADA0006FF015030FE0FB685B689B68002B02D116
:10ADB0006FF0570307E0FB685B689B687A68B968C7
:10ADC000F8689847034618461037BD4680BD80B5E1
:10ADD00082B000AF786039607B68002B03D07B685D
:10ADE0005B68002B02D16FF015030EE07B685B6897
:10ADF0009B69002B02D16FF0570306E07B685B680C
:10AE00009B69396878689847034618460837BD46F5
:10AE100080BD80B582B000AF786039607B68002B60
:10AE200003D07B685B68002B02D16FF015030EE046
:10AE30007B685B68DB69002B02D16FF0570306E08B
:10AE40007B685B68DB693968786898470346184611
:10AE50000837BD4680BD80B584B000AFF860B960EA
:10AE60007A60FB68002B03D0FB685B68002B02D183
:10AE70006FF015030FE0FB685B681B6A002B02D1C3
:10AE80006FF0570307E0FB685B681B6A7A68B96874
:10AE9000F8689847034618461037BD4680BD000045
:10AEA00080B584B000AF786039603B68002B03D078
:10AEB0003B68DB68002B02D16FF015034DE03B6867
:10AEC000DB681B68002B02D16FF0570345E03B683D
:10AED0001B68082B02D96FF015033EE03B681B6826
:10AEE000204A52F82330002B08D1386800F03CF893
:10AEF000F860FB68002B01D0FB682EE03B68DB6844
:10AF00001B68396878689847F860FB68002B01D0A7
:10AF1000FB6822E03B681A687B681B68114951F89E
:10AF200022201A607B681B681B681A790132D2B232
:10AF30001A717B681B683A68D2681A617B681B6863
:10AF40003A68D2691A627B681B683A681433103217
:10AF500092E8030083E80300002318461037BD463B
:10AF600080BD00BF002D012080B584B000AF7860A7
:10AF70001C21012007F0A2FAF860FB68002B02D127
:10AF80006FF00B0325E0FB68184608F01DFAFB681C
:10AF900000221A717B681A68FB689A607B685A689D
:10AFA000FB68DA607B685A7AFB681A747B689A7A65
:10AFB000FB685A747B68DA68FB685A617B689A6937
:10AFC000FB689A617B681B680449FA6841F8232092
:10AFD000002318461037BD4680BD00BF002D01205C
:10AFE00080B582B000AF78607B68002B03D07B68AF
:10AFF0001B69002B02D16FF0150317E07B681B68FB
:10B00000002B05D07B681B689B68184600F012F87F
:10B010007B681B695B69002B02D16FF0570305E069
:10B020007B681B695B697868984703461846083750
:10B03000BD4680BD80B584B000AF7860144A7B689F
:10B0400052F82330FB60FB681B79002B05D0FB68AE
:10B050001B79013BDAB2FB681A71FB681B79002B84
:10B0600011D1FB681B68184608F0C9F9FB68002B72
:10B0700009D0F86807F030FA0023FB60044A7B68C7
:10B08000002142F8231000BF1037BD4680BD00BF2D
:10B09000002D012080B586B000AFF860B96013467E
:10B0A000FB80FB68002B03D0FB681B69002B02D1DF
:10B0B0006FF015031CE0FB681B695B68002B02D175
:10B0C0006FF0570314E0FB681B681B68184608F014
:10B0D00084F9FB681B695B68FA88B968F868984767
:10B0E0007861FB681B681B68184608F07FF97B696C
:10B0F00018461837BD4680BD80B584B000AF786073
:10B1000039603B68002B07D03B685B69002B03D09C
:10B110003B681B780A2B02D96FF015032AE03B68C5
:10B120005B691B68002B02D16FF0570322E03B687C
:10B130005B691B68396878689847F860FB68002B82
:10B1400001D0FB6816E07B681B683A6852695A6157
:10B150003B681B789B00094A1344184608F034F9F1
:10B160003B681B7819467B681B68044A52F821200B
:10B170001A60002318461037BD4680BD242D0120DB
:10B1800080B582B000AF78607B68002B03D07B680D
:10B190005B69002B02D16FF0150319E07B685B69D6
:10B1A0005B69002B02D16FF0570311E07B681B68CD
:10B1B000184608F024F97B681B791946064B0022D3
:10B1C00043F821207B685B695B6978689847034690
:10B1D00018460837BD4680BD242D012080B586B0B5
:10B1E00000AFF860B9607A60FB68002B06D0FB689E
:10B1F0005B69002B02D0BB68002B02D16FF01503F6
:10B200001AE0FB685B695B68002B02D16FF05703A3
:10B2100012E0FB681B68184608F0DFF8FB685B6902
:10B220005B687A68B968F86898477861FB681B685A
:10B23000184608F0DBF87B6918461837BD4680BD14
:10B2400080B586B000AFF860B9607A60FB68002B0B
:10B2500006D0FB685B69002B02D0BB68002B02D1D3
:10B260006FF015031AE0FB685B699B68002B02D145
:10B270006FF0570312E0FB681B68184608F0ADF842
:10B28000FB685B699B687A68B968F8689847786179
:10B29000FB681B68184608F0A9F87B691846183740
:10B2A000BD4680BD80B584B000AF78600B46FB70B2
:10B2B0007B689B68002B03D07B681B68002B02D146
:10B2C0006FF0150313E07B681B6800211846FFF739
:10B2D000B3FCF860FB68002B01D0FB6807E07B68DB
:10B2E0009B68F91C01221846FFF7D4FE0346184656
:10B2F0001037BD4680BD80B584B000AF78600B4686
:10B30000FB707B689B68002B03D07B681B68002B5D
:10B3100002D16FF0150313E07B681B68012118460A
:10B32000FFF78AFCF860FB68002B01D0FB6807E0A0
:10B330007B689B68F91C01221846FFF7ABFE0346A9
:10B3400018461037BD4680BD80B5ADF50C7D00AF09
:10B3500007F50C73A3F50B73186007F50C73A3F5D1
:10B360000C73196007F50C73A3F5097318464FF4B5
:10B3700000731A46002113F077FCB02387F82732B8
:10B3800007F50C73A3F50C73186814F039FB03462A
:10B39000C7F820320023C7F81C32D7F81C22D7F890
:10B3A00020321344802B05DDD7F81C32C3F1800313
:10B3B000C7F820320023C7F8283247E0D7F81C220C
:10B3C000D7F82832134403F03F03C7F81432D7F8F4
:10B3D00014321B11C7F81032D7F81432DB0003F017
:10B3E0007803C7F80C320023C7F82C3225E0D7F8D1
:10B3F000143207F50C72A2F50C72126813441B7814
:10B400001846D7F80C22D7F82C3213446349C200EF
:10B410001144D7F82C220A44107807F50C72A2F5D3
:10B420000971D7F81022D2010A44134402461A7057
:10B43000D7F82C320133C7F82C32D7F82C32072B2F
:10B44000D5D9D7F828320133C7F82832D7F82032B7
:10B45000D7F828229A42B1D307F50C73A3F50B73E2
:10B46000AE211868FFF71EFFC7F81802D7F8183288
:10B47000002B02D0D7F818328AE007F50C73A3F539
:10B480000B7340211868FFF70DFFC7F81802D7F8B3
:10B490001832002B02D0D7F8183279E00023C7F811
:10B4A0002C3268E097F8272207F50C73A3F50B738D
:10B4B00011461868FFF7F6FEC7F81802D7F81832D9
:10B4C000002B02D0D7F8183262E007F50C73A3F511
:10B4D0000B7310211868FFF7E5FEC7F81802D7F8BC
:10B4E0001832002B02D0D7F8183251E007F50C7350
:10B4F000A3F50B7300211868FFF7D4FEC7F81802F4
:10B50000D7F81832002B02D0D7F8183240E00023C9
:10B51000C7F8283221E007F50C73A3F50972D7F8B4
:10B520002C32DB011A44D7F8283213441A7807F575
:10B530000C73A3F50B7311461868FFF7DCFEC7F810
:10B540001802D7F81832002B02D0D7F818321FE0B3
:10B55000D7F828320133C7F82832D7F828327F2BA2
:10B56000D9D997F82732013387F82732D7F82C3208
:10B570000133C7F82C32D7F82C32032B92D907F5B8
:10B580000C73A3F50B73AF211868FFF78BFE03460E
:10B59000184607F50C77BD4680BD00BFC8C1021034
:10B5A00080B586B000AF7860B023FB74AE217868B8
:10B5B000FFF778FEB860BB68002B01D0BB684CE099
:10B5C00040217868FFF76EFEB860BB68002B01D0A1
:10B5D000BB6842E000237B6137E0FB7C194678685A
:10B5E000FFF760FEB860BB68002B01D0BB6834E099
:10B5F00010217868FFF756FEB860BB68002B01D0B9
:10B60000BB682AE000217868FFF74CFEB860BB6891
:10B61000002B01D0BB6820E00023FB600CE0002180
:10B620007868FFF768FEB860BB68002B01D0BB6884
:10B6300013E0FB680133FB60FB687F2BEFD9FB7CD9
:10B640000133FB747B6901337B617B69032BC4D9B4
:10B65000AF217868FFF726FE034618461837BD4627
:10B6600080BD80B586B000AFF860384680E80E0037
:10B670000C21012006F022FF38613B69002B02D12A
:10B680006FF00B03C3E03B690833BA6811461846F4
:10B69000FFF706FC78617B69002B40F0B3803B69C3
:10B6A0003A6811461846FFF71BFA78617B69002B50
:10B6B00040F0A1803B6904337A6811461846FFF7D1
:10B6C0003CFA78617B69002B40F08E803B691B68F7
:10B6D00000211846FFF78AFA78617B69002B66D152
:10B6E0003B695B68002B16D03B695B6800211846FC
:10B6F000FFF77CFA78617B69002B5AD1032000F0B8
:10B700009DF83B695B6801211846FFF795FA78615F
:10B710007B69002B4FD1A0213869FFF7C3FD786109
:10B720007B69002B49D1AE213869FFF7BBFD7861F9
:10B730007B69002B43D1C8213869FFF7B3FD7861DD
:10B740007B69002B3DD1A2213869FFF7ABFD786101
:10B750007B69002B37D12F213869FFF7A3FD786172
:10B760007B69002B31D121213869FFF79BFD78617E
:10B770007B69002B2BD181213869FFF793FD78611C
:10B780007B69002B25D120213869FFF78BFD78617B
:10B790007B69002B1FD13869FFF702FF78617B6955
:10B7A000002B1AD1FB683A691A6000232FE000BF12
:10B7B00014E000BF12E000BF10E000BF0EE000BFC9
:10B7C0000CE000BF0AE000BF08E000BF06E000BFD9
:10B7D00004E000BF02E000BF00E000BF3B695B681F
:10B7E0001846FFF7E1F900E000BF3B691B68184607
:10B7F000FFF7DAF900E000BF3B699B681846FFF7E6
:10B80000EFFB00E000BF386906F066FE7B69184672
:10B810001837BD4680BD0000B0B500AFF9F75AF942
:10B82000054BD3E90023541C43F10005024BC3E947
:10B83000004500BFB0BD00BF502D012080B582B0D3
:10B8400000AF78607868F9F76FFA00BF0837BD4637
:10B8500080BD80B582B000AF78607B684FF47A72AB
:10B8600002FB03F31846F9F75FFA00BF0837BD463D
:10B8700080BD80B485B000AFF860B9601346FB713D
:10B88000FB79002B06D0FB681A68BB681A43FB687B
:10B890001A6006E0FB681A68BB68DB431A40FB6865
:10B8A0001A6000BF1437BD4680BC704780B588B0B1
:10B8B00000AF786039603B68002B07D03B681B699C
:10B8C000002B03D03B685B681F2B02DD6FF0150374
:10B8D00094E01421012006F0F1FD78617B69002BD2
:10B8E00002D16FF00B0389E00C21012006F0E6FD88
:10B8F00038613B69002B03D16FF00B03FB6179E0EA
:10B900003B681B69FB603B681B7A022B0CD0022B47
:10B910000DDC002B02D0012B03D008E00023BB611B
:10B9200009E00123BB6106E00223BB6103E06FF085
:10B930001503FB615BE03B681B68032B03DD6FF0C5
:10B940001503FB6153E03B681B68002B13D03B6879
:10B950001B68012B0DD03B681B68022B07D03B688E
:10B960001B68032B01D1274B06E0002304E0264B84
:10B9700002E0264B00E0264B3A6913603B685B68A7
:10B98000012202FA03F31A463B695A60BB69DAB234
:10B990003B695A723B6900221A72FB681A783B694C
:10B9A0009A723B681A687B691A603B685A687B69BF
:10B9B0005A603B681A7A7B691A727B693A691A6124
:10B9C0003B681B681846F7F72BFB7B691B69184619
:10B9D000F7F752FBF861FB69002B03D06FF01503FA
:10B9E000FB6104E07B687A691A60002306E038692D
:10B9F00006F072FD786906F06FFDFB691846203786
:10BA0000BD4680BD00B0004000A000400090004056
:10BA10000080004080B582B000AF786039603B683C
:10BA2000002B04D17B6800221A60002304E03968EF
:10BA30007868FFF73BFF034618460837BD4680BDD0
:10BA400080B582B000AF78607B68002B02D16FF0C8
:10BA5000150308E07B681B69184606F03DFD786811
:10BA600006F03AFD002318460837BD4680BD80B574
:10BA700084B000AF78607B68002B03D07B685B6884
:10BA80001F2B02DD6FF0150309E07B681B69FB606B
:10BA9000FB6800221A72F868F7F7EEFA00231846DE
:10BAA0001037BD4680BD80B584B000AF78600B46CE
:10BAB000FB707B68002B06D07B685B681F2B02DC69
:10BAC000FB78012B02D96FF0150330E07B681B690E
:10BAD000FB60FB681B68BB60FB6801221A72F86898
:10BAE000F7F7CAFA7B685B68012202FA03F30122C6
:10BAF0001946B868FFF7BDFEFB78002B02D0012B7A
:10BB00000AD013E07B685B68012202FA03F319464E
:10BB1000B868F7F79AFB09E07B685B68012202FAD4
:10BB200003F31946B868F7F783FB00BF00231846F4
:10BB30001037BD4680BD80B485B000AF78603960F5
:10BB40007B68002B03D07B685B681F2B02DD6FF0E6
:10BB500015030EE07B681B69FB60FB681B7A012BF9
:10BB600003D13B6801221A7002E03B6800221A7080
:10BB7000002318461437BD4680BC704780B584B09A
:10BB800000AF78600B46FB707B68002B03D07B68AE
:10BB90005B681F2B02DD6FF015033CE07B681B69BF
:10BBA000FB60FB681B68BB607B685B68012202FA74
:10BBB00003F301221946B868FFF75BFEFB78022BFE
:10BBC0001AD0022B23DC002B02D0012B0AD01EE05E
:10BBD0007B685B68012202FA03F31946B868F7F73D
:10BBE00034FB17E07B685B68012202FA03F3194615
:10BBF000B868F7F71DFB0DE07B685B68012202FA6D
:10BC000003F300221946B868FFF733FE02E06FF035
:10BC1000150300E0002318461037BD4680BD80B5EF
:10BC200084B000AF786039607B68002B03D07B68FC
:10BC30005B681F2B02DD6FF0150337E07B681B6923
:10BC4000FB60FB681B68BB607B685B68012202FAD3
:10BC500003F301221946B868FFF70BFEFB681B7A55
:10BC6000002B11D17B685B68012202FA03F31946AD
:10BC7000B868F7F7CFFA02467B685B6822FA03F3ED
:10BC8000DAB23B681A7010E07B685B68012202FA46
:10BC900003F31946B868F7F7E5FA02467B685B6874
:10BCA00022FA03F3DAB23B681A7000231846103701
:10BCB000BD4680BD80B500AF0020F7F7FAFA00BF9F
:10BCC00080BD80B500AF0120F7F7F3FA00BF80BD5B
:10BCD00080B500AF0220F7F7ECFA00BF80BD80B559
:10BCE00000AF0320F7F7E5FA00BF80BD80B500AFD5
:10BCF0000248F7F78DFC00BF80BD00BF00D00140B7
:10BD000080B500AF0248F7F783FC00BF80BD00BFDD
:10BD100000E0014080B483B000AF03463960FB719E
:10BD200097F90730002B0BDA3B68DAB20C49FB7944
:10BD300003F00F03043B5201D2B20B441A7609E020
:10BD40003B68DAB2074997F907305201D2B20B4487
:10BD500083F8002300BF0C37BD4680BC704700BF8E
:10BD600000ED00E000E100E080B582B000AF786057
:10BD70007B68013BB3F1807F01D301230FE00A4AC6
:10BD80007B68013B536007214FF0FF30FFF7C2FF94
:10BD9000054B00229A60044B07221A6000231846C4
:10BDA0000837BD4680BD00BF10E000E080B500AFA1
:10BDB000074B1B68074AA2FB03239B091846FFF7A2
:10BDC000D3FF0120F8F7B0FF0346184680BD00BF3F
:10BDD000B01F0020D34D621080B500AFFFF7E6FF23
:10BDE0000346184680BD000080B483B000AF034610
:10BDF000FB71FB7903F01F03012202FA03F1054AEC
:10BE000097F907305B0942F8231000BF0C37BD4695
:10BE100080BC704700E100E080B483B000AF03460F
:10BE2000FB71FB7903F01F03012202FA03F1064ABA
:10BE300097F907305B09203342F8231000BF0C3715
:10BE4000BD4680BC704700BF00E100E080B483B015
:10BE500000AF03463960FB7197F90730002B0BDA0E
:10BE60003B68DAB20C49FB7903F00F03043B520143
:10BE7000D2B20B441A7609E03B68DAB2074997F967
:10BE800007305201D2B20B4483F8002300BF0C37B5
:10BE9000BD4680BC704700BF00ED00E000E100E05F
:10BEA00080B483B000AF786039603B68002B4CD021
:10BEB0003B68012B47D03B68022B42D03B68032BE9
:10BEC0003DD03B68042B38D03B68052B33D03B6812
:10BED000062B2ED03B68072B29D03B68082B24D09B
:10BEE0003B68092B1FD03B680A2B1AD03B680B2BF1
:10BEF00015D03B680C2B10D03B680D2B0BD03B684A
:10BF00000E2B06D03B680F2B01D14F231EE00023E0
:10BF10001CE04E231AE04D2318E04C2316E04B237F
:10BF200014E04A2312E0492310E048230EE047239F
:10BF30000CE046230AE0452308E0442306E01F23E3
:10BF400004E01E2302E01D2300E01C2318460C37EA
:10BF5000BD4680BC704780B483B000AF7860396064
:10BF60007B681A683B681B68D31A18460C37BD46B5
:10BF700080BC704780B485B000AF78600023FB6060
:10BF80001CE0FB68002B10D0FB68012B0BD0FB687A
:10BF9000022B06D0FB68032B01D13A2306E00023D5
:10BFA00004E01A2302E0192300E018237A68934280
:10BFB00001D1012306E0FB680133FB60FB68032B22
:10BFC000DFD9002318461437BD4680BC70470000F7
:10BFD00080B58AB000AF786007F1100300221A60C4
:10BFE0005A609A60DA607B68404A93425BD07B6813
:10BFF0003E4A934203D07B683D4A934251D07B68CE
:10C000003A4A934207D07B68394A934203D07B680F
:10C01000384A934243D07B68344A93420BD07B68C2
:10C02000334A934207D07B68324A934203D07B68FD
:10C03000314A934231D07B682C4A93420FD07B68BF
:10C040002B4A93420BD07B682A4A934207D07B68E5
:10C05000294A934203D07B68284A93421BD07B68CD
:10C06000224A934215D07B68214A934211D07B68C3
:10C07000204A93420DD07B681F4A934209D07B68C7
:10C080001E4A934205D07B681D4A934201D10A2380
:10C090000AE0002308E0092306E0082304E0072360
:10C0A00002E0062300E005233B61164B7B627B6ABE
:10C0B0005B6807F1100207F10C01184606F079FFE2
:10C0C00038623B6A002B0DD1FB689B68002B05D0C2
:10C0D000FB689B68FA68D268104698477868F9F759
:10C0E00003F900E000BF2837BD4680BD00000140D5
:10C0F000001001400020014000300140004001409C
:10C1000000500140E40D002080B584B000AF78609D
:10C110007B68184A93420ED07B68174A934208D036
:10C120007B68164A934201D1022305E04FF0FF33AA
:10C1300002E0012300E000235B01114A1344FB608D
:10C140007868F9F71BFCFB681B68002B0ED0FB68B6
:10C150009B69002B03D1FB681B69002B03D1FB6893
:10C16000DB68002B02D0F868F9F7D2FB00BF10376C
:10C17000BD4680BD00200440003004400040044023
:10C180007C2D012080B500AF0248FFF7BDFF00BF46
:10C1900080BD00BF0020044080B500AF0248FFF71B
:10C1A000B3FF00BF80BD00BF0030044080B500AFCA
:10C1B0000248FFF7A9FF00BF80BD00BF0040044058
:10C1C00080B500AF0248FFF703FF00BF80BD00BF8E
:10C1D0000000014080B500AF0248FFF7F9FE00BF44
:10C1E00080BD00BF0010014080B500AF0248FFF7DE
:10C1F000EFFE00BF80BD00BF0020014080B58CB0C5
:10C2000000AF78602D4BFB622D4BBB6207F10C0336
:10C2100000221A605A609A60DA6079680020FFF79D
:10C220003FFE0346FB60274A7B6808335B011344EB
:10C2300004331B68234943F004027B6808335B0125
:10C240000B4404331A60FB6A5B68002B16D0FB6A50
:10C250005B6807F10C0207F12001184606F0A9FE01
:10C2600078627B6A002B09D13B6A9B68002B05D062
:10C270003B6A9B683A6AD26810469847BB6A5B681B
:10C28000002B16D0BB6A5B6807F10C0207F11C019A
:10C29000184606F08EFE78627B6A002B09D1FB6996
:10C2A0009B68002B05D0FB699B68FA69D268104631
:10C2B000984700BF3037BD4680BD00BFF40D002059
:10C2C000040E00200080024080B500AF0020FFF780
:10C2D00095FF00BF80BD80B500AF0120FFF78EFF46
:10C2E00000BF80BD80B500AF0220FFF787FF00BF11
:10C2F00080BD80B500AF0320FFF780FF00BF80BD89
:10C3000080B500AF0420FFF779FF00BF80BD80B586
:10C3100000AF0520FFF772FF00BF80BD80B500AF02
:10C320000620FFF76BFF00BF80BD80B500AF072080
:10C33000FFF764FF00BF80BD80B500AF0820FFF7A6
:10C340005DFF00BF80BD80B500AF0920FFF756FF3D
:10C3500000BF80BD80B500AF0A20FFF74FFF00BFD0
:10C3600080BD80B500AF0B20FFF748FF00BF80BD48
:10C3700080B500AF0C20FFF741FF00BF80BD80B546
:10C3800000AF0D20FFF73AFF00BF80BD80B500AFC2
:10C390000E20FFF733FF00BF80BD80B500AF0F2038
:10C3A000FFF72CFF00BF80BD80B584B000AFF7F76A
:10C3B00043FD0346FB60124BBB60FB6803F0400388
:10C3C000002B19D04020F7F741FDBB685B683A4667
:10C3D0001146184606F0A1FD78607B68002B0ADB49
:10C3E0003B689B68002B07D03B689B683A68D26823
:10C3F0001046984700E000BF1037BD4680BD00BF23
:10C40000D40D002080B588B000AF07F108030022EA
:10C410001A605A609A60DA600223BB600E4BFB61BF
:10C42000FB695B6807F10802391D184606F0C1FD7B
:10C43000B861BB69002B0AD17B689B68002B07D0D1
:10C440007B689B687A68D2681046984700E000BF16
:10C450002037BD4680BD00BF0C0E002080B58AB0DD
:10C4600000AF786039607B681B68454A934210D002
:10C470007B681B68434A934209D07B681B68424A29
:10C48000934201D1022305E04FF0FF3302E0012384
:10C4900000E000233B6207F1080300221A605A60A3
:10C4A0009A60DA603B6A002B0BD03B6A012B06D006
:10C4B0003B6A022B01D1222304E0002302E00F2378
:10C4C00000E00E23BB603B68002B16D02F4B7B6235
:10C4D0003B6A002B0BD03B6A012B06D03B6A022B38
:10C4E00001D1294B04E0002302E0264B00E0244B5D
:10C4F0000B211846F9F7C2F918E07B68DA687B6807
:10C500005B699A4206D17B68DB68002B02D0204B26
:10C510007B620BE07B681A697B689B699A4229D130
:10C520007B681B69002B25D01A4B7B627B6A5B689A
:10C5300007F1080207F11801184606F03AFDF86104
:10C54000FB69002B18D1144A3B6A5B01134400229B
:10C550001A60BB699B68002B0FD0104B01221A7028
:10C56000BB699B68BA69D268104698470B4B00229A
:10C570001A7002E000BF00E000BF2837BD4680BD52
:10C58000002004400030044000400440CC0D002056
:10C59000BC0D0020C40D00207C2D0120DC2D0120CD
:10C5A00080B584B000AF786039603B68002B02D161
:10C5B0006FF0150323E0144B1B68002B05D0124BC2
:10C5C0001A687B681A60002319E01021012005F029
:10C5D00075FFF860FB68002B02D16FF00B030EE0D3
:10C5E0003B681A68FB681A603B689A68FB68DA6007
:10C5F0007B68FA681A60044AFB68136000231846D7
:10C600001037BD4680BD00BF582D012080B584B0D5
:10C6100000AF78607B68002B02D16FF015032FE02C
:10C620000023FB6022E0BB68184605F055FF164A60
:10C63000FB68DB0013445B6807F1080211461846EB
:10C6400006F0F0FC0346002BEDD00F4AFB68DB0040
:10C6500013445B68184606F03DFB0B4AFB68DB00A1
:10C66000134400225A60FB680133FB60FB680B2B0C
:10C67000DDD9786805F030FF044B00221A600023F2
:10C6800018461037BD4680BDB40D0020582D01203E
:10C6900080B58CB000AFF860B9607A60002387F88D
:10C6A0002B3007F1100300221A605A609A60DA609A
:10C6B000BB683B61B868FFF75DFC0346002B02D006
:10C6C0006FF05703BFE0FB68002B06D07B68002BA0
:10C6D00003D07B681B7A0B2B02D96FF01503B2E0F5
:10C6E0007B681B7A5A4ADB0013445B68002B10D12D
:10C6F0007B681B7ADB00564A13440433554A0321F6
:10C70000184606F0A3FAF862FB6A002B01D0FB6A18
:10C7100099E07B681B7A4E4ADB0013445B6807F1A3
:10C72000100207F12001184606F043FCF862FB6A8C
:10C73000002B2CD01021012005F0C0FE03463B62E7
:10C740003B6A002B02D16FF00B037CE03B6ABA68B6
:10C750001A603B6A7A68D2685A603B6A7A681268E3
:10C760009A603B6A7A685268DA607B681B7A384A5A
:10C77000DB0013445B683A6A1146184606F025FB55
:10C78000F862FB6A002B58D1012387F82B307B68B5
:10C790005B7A013B072B1DD801A252F823F000BFA2
:10C7A00005C80010C1C7001005C80010D5C700108B
:10C7B000D5C7001005C8001005C8001005C8001036
:10C7C0000220F7F719FBF862FB6A002B1CD06FF010
:10C7D0000F0338E097F82B30002B10D06FF01503C3
:10C7E000FB6200BF7B681B7A194ADB0013445B685D
:10C7F00007F124021146184606F055FC1EE06FF0C2
:10C80000150320E000BF00E000BF97F82B3083F055
:10C810000103DBB2002B0ED03B6ABA681A603B6A98
:10C820007A68D2685A603B6A7A6812689A603B6A92
:10C830007A685268DA60002305E000BF3B6A184658
:10C8400005F04AFEFB6A18463037BD4680BD00BF82
:10C85000B40D002057BF001080B58AB000AFF8605B
:10C86000B9607A6000233B6207F1100300221A606E
:10C870005A609A60DA60BB683B61B868FFF77AFB80
:10C880000346002B02D06FF0570332E0FB68002B09
:10C8900002D07B68002B02D16FF0150329E07B6882
:10C8A0005B7A012B02D0022B04D009E07B68DB68A5
:10C8B0007B6105E0114B7B610220F7F7ADFA00BF09
:10C8C0007B681B7A0E4ADB0013445B6807F1100299
:10C8D00007F12001184606F027FC78627B6A002BDE
:10C8E00002D06FF0120304E03B6A184605F0F4FD35
:10C8F0007B6A18462837BD4680BD00BF00600040F7
:10C90000B40D002080B485B000AFF860B960134664
:10C91000FB716FF0570318461437BD4680BC704753
:10C9200080B483B000AF786062B600BF00231846C1
:10C930000C37BD4680BC704780B483B000AF7860D0
:10C9400072B600BF002318460C37BD4680BC704746
:10C9500080B582B000AF786039603B68502B02D957
:10C960006FF0150305E03B685BB21846FFF73CFA31
:10C97000002318460837BD4680BD80B582B000AFA1
:10C98000786039603B68502B02D96FF0150305E0E1
:10C990003B685BB21846FFF73FFA0023184608379A
:10C9A000BD4680BD80B584B000AFF860B9607A60E4
:10C9B000BB68502B02D96FF0150306E0BB685BB271
:10C9C00079681846FFF742FA002318461037BD462B
:10C9D00080BD000080B588B000AFF860B9607A60B3
:10C9E0007B68FB61FB691B68DB69BB61FB691B68DA
:10C9F0005B68002B16D0FB691B685B68012B0FD0AE
:10CA0000FB691B685B68022B08D0FB691B685B68CD
:10CA1000032B01D1344B06E0002304E0334B02E04A
:10CA2000334B00E0334B7B6100BFBB69DA68FB69C5
:10CA30009B6819461046FEF71FF80346002B0AD0E4
:10CA4000BB69DA68FB695B6819461046FEF714F8A3
:10CA50000346002BE9D100BF7B691B6B03F0010388
:10CA6000002BF9D1BB68002B21D1FB695B69002B3E
:10CA700005D0FB695B69FA69926910469847FB69C2
:10CA80005B681846FDF746FFFB699B681846FDF793
:10CA900041FFFB69DB68184605F01EFDFB691B6959
:10CAA000184605F019FDF86905F016FD18E07B69D8
:10CAB0009A68BB689B681A437B699A60BB689B68ED
:10CAC00019460D4806F0C1FC02467B699B681A4373
:10CAD0007B699A607B695B6843F020027B695A60DE
:10CAE0002037BD4680BD00BF00E00B400080044001
:10CAF00000700440006004400000FFFF80B485B077
:10CB000000AF78607B68DB69FB607B685B68032B48
:10CB100026D801A252F823F029CB001037CB001001
:10CB200045CB001053CB0010FB6821225A61FB68F3
:10CB300001221A6115E0FB6822225A61FB68022279
:10CB40001A610EE0FB6823225A61FB6803221A6116
:10CB500007E0FB682F225A61FB680F221A6100E090
:10CB600000BF1437BD4680BC704700BF80B58AB097
:10CB700000AF78607B68DB697B627B685B68032B56
:10CB800000F2C28001A252F823F000BF9DCB00103A
:10CB9000C7CB001031CC00109DCC0010684A07F1C3
:10CBA000180307CA83E807007B681B7B002B07D1AB
:10CBB000644A07F10C0307CA83E8070000BFA6E038
:10CBC0006FF01503B7E0604A07F1180307CA83E85E
:10CBD00007007B681B7B032B26D801A252F823F0A9
:10CBE000F1CB0010FFCB00100DCC00101BCC0010BF
:10CBF000564A07F10C0307CA83E8070017E0544AB6
:10CC000007F10C0307CA83E8070010E0514A07F157
:10CC10000C0307CA83E8070009E04F4A07F10C0339
:10CC200007CA83E8070002E06FF0150383E06EE0B7
:10CC30004A4A07F1180307CA83E807007B681B7B91
:10CC4000032B27D801A252F823F000BF5DCC0010BF
:10CC50006BCC001079CC001087CC0010404A07F153
:10CC60000C0307CA83E8070017E03E4A07F10C03EC
:10CC700007CA83E8070010E03B4A07F10C0307CA24
:10CC800083E8070009E0394A07F10C0307CA83E883
:10CC9000070002E06FF015034DE038E0344A07F179
:10CCA000180307CA83E807007B681B7B032B27D880
:10CCB00001A252F823F000BFC9CC0010D7CC00105D
:10CCC000E5CC0010F3CC0010254A07F10C0307CA8D
:10CCD00083E8070017E0234A07F10C0307CA83E83B
:10CCE000070010E0204A07F10C0307CA83E8070099
:10CCF00009E0204A07F10C0307CA83E8070002E0B5
:10CD00006FF0150317E002E06FF0150313E07B6A84
:10CD10001B685B7987F822307B6A1B685B79BB757F
:10CD200007F118031846F6F7A7F907F10C031846A0
:10CD3000F6F7A2F9002318462837BD4680BD00BF8C
:10CD400008BA0210FCB9021014BA021020BA02107C
:10CD50002CBA021038BA021044BA021050BA0210AB
:10CD60005CBA021068BA021074BA021080BA0210DB
:10CD70008CBA021098BA021080B58AB000AF786001
:10CD800039607B68DB693B623B685B694FF47A72B0
:10CD900003FB02F27B685B691344FB613B689B69A0
:10CDA0004FF47A7203FB02F27B689B691344BB6108
:10CDB0003B6A5B68FA699A4205D13B6A9B68BA692B
:10CDC0009A4200F084807B685B68002B13D07B68FC
:10CDD0005B68012B0DD07B685B68022B07D07B68FA
:10CDE0005B68032B01D13C4B06E0002304E03B4B86
:10CDF00002E03B4B00E03B4B7B617B691B693B6185
:10CE00007869F7F78DF90346FB60FB685A08364BE3
:10CE10001344FA68B3FBF2F3BB603B6A5B68FA69E0
:10CE20009A4221D0FB69002B02D101237B6204E0EE
:10CE3000FA69BB68B2FBF3F37B627B6AFF2B03D911
:10CE40002A4811F0BFFF3EE07B691B6923F0FF0217
:10CE50007B691A61796AFF2006F0F7FA02467B695E
:10CE60001B691A437B691A613B6A9B68BA699A42DB
:10CE700022D0BB69002B02D101237B6204E0BA6996
:10CE8000BB68B2FBF3F37B627B6AFF2B03D91848C4
:10CE900011F098FF17E07B691B6923F47F427B69DF
:10CEA0001A61796A4FF47F4006F0CFFA02467B6937
:10CEB0001B691A437B691A613B6AFA695A603B6ACB
:10CEC000BA699A6004E07B693A691A6100E000BFC0
:10CED0002837BD4680BD00BF00E00B400080044005
:10CEE000007004400060044000CA9A3B14CA02105B
:10CEF00040CA021080B588B002AF78607B68DB69F9
:10CF00003B613B691B68FB607B685B68002B13D04F
:10CF10007B685B68012B0DD07B685B68022B07D0B8
:10CF20007B685B68032B01D15D4806E0002004E0CC
:10CF30005C4802E05C4800E05C48FB681B681946FE
:10CF4000FB681B791A467B689B68019300920B462D
:10CF500000220121F7F706F878617B69002B03D0E6
:10CF60006FF015037B617AE07868FFF7FFFD786169
:10CF70007B69002B72D17B685B68002B13D07B68C8
:10CF80005B68012B0DD07B685B68022B07D07B6848
:10CF90005B68032B01D1424B06E0002304E0414BC8
:10CFA00002E0414B00E0414B7A68527B1146184643
:10CFB000F7F72CF978617B69002B03D06FF015032C
:10CFC0007B614CE07B685B68002B13D07B685B68FF
:10CFD000012B0DD07B685B68022B07D07B685B68F8
:10CFE000032B01D12E4B06E0002304E02D4B02E081
:10CFF0002D4B00E02D4B01211846F7F7F7F878612B
:10D000007B69002B03D06FF015037B6127E07B6801
:10D010005B68002B13D07B685B68012B0DD07B68AD
:10D020005B68022B07D07B685B68032B01D11C4B2C
:10D0300006E0002304E01B4B02E01B4B00E01B4B0F
:10D0400008211846F7F7B8F878617B69002B03D000
:10D050006FF015037B6102E000231DE000BF7B68D9
:10D060005B68002B13D07B685B68012B0DD07B685D
:10D070005B68022B07D07B685B68032B01D1084BF0
:10D0800006E0002304E0074B02E0074B00E0074BFB
:10D090001846F6F7F7FF7B6918461837BD4680BD7E
:10D0A00000E00B4000800440007004400060044039
:10D0B00080B586B000AF786039603B68002B03D044
:10D0C0003B689B69002B02D16FF015036FE02421B0
:10D0D000012005F0F3F938613B69002B02D16FF0B4
:10D0E0000B0364E01821012005F0E8F9F860FB6803
:10D0F000002B03D16FF00B037B6151E03B689B6910
:10D10000BB603B681A683B695A603B685A683B6978
:10D110009A603B681A7A3B691A733B685A7A3B6992
:10D120005A733B689A7A3B699A73FB68BA681A60CB
:10D130003B69FA68DA613B695B68032B03D96FF0DE
:10D1400015037B612CE03869FFF7D4FE78617B69B9
:10D15000002B22D1BB689B68002B19D0BB68DA6812
:10D16000BB681B699A4203D36FF015037B6117E01C
:10D17000FB6803F10C02BB689B6819461046FDF77B
:10D180009CF978617B69002B09D13869FFF7B6FCFF
:10D190007B683A691A60002309E000BF00E000BF25
:10D1A000F86805F099F9386905F096F97B69184631
:10D1B0001837BD4680BD000080B582B000AF7860F2
:10D1C0007B68002B02D16FF0150324E07B685B685D
:10D1D000002B13D07B685B68012B0DD07B685B68EC
:10D1E000022B07D07B685B68032B01D10C4B06E058
:10D1F000002304E00B4B02E00B4B00E00B4B184606
:10D20000F6F740FF7B68DB69184605F065F978683A
:10D2100005F062F9002318460837BD4680BD00BFFF
:10D2200000E00B40008004400070044000600440B7
:10D2300080B58EB000AFF860B9607A603B60FB6883
:10D240005B68002B13D0FB685B68012B0DD0FB687B
:10D250005B68022B07D0FB685B68032B01D16B4B2B
:10D2600006E0002304E06A4B02E06A4B00E06A4BF0
:10D27000FB62FB68DB69BB6200237B63FB681B7B93
:10D280007B62FB685B68654A52F823307A6A9A428F
:10D290000ED0F868FFF72EFE38633B6B002B01D0F1
:10D2A0003B6B15E2FB685B685C497A6A41F82320B6
:10D2B000FB6A5B6823F47022FB6A5A60FB681B7B85
:10D2C0001A460123934019464FF4702006F0BDF82A
:10D2D0000246FB6A5B681A43FB6A5A60242178683D
:10D2E00005F0ECF838623B6A002B02D16FF00B03BB
:10D2F000EEE12421786805F0E1F8F861FB69002B84
:10D3000003D16FF00B033B63DEE11C21012005F02C
:10D31000D5F8B861BB69002B03D16FF00B033B63F9
:10D32000CFE1FB6ADB6943F08012FB6ADA61FB6ADA
:10D330001B6A43F40062FB6A1A62BB681B7B002B0A
:10D3400006D0FB6A5B6823F48072FB6A5A6005E0D2
:10D35000FB6A5B6843F48072FB6A5A60BB689A6838
:10D36000FB6A9A60FB6ADB6943F04002FB6ADA61A0
:10D37000BB689B6819462A4806F067F80246FB6AB4
:10D380009B681A43FB6A9A60FB6ADB6943F480027C
:10D39000FB6ADA61FB6ADB6943F08022FB6ADA61CF
:10D3A000BB6ADB6807F1140211461846FDF78CF9D9
:10D3B00038633B6B002B40F08081BB6ADB6807F170
:10D3C000100211461846FDF77FF938633B6B002BBE
:10D3D00040F06A81BB69FA681A603A69BB699A6071
:10D3E0007A69BB695A60BB69FA69DA60BB693A6AF3
:10D3F0001A6197F84430002B05D0BB693A685A612E
:10D40000BB693A6C9A6100237B63C2E000E00B4089
:10D410000080044000700440006004405C2D012046
:10D420000000FFFF7A6B1346DB009B1A9B001A4635
:10D43000BB6899187A6B1346DB0013449B001A46AD
:10D44000FB6913440A681A60BB6A59697A6B134610
:10D45000DB0013449B001A46FB6913440A465A60DA
:10D460007A6B1346DB009B1A9B001A46BB6899181F
:10D470007A6B1346DB0013449B001A46FB69134486
:10D480008A689A607A6B1346DB0013449B001A4645
:10D49000FB69134407221A777A6B1346DB001344A7
:10D4A0009B001A46FB6913448B4A1A617A6B134638
:10D4B000DB0013449B001A46FB691344BA695A61A6
:10D4C0007A6B1346DB0013449B001A46FB69134436
:10D4D00001221A73BB6A19687A6B1346DB00134486
:10D4E0009B001A46FB6913440A699A617A6B1346DA
:10D4F000DB009B1A9B001A46BB6899187A6B13468F
:10D50000DB0013449B001A463B6A13444A685A6086
:10D51000BB6A19697A6B1346DB0013449B001A46F9
:10D520003B6A13440A461A607A6B1346DB009B1A67
:10D530009B001A46BB6899187A6B1346DB001344AC
:10D540009B001A463B6A13448A689A607A6B1346BA
:10D55000DB0013449B001A463B6A134407221A77E8
:10D560007A6B1346DB0013449B001A463B6A134454
:10D5700002221A73BB6A19687A6B1346DB001344E4
:10D580009B001A463B6A1344CA689A617B6B01335D
:10D590007B637A6B7B689A42FFF444AFBB6AD868BE
:10D5A0007B697A68F969FDF7FFF838633B6B002BFC
:10D5B00071D1BB6AD8683B697A68396AFDF7F4F8BB
:10D5C00038633B6B002B52D1FB6A5B6843F020024F
:10D5D000FB6A5A60BB6ADB683A6911461846FDF778
:10D5E000B6F938633B6B002B43D1BB6ADB687A69C1
:10D5F00011461846FDF7ABF938633B6B002B3AD167
:10D6000097F8443083F00103DBB2002B2DD000BF2C
:10D61000BB6ADB683A6911461846FDF71CFA0346F7
:10D6200083F00103DBB2002BF2D1BB6ADB687A69BD
:10D6300011461846FDF70FFA034683F00103DBB2EB
:10D64000002BE5D100BFFB6A1B6B03F00103002B2D
:10D65000F9D1FB6A5B6823F02002FB6A5A60FB6A1F
:10D66000DB6923F04012FB6ADA61002330E000BF7F
:10D6700002E000BF00E000BFBB6ADB687A691146C8
:10D680001846FDF7A0F9BB6ADB683A6911461846EF
:10D69000FDF799F900E000BFBB6ADB683A69114603
:10D6A0001846FDF74FF800E000BFBB6ADB687A69F7
:10D6B00011461846FDF746F800E000BFB86904F0CF
:10D6C0000BFFF86904F008FF386A04F005FF3B6BB4
:10D6D00018463837BD4680BDD5C9001080B586B024
:10D6E00002AFF860B9607A600023019300230093D1
:10D6F00000237A68B968F868FFF79AFD0346184670
:10D700001037BD4680BD80B586B002AFF860B96005
:10D710007A603B6001230193BB6900933B687A68A0
:10D72000B968F868FFF784FD034618461037BD4610
:10D7300080BD000080B58CB000AFF860B9607A6041
:10D74000FB685B68002B13D0FB685B68012B0DD076
:10D75000FB685B68022B07D0FB685B68032B01D179
:10D760007F4B06E0002304E07E4B02E07E4B00E0AE
:10D770007E4BFB61012387F82730012387F8263091
:10D7800000233B62FB68002B02D0BB68002B02D158
:10D790006FF01503B2E1FB681B7BBB61FB685B6844
:10D7A000734A52F82330BA699A420ED0F868FFF7EC
:10D7B000A1FB78617B69002B01D07B699EE1FB684E
:10D7C0005B686B49BA6941F82320FB695B6823F405
:10D7D0007022FB695A60FB681B7B1A460123934049
:10D7E00019464FF4702005F030FE0246FB695B6875
:10D7F0001A43FB695A6000233B6279E1FB69DB69EC
:10D8000043F08012FB69DA61FB691B6A43F4006232
:10D81000FB691A62FB6900229A600023BB62002345
:10D82000FB623A6A1346DB009B1A9B001A46BB68F0
:10D8300013441B7B002B06D0FB695B6823F48072CA
:10D84000FB695A6005E0FB695B6843F48072FB6921
:10D850005A603A6A1346DB009B1A9B001A46BB6863
:10D8600013441946F868FFF787FA3A6A1346DB0053
:10D870009B1A9B001A46BB6813441B68002B41D0BF
:10D880003A6A1346DB009B1A9B001A46BB68134496
:10D890009A68FB699A60002387F82630FB69DB6988
:10D8A00043F04002FB69DA613A6A1346DB009B1AD7
:10D8B0009B001A46BB6813441A68FB6AD1183A6A7F
:10D8C0001346DB009B1A9B001A46BB6813449A68F8
:10D8D000FB6AD31A1A46F869F6F7C4FC0246FB6ADB
:10D8E0001344FB623A6A1346DB009B1A9B001A46FC
:10D8F000BB6813449B68FA6A9A420CBF0123002359
:10D9000087F826303A6A1346DB009B1A9B001A46BA
:10D91000BB6813445B68002B1BD03A6A1346DB00DC
:10D920009B1A9B001A46BB6813449B681946114812
:10D9300005F08BFD0246FB699B681A43FB699A6000
:10D94000FB69DB6943F48002FB69DA61002387F835
:10D950002730FB695B6843F02002FB695A6095E061
:10D9600000E00B4000800440007004400060044070
:10D970006C2D01200000FFFF3A6A1346DB009B1A62
:10D980009B001A46BB6813441B68002B39D03A6AC7
:10D990001346DB009B1A9B001A46BB6813449B6826
:10D9A000FA6A9A422DD23A6A1346DB009B1A9B0010
:10D9B0001A46BB6813441A68FB6AD1183A6A1346C0
:10D9C000DB009B1A9B001A46BB6813449A68FB6AEB
:10D9D000D31A1A46F869F6F745FC0246FB6A134467
:10D9E000FB623A6A1346DB009B1A9B001A46BB682F
:10D9F00013449B68FA6A9A420CBF0123002387F8FC
:10DA000026303A6A1346DB009B1A9B001A46BB6815
:10DA100013445B68002B39D03A6A1346DB009B1A2B
:10DA20009B001A46BB6813449B68BA6A9A422DD27F
:10DA30003A6A1346DB009B1A9B001A46BB681344E4
:10DA40005A68BB6AD1183A6A1346DB009B1A9B00DE
:10DA50001A46BB6813449A68BB6AD31A1A46F86917
:10DA6000F6F7E4FB0246BB6A1344BB623A6A13460C
:10DA7000DB009B1A9B001A46BB6813449B68BA6A7A
:10DA80009A420CBF0123002387F8273097F82730EC
:10DA900083F00103DBB2002B7FF46EAF97F82630E2
:10DAA00083F00103DBB2002B7FF466AF00BFFB699C
:10DAB0001B6A03F40063002BF9D0FB695B6823F059
:10DAC0002002FB695A60FB69DB6923F04012FB69A5
:10DAD000DA613A6A1346DB009B1A9B001A46BB6860
:10DAE00013441B691846FDF7A9FE3B6A01333B62EC
:10DAF0003A6A7B689A42FFF481AE002318463037B9
:10DB0000BD4680BD80B58CB000AFF860B9601346EB
:10DB1000FB8007F1140300221A605A609A60DA60F1
:10DB20001A615A619A61BB687B61BB68BB61FB8803
:10DB3000FB61012387F8203007F114030122194605
:10DB4000F868FFF7F7FD034618463037BD4680BD3D
:10DB500080B586B000AF78600B46FB707B68022B07
:10DB600017D07B68022B1BD87B68002B03D07B6807
:10DB7000012B07D014E0124A07F10C0307CA83E80F
:10DB8000070010E00F4A07F10C0307CA83E80700FB
:10DB900009E00D4A07F10C0307CA83E8070002E019
:10DBA0006FF0150307E0FB78BB7507F10C0318460F
:10DBB000F5F762FA002318461837BD4680BD00BF4E
:10DBC000B4B90210CCB90210E4B9021080B586B025
:10DBD00000AFF860B9607A6000237B61FB68002BBE
:10DBE00005D0BB68002B02D07B68002B02D16FF000
:10DBF000150343E0FB68DB68002B1FD000237B612B
:10DC000016E0FB68D868BA687B691344194604F0CB
:10DC1000F8FE38613B69002B07D07B69002B01D0EF
:10DC20007B692BE06FF00A0328E07B6901337B619D
:10DC30007B687A699A42E4D37B691FE0FB681B79B1
:10DC4000002B0DD0FB681B79012B07D0FB681B79DB
:10DC5000022B01D10B4B04E0002302E00A4B00E051
:10DC60000A4B3A1DB9681846F7F746FD38613B691B
:10DC7000002B02D06FF0040300E07B6818461837D1
:10DC8000BD4680BD004004400030044000200440F8
:10DC900080B588B000AFF860B9607A600023FB619E
:10DCA000FB68002B05D0BB68002B02D07B68002BE3
:10DCB0004ED16FF015034FE07B68202B28BF202347
:10DCC0007B6100BFFB681B79002B0DD0FB681B79C3
:10DCD000012B07D0FB681B79022B01D1204B04E0FC
:10DCE000002302E01F4B00E01F4B1846F7F7EEFD44
:10DCF000034603F04003002BE4D0FB681B79002BA4
:10DD00000DD0FB681B79012B07D0FB681B79022B18
:10DD100001D1134B04E0002302E0124B00E0124B50
:10DD2000FA69B968114407F114021846F7F7F4FCD0
:10DD3000B8617B69FA691344FB617B691A467B68A9
:10DD40009B1A7B60BB69002B02D06FF0040303E0D9
:10DD50007B68002BB0D1FB6918462037BD4680BDDB
:10DD600000400440003004400020044080B586B0EC
:10DD700000AFF860B9607A60FB68002B05D0BB6823
:10DD8000002B02D07B68002B02D16FF0150358E006
:10DD9000FB681B797B617B69002B0BD07B69012BB6
:10DDA00006D07B69022B01D1284B04E0002302E05E
:10DDB000274B00E0274B28497A6952010A44136037
:10DDC000254A7B695B0113440833BA681A60224A0A
:10DDD0007B695B01134410337A681A601E4A7B69C1
:10DDE0005B011344043300221A601B4A7B695B0108
:10DDF00013440C3300221A60174A7B695B011344F9
:10DE0000183300221A60144A7B695B0113441C33E7
:10DE1000124A1A60124B1B7883F00103DBB2002B0D
:10DE20000ED07B695B010C4A13441846F7F770FD6E
:10DE300038613B6913F1060F02D16FF00F0300E068
:10DE4000002318461837BD4680BD00BF004004407F
:10DE500000300440002004407C2D01205DC40010EF
:10DE6000DC2D012080B586B000AFF860B9607A6023
:10DE7000FB68002B05D0BB68002B02D07B68002B11
:10DE800002D16FF0150358E0FB681B797B617B6959
:10DE9000002B0BD07B69012B06D07B69022B01D1B3
:10DEA000284B04E0002302E0274B00E0274B2849E1
:10DEB0007A6952010A441360254A7B695B01134465
:10DEC0000433BA681A60224A7B695B0113440C333D
:10DED0007A681A601E4A7B695B011344083300228A
:10DEE0001A601B4A7B695B011344103300221A60DD
:10DEF000174A7B695B011344143300221A60144AE9
:10DF00007B695B0113441C33124A1A60124B1B7865
:10DF100083F00103DBB2002B0ED07B695B010C4A5E
:10DF200013441846F7F7F4FC38613B6913F1060F08
:10DF300002D16FF00F0300E0002318461837BD46EA
:10DF400080BD00BF00400440003004400020044079
:10DF50007C2D01205DC40010DC2D012080B584B033
:10DF600000AF78607B68FB60FB68DB68074A12786B
:10DF70001146184604F066FD01220449F868FFF7CF
:10DF8000F5FE00BF1037BD4680BD00BFDD2D01206E
:10DF900080B592B000AF786039603B68002B03D049
:10DFA0003B689B69002B02D16FF01503A4E11C2193
:10DFB000012004F083FA38633B6B002B02D16FF031
:10DFC0000B0399E10421012004F078FAF862FB6A5E
:10DFD000002B03D16FF00B037B6489E13B6BFA6A82
:10DFE0009A613B681B78002B0DD03B681B78012B96
:10DFF00007D03B681B78022B01D1944B04E000232F
:10E0000002E0934B00E0934BBB623B689B697B62F1
:10E010003B681A783B6B1A713B68DA683B6B1A6194
:10E020003B685B7C042B1CD801A252F823F000BF94
:10E0300045E000104BE0001051E0001057E00010E8
:10E040005DE0001000237B630FE003237B630CE0A3
:10E0500004237B6309E002237B6306E001237B63E7
:10E0600003E06FF015037B643FE13B681B7C032BEF
:10E0700016D801A252F823F089E000108FE00010BA
:10E0800095E000109BE000100523FB630CE00623E5
:10E09000FB6309E00723FB6306E00823FB6303E05F
:10E0A0006FF015037B6420E13B689B7C002B02D062
:10E0B000012B03D005E000233B6406E001233B6411
:10E0C00003E06FF015037B640FE17B6A1B78022B82
:10E0D0000CD0022B0DDC002B02D0012B03D008E06A
:10E0E0000023BB6309E00123BB6306E00223BB639B
:10E0F00003E06FF015037B64F7E03B6B1B69194687
:10E10000B86AF7F733F978647B6C002B03D06FF0B3
:10E1100015037B64E9E03B6B1B791A467B6A5B78ED
:10E1200019461046FFF714FD78647B6C002B40F015
:10E13000D480F96BB86AF7F703FA78647B6C002B2C
:10E1400003D06FF015037B64CCE07B6BDBB2194628
:10E15000B86AF7F713FA78647B6C002B03D06FF082
:10E1600015037B64BEE03B6CDBB21946B86AF7F777
:10E17000F5F978647B6C002B03D06FF015037B649A
:10E18000B0E0BB6BDBB208221946B86AF7F706FAB3
:10E1900078647B6C002B03D06FF015037B64A1E0E7
:10E1A0007B683A6B1A603B681B7A002B00F0888012
:10E1B0003B6B0C33184604F0D0FB78647B6C002B6F
:10E1C00040F08D8007F1180300221A605A609A60AF
:10E1D000214BFB61FB6A07F1180211461846FCF758
:10E1E00051FD78647B6C002B7BD11C4BBB603B6B7F
:10E1F000FB6002233B7401237B743B6B1B79002B78
:10E200000DD03B6B1B79012B07D03B6B1B79022B8D
:10E2100001D10E4B04E0002302E00D4B00E00D4B5A
:10E220007B61FB6A18683B6B1B79002B18D03B6B3A
:10E230001B79012B07D03B6B1B79022B01D12223C9
:10E240000FE000230DE00F230BE000BF004004406F
:10E250000030044000200440E8C902105DDF0010D7
:10E260000E2307F108021946FCF769FD78647B6C00
:10E27000002B27D1FB6A1A683B6B1B79002B0DD052
:10E280003B6B1B79012B07D03B6B1B79022B01D118
:10E29000222304E0002302E00F2300E00E231946AE
:10E2A0001046FCF794FD78647B6C002B0CD10122A6
:10E2B0001349386BFFF75AFD78647B6C002B05D14E
:10E2C000002319E000BF02E000BF00E000BFFB6ACE
:10E2D0001B681846FCF708FD04E000BF02E000BF21
:10E2E00000E000BFB86AF7F7CDF8F86A04F0F4F878
:10E2F000386B04F0F1F87B6C18464837BD4680BD9A
:10E30000DD2D012080B588B000AF786007F10C03E7
:10E3100000221A605A609A60DA6002233B7501237A
:10E320007B757B681B79002B0DD07B681B79012BDB
:10E3300007D07B681B79022B01D13D4B04E0002301
:10E3400002E03C4B00E03C4BBB617B68002B02D100
:10E350006FF0150367E07B689B69FB617B68DB6896
:10E36000002B41D0FB691A687B681B79002B0DD00C
:10E370007B681B79012B07D07B681B79022B01D1AD
:10E38000222304E0002302E00F2300E00E231946BD
:10E390001046FCF73EFDFB6918687B681B79002B73
:10E3A0000DD07B681B79012B07D07B681B79022B72
:10E3B00001D1222304E0002302E00F2300E00E231A
:10E3C00007F10C021946FCF7DEFCFB691B681846D6
:10E3D000FCF78AFC7B68DB68184604F054FB7B681A
:10E3E000DB68184604F078F87B681B79002B0DD0A9
:10E3F0007B681B79012B07D07B681B79022B01D12D
:10E400000B4B04E0002302E00A4B00E00A4B1846E5
:10E41000F7F738F87B689B69184604F05DF8786870
:10E4200004F05AF8002318462037BD4680BD00BFCF
:10E4300000400440003004400020044080B483B019
:10E4400000AF78606FF0570318460C37BD4680BCAC
:10E450007047000080B582B000AF78607B68002B09
:10E460000BD0084A7B681360074B1B689868002331
:10E470000222002110F0ACFE00E000BF0837BD46CC
:10E4800080BD00BFE02D0120D015002080B582B0F6
:10E4900000AF78607B68002B04DB7B68022B01DC1B
:10E4A000002306E010F04CF8034609221A604FF0F2
:10E4B000FF3318460837BD4680BD80B582B000AF37
:10E4C00078607B68002B04DB7B68022B01DC012376
:10E4D00005E010F035F8034609221A6000231846BB
:10E4E0000837BD4680BD80B584B000AFF860B96024
:10E4F0007A6010F025F8034609221A604FF0FF33C6
:10E5000018461037BD4680BD80B582B000AF786038
:10E5100039607B68002B08DB7B68022B05DC3B68DD
:10E520004FF400525A60002305E010F009F803464A
:10E5300009221A60002318460837BD4680BD000036
:10E5400080B586B000AFF860B9607A60FB68002BD8
:10E5500015D1104B1B687A68B9681846FCF73EFE67
:10E5600078617B69002B08DA0FF0EAFF02467B69CD
:10E570005B4213604FF0FF3308E07B6906E00FF069
:10E58000DFFF034609221A604FF0FF3318461837A1
:10E59000BD4680BDE02D012080B586B000AFF8609B
:10E5A000B9607A60FB68012B02D0FB68022B15D1A1
:10E5B000104B1B687A68B9681846FCF741FE786111
:10E5C0007B69002B08DA0FF0BBFF02467B695B42D8
:10E5D00013604FF0FF3308E07B6906E00FF0B0FFF7
:10E5E000034609221A604FF0FF3318461837BD461C
:10E5F00080BD00BFE02D012080B582B000AF786003
:10E60000F3F784F900BF0837BD4680BD80B582B0FE
:10E6100000AF78607868F6F787FB00BF0837BD4623
:10E6200080BD80B584B000AFF860B9607A60796869
:10E63000B868F3F793FB034618461037BD4680BD14
:10E6400080B584B000AFF860B9607A60F3F77CFB06
:10E650000346002B05D07968B868F3F7B7FB03468B
:10E6600001E06FF0120318461037BD4680BD80B43C
:10E6700085B000AFF860B9607A606FF05703184654
:10E680001437BD4680BC704780B485B000AFF860D9
:10E69000B9607A606FF0570318461437BD4680BCE6
:10E6A0007047000080B592B000AF786039603B6879
:10E6B000002B03D03B689B69002B02D16FF0150340
:10E6C00007E13B681B7A83F00103DBB2002B02D029
:10E6D0006FF01503FDE01C21012003F0EFFE38640C
:10E6E0003B6C002B02D16FF00B03F2E00421012000
:10E6F00003F0E4FEF863FB6B002B03D16FF00B0318
:10E700007B64E2E03B6CFA6B9A613B689B69BB639C
:10E71000BB6B002B07D0BB6B5A88704B5A81BB6B0D
:10E720001A886E4B1A816E4B00221A606D4B0022C4
:10E730001A606D4B00221A606C4B00221A60012394
:10E74000BB626B4BFB626B4B3B636B4B7B6307F1B9
:10E7500028031846F1F76AFF0346002B03D06FF039
:10E760000D037B64AEE0F3F73FFE0346002B03D0BE
:10E770006FF00D037B64A5E0002258490020F3F7F9
:10E7800095FE00225D490120F3F790FEBB6A002B45
:10E7900009D000225A490220F3F788FE0022594985
:10E7A0000320F3F783FE002257490420F3F77EFE8F
:10E7B000012256490420F3F779FE0222544904202D
:10E7C000F3F774FE032253490420F3F76FFE04228B
:10E7D00051490420F3F76AFE002250490220F3F762
:10E7E00023FE00224E490520F3F71EFE00224D496C
:10E7F0000620F3F719FE4C48F3F736F90346002BD1
:10E8000003D06FF00D037B645CE0002247490520D4
:10E81000F3F71CF8002245490620F3F717F844499E
:10E820000320F3F757F9434B00221A6000F06EF90A
:10E8300007F11C0300221A605A609A603E4B3B624B
:10E84000FB6B07F11C0211461846FCF71BFA7864B3
:10E850007B6C002B35D107F10C0300221A605A6043
:10E860009A60DA60354BFB600B233B7508237B75A0
:10E87000334BBB61FB6B18683B685B6807F10C02AC
:10E880001946FCF75CFA78647B6C002B10D1FB6BAB
:10E890001A683B685B6819461046FCF798FA78647A
:10E8A0007B6C002B06D17B683A6C1A60002310E069
:10E8B00000BF00E000BFFB6B1B681846FCF714FAB2
:10E8C00000E000BFF86B03F007FE386C03F004FEB5
:10E8D0007B6C18464837BD4680BD00BF140E002033
:10E8E000E42D0120E82D0120EC2D0120F02D012048
:10E8F0000DE6001099E90010DBE90010340E00204D
:10E90000780E0020280E0020BC0E0020C00E002033
:10E91000E40E0020080F00201C0F0020E9E9001081
:10E92000ADEA0010DDEA00103D0E00203DEB0010C6
:10E930007DEC0010F42D0120E8C90210F9E500106B
:10E9400000100B4080B584B000AF78607B68002B6E
:10E9500002D16FF0150310E07B689B69FB60FB68D8
:10E960001B681846FCF7C0F97B689B69184603F0E2
:10E97000B3FD786803F0B0FD002318461037BD469C
:10E9800080BD80B483B000AF78606FF05703184645
:10E990000C37BD4680BC704780B500AF4FF0804358
:10E9A0009B6803F40023002B11D14FF080439B6838
:10E9B0004FF0804243F4002393604FF00060F6F77D
:10E9C0007DFB0346002B02D06FF0090303E0032018
:10E9D000F6F741FA0023184680BD80B500AFF6F780
:10E9E0007BFC0346184680BD80B582B000AF7860DE
:10E9F00039607B685A88294B5B799BB29A423CD13B
:10EA0000274B01221A60274B5A01264B03F0704313
:10EA100003F10073243313441A46012313601F4B80
:10EA200093F8373003F00703DAB21F4B1A701B4B11
:10EA3000B3F839309AB21C4B5A80184B93F83E30D9
:10EA400003F00703DAB2184B1A71144BB3F84020E5
:10EA5000154BDA80114B93F8273003F00703DAB235
:10EA6000114B1A720D4BB3F829309AB20E4B5A81E2
:10EA70000D48F3F749F803460CE07B685B88002BF0
:10EA800006D1074B00221A60F3F716F9034601E09E
:10EA90004FF0FF3318460837BD4680BD340E0020C6
:10EAA000E42D0120EC2D01203C0F002080B483B028
:10EAB00000AF786039607B685B88012B04D1064B1E
:10EAC00001221A60002301E04FF0FF3318460C3793
:10EAD000BD4680BC704700BFF02D012080B483B0DC
:10EAE00000AF786039607B685B88012B04D1064BEE
:10EAF00000221A60002301E04FF0FF3318460C3764
:10EB0000BD4680BC704700BFF02D012080B400AF2F
:10EB1000034B01221A6000BFBD4680BC704700BF96
:10EB2000E82D012080B400AF034B00221A6000BF23
:10EB3000BD4680BC704700BFE82D012080B582B083
:10EB400000AF03463960FB71FB799B001946454BCA
:10EB500003F07042434B5B01134403F100730B4419
:10EB60001A4601231360FB79072B75D801A252F8CE
:10EB700023F000BF53EC001059EC001059EC0010CA
:10EB8000F9EB00104DEC001095EB0010BFEB0010FE
:10EB900013EC00100320F2F77FFE0420F2F77CFE56
:10EBA0000020F2F779FEF1F7F3FD2F4B00221A60F7
:10EBB000F4F7DCF8F3F780F8FFF7A8FF4DE0032047
:10EBC000F2F790FE002229490320F2F73FFE0720CA
:10EBD000F2F788FE002225490720F2F737FE0420CD
:10EBE000F2F780FE002221490420F2F72FFEF1F710
:10EBF000A1FDFFF78BFF30E0FFF794FFF4F7B6F8C5
:10EC0000F3F75AF8184B00221A60194B00221A60C9
:10EC100023E0F1F7D3FD034603F00203002B0AD0F3
:10EC2000002214490120F3F741FC0022124902207E
:10EC3000F3F73CFC11E000220F490120F3F736FC0A
:10EC400000220C490220F3F731FC06E0FFF75EFFDB
:10EC500003E0FFF767FF00E000BF00231846083716
:10EC6000BD4680BDEC2D0120E42D01203DEB0010C0
:10EC7000E82D0120780E0020340E002080B400AF73
:10EC8000034B01221A6000231846BD4680BC704722
:10EC9000F42D012080B584B000AF786039607B68C6
:10ECA000DB6E07F10C021146184603F08CFCFB6882
:10ECB000032B02D86FF00A0307E07B68DB6E0422A7
:10ECC0003968184603F038FE034618461037BD462B
:10ECD00080BD80B582B000AF786039607B68DB6E44
:10ECE00039460422184603F016FE03461846083734
:10ECF000BD4680BD80B586B000AFF860B9607A606F
:10ED0000FB681B687B617B695B6EFA6850687A6898
:10ED1000B9689847034618461837BD4680BD80B588
:10ED200086B000AFF860B9607A60FB681B687B61F1
:10ED30007B699B6EFA6850687A68B96898470346A1
:10ED400018461837BD4680BD80B584B002AF7860E4
:10ED500039603B6893F82130002B0FD03B681B795A
:10ED60001A46264B53F822203B68DB68244951F8A9
:10ED700023302449786810F085FB3AE03B6893F82B
:10ED80002230002B2AD03B6893F82330002B18D078
:10ED90003B681B791A46194B53F822103B68986858
:10EDA0003B681B791A46154B53F822303A68D268F3
:10EDB0000192009303460A461349786810F062FBFB
:10EDC00017E03B681B791A460C4B53F822203B682E
:10EDD0009B680E49786810F055FB0AE03B681B7988
:10EDE0001A46064B53F822301A460949786810F043
:10EDF00049FB00BF0837BD4680BD00BF50CE0210A2
:10EE000094CE021084CB02108CCB021098CB02104F
:10EE1000A0CB021080B596B000AFF860B960134681
:10EE2000FB710023A7F8563036E0BB689968B7F944
:10EE300056201346DB0013449B00CA1807F1140345
:10EE400011461846FFF780FF07F114031946F868CA
:10EE500010F0FAFB0346002B17D1BB689968B7F98D
:10EE600056201346DB0013449B000B4493F82030DC
:10EE7000FA799A4209D1BB689968B7F956201346C6
:10EE8000DB0013449B000B440DE0B7F956309BB2F6
:10EE900001339BB2A7F85630B7F95630BA6892885A
:10EEA0009342C2DB002318465837BD4680BD80B56B
:10EEB00084B000AF786039600023FB6018E07B68A5
:10EEC0001A6DFB68B02101FB03F31344396818463F
:10EED00010F0BAFB0346002B07D17B681A6DFB6864
:10EEE000B02101FB03F3134408E0FB680133FB602E
:10EEF0007B685B6DFA689A42E1D3002318461037AD
:10EF0000BD4680BD80B584B000AF78603960002315
:10EF1000FB601AE07B68996DFA6813469B00134406
:10EF20001B010B443968184610F08EFB0346002B7A
:10EF300008D17B68996DFA6813469B0013441B0146
:10EF40000B4408E0FB680133FB607B68DB6DFA680B
:10EF50009A42DFD3002318461037BD4680BD80B5E6
:10EF600086B000AFF860B9607A60FB681B687B61AF
:10EF7000B9687869FFF79BFF0346002B02D16FF059
:10EF8000120306E07B68012B02D06FF0150300E04E
:10EF9000002318461837BD4680BD80B483B000AF4B
:10EFA000786039606FF0150318460C37BD4680BC99
:10EFB000704780B483B000AF786039606FF015039C
:10EFC00018460C37BD4680BC7047F0B589B002AF1B
:10EFD000F860B9607A60FB700023FB8216E0B7F935
:10EFE000162013469B0013449B001A46BB6813442B
:10EFF0001B681946786810F027FB0346002B12D0D7
:10F00000B7F916309BB201339BB2FB82B7F91620D9
:10F0100013469B0013449B001A46BB6813441B68AD
:10F02000002BDCD100E000BFB7F9162013469B008F
:10F0300013449B001A46BB6813441B68002B02D183
:10F040006FF0010363E0FB78002B30D0B7F9162096
:10F0500013469B0013449B001A46BB6813441B696C
:10F06000002B02D16FF0010351E0B7F916201346CF
:10F070009B0013449B001A46BB6813441C69FB6841
:10F080001868FB685968FB689D68FB68DE68B7F91B
:10F09000162013469B0013449B001A46BB6813447A
:10F0A0005B68009333462A46A04703462FE0B7F932
:10F0B000162013469B0013449B001A46BB6813445A
:10F0C000DB68002B02D16FF0010320E0B7F91620B6
:10F0D00013469B0013449B001A46BB681344DC682C
:10F0E000FB681868FB685968FB689D68FB68DE6808
:10F0F000B7F9162013469B0013449B001A46BB68C1
:10F1000013445B68009333462A46A04703461846DB
:10F110001C37BD46F0BD000080B586B000AFF8607A
:10F12000B9607A6000233B61FB685B6D1B6BFA681A
:10F13000506CFA68116D07F11002984778617B698D
:10F14000002B01DA7B6906E03B69054A7968B868FB
:10F1500010F038F9034618461837BD4680BD00BF89
:10F16000A4CB021080B588B000AFF860B9607A60B7
:10F1700007F1100307F114021749B86810F0A2F95B
:10F180000346FB61FB69022B0DD1FB685B6D5B6B7A
:10F19000FA68506C79693A699847B861BB69002B85
:10F1A00015DABB6914E007F114031A460B49B86875
:10F1B00010F088F90346FB61FB69012B04D17A69E1
:10F1C000FB681A657B6803E06FF0150300E07B685D
:10F1D00018462037BD4680BDA8CB0210A4CB021034
:10F1E00080B485B000AF0346B9607A60FB73FB7BE7
:10F1F000042B1CD801A252F823F000BF11F200101A
:10F2000021F2001029F2001029F2001019F200106A
:10F21000BB685B6D1B690BE0BB685B6DDB6807E07F
:10F22000BB685B6D5B6903E07B68DB6900E0002322
:10F2300018461437BD4680BC704700BF80B483B009
:10F2400000AF03463960FB71FB79042B03D13B68A7
:10F250009B6C5B6801E000BF002318460C37BD467D
:10F2600080BC704780B590B000AFF860B9607A603C
:10F270003B600023FB63FB681B68B9681846FFF717
:10F2800016FEB863BB6B002B00F084807B681B7894
:10F29000002B17D17B685B685A49184610F0D4F9E7
:10F2A0000346002B0ED1BB6B5B6D1B6B002B06D096
:10F2B000BA6C3968B86BFFF72FFF03469DE06FF01B
:10F2C00001039AE07B689B681B78002B3AD07B682F
:10F2D0001B78022B0CBF01230023DBB287F82F30F1
:10F2E0007B689868BB6B596D97F92F30002B14BF62
:10F2F00001230023DBB21A46FFF78CFDF863FB6B9A
:10F30000002B02D16FF0010377E097F92F30002B2B
:10F3100014BF01230023DBB287F82230FB6B9B680C
:10F320001BB23B84FB6B1B7987F82330FB6B93F894
:10F33000233087F82430FB6B1B69BB6207F1200385
:10F34000FB6101E00023FB613B687B61BB6CBB613F
:10F35000BB6B5B6C3B617B681B78FA6BB96B1846C7
:10F36000FFF73EFF38637B685B681B78002B07D193
:10F3700007F11003396B1846FFF70FFE03463CE018
:10F380007B685A6807F110000023396BFFF71DFEF8
:10F39000034632E0FB681B68B9681846FFF7B2FD08
:10F3A00078637B6B002B26D00023FB613B687B617D
:10F3B000BB6CBB617B6B5B6C3B617B681B78796B67
:10F3C0001846FFF73BFF38637B685B681B78002BB0
:10F3D00007D107F11003396B1846FFF7DEFD03462E
:10F3E0000BE07B685A6807F110000023396BFFF7C8
:10F3F000ECFD034601E06FF0120318464037BD46AE
:10F4000080BD00BF10CC021080B590B000AFF86096
:10F41000B9607A603B600023FB63FB681B68B968D6
:10F420001846FFF744FDB863BB6B002B00F08180EA
:10F430007B681B78002B17D17B685B68584918469E
:10F4400010F002F90346002B0ED1BB6B5B6D5B6BBA
:10F45000002B06D0BA6C3968B86BFFF783FE034601
:10F460009AE06FF0010397E07B689B681B78002BA4
:10F4700037D07B681B78022B0CBF01230023DBB243
:10F4800087F82F307B689868BB6B596D97F92F30E0
:10F49000002B14BF01230023DBB21A46FFF7BAFC8E
:10F4A000F863FB6B002B02D16FF0010374E097F956
:10F4B0002F30002B14BF01230023DBB2BB74FB6B86
:10F4C0009B681BB23B82FB6B1B79FB74FB6B93F855
:10F4D00023303B75FB6B1B69BB6107F11003BB62FB
:10F4E00001E00023BB623B683B62BB6C7B62BB6B91
:10F4F0005B6CFB617B681B78FA6BB96B1846FFF796
:10F500006FFE38637B685B681B78002B07D107F1BF
:10F510001C03396B1846FFF74CFD03463CE07B6843
:10F520005A6807F11C000123396BFFF74EFD0346B3
:10F5300032E0FB681B68B9681846FFF7E3FC7863A4
:10F540007B6B002B26D00023BB623B683B62BB6C0D
:10F550007B627B6B5B6CFB617B681B78796B18460D
:10F56000FFF76CFE38637B685B681B78002B07D164
:10F5700007F11C03396B1846FFF70FFD03460BE03C
:10F580007B685A6807F11C000123396BFFF71DFDEA
:10F59000034601E06FF0120318464037BD4680BDB8
:10F5A00010CC021080B584B000AF786039603B6841
:10F5B000002B02D14FF0FF331DE00023FB6013E06E
:10F5C0007B68996DFA6813469B0013441B010B443A
:10F5D0003968184610F038F80346002B01D1FB6853
:10F5E00009E0FB680133FB607B68DB6DFA689A42D7
:10F5F000E6D34FF0FF3318461037BD4680BD0000FC
:10F6000080B588B000AFF860B9607A603B60FB6895
:10F610001B68FB61FB69DB6D002B02D16FF00103FE
:10F6200031E0B968F869FFF76DFCB861BB69002B80
:10F6300002D06FF0010326E0B968F869FFF737FCE4
:10F6400078617B69002B02D16FF012031BE07B69AC
:10F65000D3F8AC30B3F1FF3F04D17B6800221A70BD
:10F66000002310E0FB69996D7B69D3F8AC20134649
:10F670009B0013441B010B441B6C054A39687868D6
:10F680000FF0A0FE034618462037BD4680BD00BFE0
:10F69000A0CB021080B588B000AFF860B9607A6086
:10F6A0003B60FB681B68FB61FB69DB6D002B02D1D3
:10F6B0006FF0010331E0B968F869FFF723FCB86126
:10F6C000BB69002B02D06FF0010326E0B968F8692E
:10F6D000FFF7EDFB78617B69002B02D16FF012031D
:10F6E0001BE07B681B78002B06D17B694FF0FF3253
:10F6F000C3F8AC20002310E07968F869FFF752FFE7
:10F7000038613B69B3F1FF3F02D16FF0150304E0AC
:10F710007B693A69C3F8AC203B6818462037BD4680
:10F7200080BD80B584B000AF78600023FB603CE012
:10F730007B681A6DFB68B02101FB03F31344BB60C7
:10F74000BB68D3F8AC30B3F1FF3F28D07B68996D2C
:10F75000BB68D3F8AC2013469B0013441B010B4439
:10F7600093F84C3083F00103DBB2002B19D1BB6856
:10F770005B6DDB6A002B15D0BB685B6DDB6ABA681A
:10F780004832104698477B68996DFA6813469B008B
:10F7900013441B010B44002283F84C2002E000BFFD
:10F7A00000E000BFFB680133FB607B685B6DFA68BB
:10F7B0009A42BDD300BF00BF1037BD4680BD80B4A4
:10F7C00087B000AF786039600123FB6000237B6164
:10F7D00000233B613AE03B6803F00103002B2FD08C
:10F7E0003A691346DB0013449B001A467B681344B6
:10F7F0009B699B78DB08DBB2BB60BA68FB689A4206
:10F8000001D9BB68FB607B69BA68B3FBF2F2B968E7
:10F8100001FB02F29B1A002B0ED0BB685A007B69D9
:10F82000B968B3FBF1F1B86800FB01F15B1AD31AB8
:10F830007A6913447B6103E07A69BB6813447B6196
:10F840003B685B083B603B6901333B613B68002BD5
:10F85000C1D17B69FA68B3FBF2F2F96801FB02F2ED
:10F860009B1A002B0CD07B69FA68B3FBF2F2F968A3
:10F8700001FB02F29B1AFA68D31A7A6913447B617E
:10F880007B6918461C37BD4680BC704780B58CB07C
:10F8900000AFF860B9607A603B60FB681B68B968CC
:10F8A0001846FFF704FB38623B6A002B02D16FF069
:10F8B0001203E5E03B6A93F8A83083F00103DBB262
:10F8C000002B02D06FF01503DAE03B6A5B6D9B887A
:10F8D000C3F120034FF0FF3222FA03F3FB613A68D1
:10F8E000FB6913403B603B68002B02D16FF00103C2
:10F8F000C6E03B6A97F8382083F870203B6A002204
:10F900005A673B6A3A689A653B6A5B6D9B683968DF
:10F910001846FFF754FF02463B6A1A663B6A1B6EA5
:10F920007A6803FB02F23B6ADA653B6A7A685A66D8
:10F930003B6AD3F8A030002B22D03B6AD3F8A43026
:10F94000002B1DD03B6AD3F8A4203B6ADB6D9A42A2
:10F9500002D26FF00B0393E03B6AD3F8A4103B6A2A
:10F96000D3F8A4303A6AD26DB3FBF2F000FB02F296
:10F970009B1ACB1A7B623B6AD3F8A030BB6221E0B2
:10F980003B6A93F8A930002B08D03B6ADB6F18461E
:10F9900002F0A2FD3B6A002283F8A9203B6ADB6DDE
:10F9A0007B623B6ADB6D0121184602F087FDB8627D
:10F9B000BB6A002B02D16FF00B0361E03B6A0122AE
:10F9C00083F8A9203B6A78337A6AB96A184602F04C
:10F9D0008EFDF862FB6A002B0FDA3B6A93F8A930C0
:10F9E000002B08D03B6ADB6F184602F075FD3B6ABE
:10F9F000002283F8A920FB6A42E03B6A5B6D1B6A28
:10FA0000002B1BD03B6A5B6D1B6A3A6A526C3968EB
:10FA100010469847F862FB6A002B0FDA3B6A93F8AE
:10FA2000A930002B08D03B6ADB6F184602F054FD6A
:10FA30003B6A002283F8A920FB6A21E0FB681B686F
:10FA4000BB613B6AD3F8AC30B3F1FF3F17D0BB6961
:10FA5000996D3B6AD3F8AC2013469B0013441B01FD
:10FA60000B447B617B699B6C9B68002B07D07B6997
:10FA70009B6C9B687A69526C10469847F862FB6AE7
:10FA800018463037BD4680BD80B586B000AF78607F
:10FA9000396000237B617B681B6839681846FFF773
:10FAA00006FA38613B69002B02D14FF0FF334FE07B
:10FAB0003B6993F8A83083F00103DBB2002B02D03E
:10FAC0006FF0150344E03B6993F8A930002B08D090
:10FAD0003B69DB6F184602F0FFFC3B69002283F8AC
:10FAE000A9207B681B68FB603B69D3F8AC30B3F19D
:10FAF000FF3F1CD0FB68996D3B69D3F8AC201346DF
:10FB00009B0013441B010B44BB60BB689B6CDB6810
:10FB1000002B0CD0BB689B6CDB68BA68526C10463B
:10FB2000984778617B69002B01D07B6910E03B69C5
:10FB300000229A653B695B6D5B6A002B07D03B69CD
:10FB40005B6D5B6A3A69526C1046984778617B69D5
:10FB500018461837BD4680BD80B588B000AFF86044
:10FB6000B9601346FB71FB681B68B9681846FFF75C
:10FB70009EF9B861BB69002B07D0BB6993F8A83028
:10FB800083F00103DBB2002B02D06FF0150365E0B8
:10FB9000BB69FA7983F86820BB695B6D9B6A002BAF
:10FBA0000ED0BB69D3F8AC30B3F1FF3F08D1BB69CD
:10FBB0005B6D9B6ABA6948321046984703464DE030
:10FBC000FB79002B0AD1BB695B6D9B69002B05D0CB
:10FBD000BB69D3F8AC30B3F1FF3F0DD0FB79012BFB
:10FBE0003BD1BB695B6DDB69002B36D0BB69D3F8B9
:10FBF000AC30B3F1FF3F30D1BB6958337B6107F1C3
:10FC000010031946786900F0E4F8F861FB69002BED
:10FC100001DAFB6922E0FB79002B0AD1BB695B6D3D
:10FC20009B69BA69506C39697A69D2689847F861FA
:10FC300009E0BB695B6DDB69BA69506C39697A6947
:10FC4000D2689847F861FB69002B01DAFB6905E08F
:10FC5000786900F0E6F8034600E0002318462037F4
:10FC6000BD4680BD80B582B000AF786039600122AA
:10FC700039687868FFF770FF034618460837BD46B5
:10FC800080BD80B582B000AF7860396000223968ED
:10FC90007868FFF761FF034618460837BD4680BD08
:10FCA00080B588B000AFF860B9607A603B60FB68EF
:10FCB0001B68B9681846FFF7FAF8F861FB69002B72
:10FCC00007D0FB6993F8A83083F00103DBB2002B67
:10FCD00002D06FF0150331E0FB69783307F11402AD
:10FCE0001146184602F06FFCB861BB696FF4FA6206
:10FCF000934204D0BB69002B01DABB691EE07B692B
:10FD00003A68934228BF13463B603B68002B02D100
:10FD10006FF00A0312E0FB6978333A687968184695
:10FD200002F00AFEB861BB696FF4FA62934204D034
:10FD3000BB69002B01DABB6900E03B68184620373D
:10FD4000BD4680BD80B588B000AFF860B9607A600C
:10FD50003B60FB681B68B9681846FFF7A8F8F861B4
:10FD6000FB69002B07D0FB6993F8A83083F00103EF
:10FD7000DBB2002B02D06FF0150326E0FB6978336D
:10FD800007F110021146184602F01DFCB861BB696C
:10FD9000002B01DABB6918E0FB69DA6D3B69D31A05
:10FDA0007B613A687B69934228BF13463B60FB69DD
:10FDB00078333A687968184602F0ADFDB861BB69DE
:10FDC000002B01DABB6900E03B6818462037BD46CE
:10FDD00080BD80B584B000AF786039607B68002B4F
:10FDE00002D16FF0150318E07B681B7C002B0AD151
:10FDF0007B6858697B68596807F10C033A6802F020
:10FE000048FD034609E07B6858697B68596807F13B
:10FE10000C033A6802F051FD034618461037BD4600
:10FE200080BD80B582B000AF78607B68002B02D1C6
:10FE30006FF0150310E07B681B7C002B06D17B68FC
:10FE40005B69184602F04DFD034605E07B685B697F
:10FE5000184602F053FD034618460837BD4680BDDC
:10FE600080B582B000AF786039607B68002B02D12A
:10FE70006FF0150308E07B6858697B689B681A4639
:10FE8000396802F048FD034618460837BD4680BD74
:10FE900080B588B000AF78607868FFF742FC07F162
:10FEA0000C0319467868FEF7F5FEF861FB69002B34
:10FEB00001DAFB6911E07B681B68FA681146184695
:10FEC00002F0BCFAF861FB6913F1800F04D0FB6803
:10FED00019467868FEF7FDFEFB6918462037BD46D7
:10FEE00080BD000080B596B000AFF860B9607A6060
:10FEF0007B68B3F1FF3F02D10023FB6401E07B6824
:10FF0000FB64BB68002B02D107F11403BB60002324
:10FF10007B65FB689B6CBB64BB6C002B35D00023FE
:10FF20003B652CE07B6DBA68D018FA6C7B6DD31AF8
:10FF300023EAE37319463B6DDB00BA6C13441B687C
:10FF4000144A0FF03FFA02467B6D13447B657B6DCC
:10FF5000BA68D018FA6C7B6DD31A23EAE37319469A
:10FF60003B6DDB00BA6C13445B680B4A0FF02AFA56
:10FF700002467B6D13447B653B6D01333B65FB683B
:10FF8000DB6C1A463B6D9342CCDB7B6D18465837D1
:10FF9000BD4680BD24CC021044CC0210F0B59FB009
:10FFA00006AFF860B9607A603B60BB6FB3F1FF3FAA
:10FFB00002D100233B6501E0BB6F3B653B68002B32
:10FFC00002D107F114033B600023FB65FB6D3A6827
:10FFD000D0183A6DFB6DD31A23EAE3731946BB6858
:10FFE00000937B68A14A0FF0EDF90246FB6D1344C4
:10FFF000FB65FB689B68002B00F06C820023BB65EF
:020000041001E9
:1000000061E2FB689968BA6D1346DB0013449B00FC
:100010000B44FB6407F11403F96C1846FEF794FED9
:10002000FB6D3A68D0183A6DFB6DD31A23EAE3737F
:10003000194607F114038E4A0FF0C4F90246FB6D0E
:100040001344FB65FB6C1B68002B11D0FB6D3A68F9
:10005000D0183A6DFB6DD31A23EAE3731946FB6C93
:100060001B68844A0FF0AEF90246FB6D1344FB6532
:10007000FB6D3A68D0183A6DFB6DD31A23EAE3732F
:100080001946FB6C93F82030002B01D07A4B00E02E
:100090007A4B7B4A0FF096F90246FB6D1344FB65E1
:1000A000FB6C9B69002B2FD0FB6D3A68D0183A6D22
:1000B000FB6DD31A23EAE3739C46FB6C5969FB6C16
:1000C0009B691B79002B01D06E4B00E06E4BFA6CE4
:1000D000926912781446FA6C926952781546FA6C55
:1000E000926992781646FA6C9269D27804920396D5
:1000F0000295019400930B46644A61460FF062F941
:100100000246FB6D1344FB65FB6CDB69002B00F0C2
:10011000C78100237B65B7E1FB6CD9697A6D134613
:100120009B0013449B000B44BB64FB6D3A68D018E2
:100130003A6DFB6DD31A23EAE3731946BB6C1B6857
:10014000534A0FF03FF90246FB6D1344FB65FB6C0D
:1001500093F82330002B00F0CC80BB6C1B7A032B70
:1001600000F27F8101A252F823F000BF3502011096
:10017000DD010110A30101107D010110FB6D3A6842
:10018000D0183A6DFB6DD31A23EAE3731946BB6CA2
:100190001B68404A0FF016F90246FB6D1344FB65DD
:1001A0005FE1FB6D3A68D0183A6DFB6DD31A23EA14
:1001B000E3731946FB6C93F82030002B01D0364ACC
:1001C00000E0364ABB6C1B6800931346344A0FF0BC
:1001D000F9F80246FB6D1344FB6542E1FB6D3A689A
:1001E000D0183A6DFB6DD31A23EAE3731D46FB6CFE
:1001F00093F82030002B01D0274C00E0274CFB6CFB
:100200001B791A46274B53F82230FA6C12791146A3
:10021000244A52F82120B96C096802910192009396
:100220002346214A29460FF0CDF80246FB6D1344C0
:10023000FB6516E1FB6C93F8223083F00103DBB21F
:10024000002B02D06FF015030FE2FB6D3A68D51852
:100250003A6DFB6DD31A23EAE3739C46FB6C93F86B
:100260002030002B22D00C4E21E000BF54CC0210D5
:1002700070CC021084CC021090CC021098CC0210EA
:10028000A0CC0210B0CC0210B4CC0210B8CC02103A
:10029000ECCC021004CD021014CD021018CD0210C7
:1002A0001CCD021050CE021030CD02108D4EFB6CD2
:1002B0001B791A468C4B53F82230FA6C9268F96C11
:1002C00009790846884951F82010F86CC068BC6C60
:1002D0002468049403900291019200933346834A68
:1002E000614628460FF06EF80246FB6D1344FB652D
:1002F000B7E0BB6C1B7A032B00F2B38001A252F86B
:1003000023F000BFBF030110750301103B03011070
:1003100015030110FB6D3A68D0183A6DFB6DD31AC6
:1003200023EAE3731946BB6C1B68714A0FF04AF865
:100330000246FB6D1344FB6593E0FB6D3A68D018F1
:100340003A6DFB6DD31A23EAE3731946FB6C93F8FD
:100350002030002B01D0674A00E0624ABB6C1B686A
:1003600000931346644A0FF02DF80246FB6D1344C8
:10037000FB6576E0FB6D3A68D0183A6DFB6DD31AD9
:1003800023EAE3731C46FB6C93F82030002B01D06A
:10039000584900E05349FB6C1B791A46524B53F8FD
:1003A0002230BA6C1268019200930B46534A2146E0
:1003B0000FF008F80246FB6D1344FB6551E0FB6C3F
:1003C00093F82230002B27D0FB6D3A68D0183A6D95
:1003D000FB6DD31A23EAE3731D46FB6C93F82030C0
:1003E000002B01D0434C00E03E4CFB6C1B791A46BD
:1003F0003D4B53F82230FA6C9268B96C096802914F
:100400000192009323463E4A29460EF0DBFF024646
:10041000FB6D1344FB6523E0FB6D3A68D0183A6D21
:10042000FB6DD31A23EAE3731C46FB6C93F8203070
:10043000002B01D02F4900E02A49FB6C1B791A469A
:10044000294B53F82230BA6C1268019200930B4684
:100450002A4A21460EF0B6FF0246FB6D1344FB65A7
:1004600000BFFB6D3A68D0183A6DFB6DD31A23EAD2
:10047000E373244A19460EF0A5FF0246FB6D1344B0
:10048000FB657B6D01337B65FB6CD9697A6D134627
:100490009B0013449B000B441B68002B7FF43CAE75
:1004A000FB6D3A68D0183A6DFB6DD31A23EAE373FB
:1004B000154A19460EF086FF0246FB6D1344FB6594
:1004C000BB6D0133BB65FB689B881A46BB6D9342CD
:1004D000FFF697ADFB68DB68002B3FD00023BB65C0
:1004E00031E000BF18CD021050CE021048CD0210EE
:1004F00004CD021014CD02101CCD021064CD0210E8
:1005000078CD021090CD021094CD0210FB6D3A68A8
:10051000D0183A6DFB6DD31A23EAE3731C46FB68CF
:10052000D968BA6D13469B0013449B000B441B68AB
:10053000504A21460EF046FF0246FB6D1344FB6510
:10054000BB6D0133BB65FB68D968BA6D13469B0070
:1005500013449B000B441B68002BD7D1FB681B691D
:10056000002B2AD00023BB651CE0FB6D3A68D01835
:100570003A6DFB6DD31A23EAE3731C46FB681969D5
:10058000BA6D13469B0013449B000B441B683A4A08
:1005900021460EF017FF0246FB6D1344FB65BB6D51
:1005A0000133BB65FB681969BA6D13469B001344A0
:1005B0009B000B441B68002BD7D1FB681B6B002BE7
:1005C00003D1FB685B6B002B0FD0FB6D3A68D01832
:1005D0003A6DFB6DD31A23EAE373284A19460EF0ED
:1005E000F1FE0246FB6D1344FB65FB685B69002B63
:1005F0002AD00023BB651CE0FB6D3A68D0183A6D29
:10060000FB6DD31A23EAE3731C46FB685969BA6D84
:1006100013469B0013449B000B441B68184A214659
:100620000EF0D0FE0246FB6D1344FB65BB6D01333B
:10063000BB65FB685969BA6D13469B0013449B0068
:100640000B441B68002BD7D1FB6D3A68D0183A6D6C
:10065000FB6DD31A23EAE3730A4A19460EF0B2FE81
:100660000246FB6D1344FB65FB6D18466437BD46BF
:10067000F0BD00BFA0CD0210B8CD0210D8CD021041
:1006800008CE021028CE0210B0B598B002AF786044
:1006900007F10C033822002118460EF0E5FA40F26B
:1006A000F5333B654FF0FF3200217868FFF71AFC05
:1006B00002463B6D13443B6500237B6519E07B6874
:1006C0001A6D7B6DB02101FB03F313447B647B6CDB
:1006D000586D7B6C196C7A6C4FF0FF3300930023DC
:1006E000FFF75CFC02463B6D13443B657B6D0133B9
:1006F0007B657B685B6D7A6D9A42E0D300237B65F6
:100700001EE07B68996D7A6D13469B0013441B01B4
:100710000B44BB64BB6C9B6C5B68BB61BB6C196CB2
:10072000BA6C07F10C004FF0FF3300930023FFF782
:1007300035FC02463B6D13443B657B6D01337B65A5
:100740007B68DB6D7A6D9A42DBD33B6D013301210F
:10075000184601F0B3FE02467B681A647B681B6C86
:10076000002B02D16FF00B0378E07B683A6D5A647E
:100770007B681B6C3B4918460FF0D0F840F2EB3316
:10078000FB647B681A6CFB6CD1183A6DFB6CD31A56
:100790001A467868FFF7A6FB0246FB6C1344FB641D
:1007A00000237B651FE07B681A6D7B6DB02101FB28
:1007B00003F313447B647B6C586D7B6C196C7C6C0D
:1007C0007B681A6CFB6CD5183A6DFB6CD31A0093DE
:1007D0002B462246FFF7E2FB0246FB6C1344FB6408
:1007E0007B6D01337B657B685B6D7A6D9A42DAD3F2
:1007F00000237B6524E07B68996D7A6D13469B002E
:1008000013441B010B44BB64BB6C9B6C5B68BB61FA
:10081000BB6C196CBC6C7B681A6CFB6CD5183A6DA0
:10082000FB6CD31A07F10C0000932B462246FFF70E
:10083000B5FB0246FB6C1344FB647B6D01337B65A7
:100840007B68DB6D7A6D9A42D5D37B681A6CFB6C42
:100850001344054918460FF061F80023184658372D
:10086000BD46B0BD480F00203413002080B588B0CD
:1008700000AFF860B9607A60FB687A685A65FB6817
:100880005B6DB021184601F019FE0246FB681A653F
:10089000FB681B6D002B02D16FF00B036CE0002393
:1008A000FB6164E0FA6913465B001344DB001A46FF
:1008B000BB681344BB61FB681A6DFB69B02101FB87
:1008C00003F313447B61BB699A687B695A657B6952
:1008D000FA692B4918460EF0D5FDBB695B691946CC
:1008E000F868FEF75FFE02467B69C3F8AC20BB697F
:1008F0005A687B695A64BB695A687B699A647B69E8
:1009000003F158027B69DA64BB691A687B691A646F
:10091000BB699B689B69002B0ED1BB699B68DB6937
:10092000002B09D1BB699B689B6A002B04D1BB6972
:100930009B68DB6A002B13D0BB69DA687B69C3F85C
:10094000A020BB691A697B69C3F8A4207B6903F105
:1009500078027B69DA667B69012283F8A82003E0CC
:100960007B69002283F8A820FB690133FB61FA69E7
:100970007B689A4296D3002318462037BD4680BD37
:1009800034CE021080B588B000AFF860B9607A60EC
:10099000FB687A68DA65FB68DB6D5021184601F068
:1009A0008DFD0246FB689A65FB689B6D002B02D1AA
:1009B0006FF00B032EE00023FB6126E0FA6913467B
:1009C0005B0013449B001A46BB681344BB61FB6881
:1009D000996DFA6913469B0013441B010B447B611C
:1009E000BB695A687B695A64BB691A687B691A6477
:1009F000BB699A687B699A647B69FA6907491846FA
:100A00000EF040FDFB690133FB61FA697B689A4295
:100A1000D4D3002318462037BD4680BD44CE0210F3
:100A200080B592B000AF786039607B68002B02D04F
:100A30003B68002B02D16FF0150308E17021012003
:100A400001F03CFD38643B6C002B02D16FF00B03CE
:100A5000FDE03B68DA683B6C9A643B681A693B6C62
:100A6000DA643B68D9693B681B6A1A46386CFFF741
:100A700089FF78647B6C002BC0F2DD803B6859698C
:100A80003B689B691A46386CFFF7F0FE78647B6C14
:100A9000002BC0F2D780386CFFF7F6FD78647B6CD2
:100AA000002BC0F2C1803B6C0433FB63FB6B6A4AD2
:100AB0001A62FB6B694A5A62FB6B694A9A62FB6B6A
:100AC000684ADA62FB6B684A1A61FB6B674A9A6193
:100AD000FB6B674A5A61FB6B664ADA61FB6B664ADD
:100AE0009A60FB6B654ADA60FB6B654A1A60FB6BC8
:100AF000644A5A60FB6B644A5A633B6CFB62FB6B53
:100B0000BB623B6C1B6C3B633B6C5B6C7B633B680D
:100B10001B7887F838303B6C07F1280211461846DD
:100B200000F0F6FD78647B6C002B76DB3B6C6C335D
:100B30002C21184601F0F7FC78647B6C002B65DBF8
:100B40003B681B78002B24D13B6C504A9A663B6C67
:100B50004F4A5A663B685A683B6C1A663B6C1B6E80
:100B6000BB614C4BFB614FF480533B623B6C1B6899
:100B700007F1240207F11801184600F05AFE7864C4
:100B80007B6C002B39DB7B6A1946386CFEF7A1F8C9
:100B90002EE03B681B78012B26D13B689B681A68C6
:100BA0003B6C5A663B689B685A683B6C9A660023AC
:100BB000FB603B689B689B683B613B689B68DB68AC
:100BC0007B613B6C1B6807F1240207F10C0118469E
:100BD00000F02FFE78647B6C002B10DB7B6A1946DB
:100BE000386CFEF776F803E06FF015037B6407E0DE
:100BF0007B683A6C1A60002329E000BF00E000BF68
:100C00003B6CDB6E184601F0C3FC00E000BF3B6CA0
:100C10001B68184600F0D2FD00E000BF3B6C1B6C67
:100C2000184601F059FC00E000BF3B6C9B6D184674
:100C300001F052FC00E000BF3B6C1B6D184601F058
:100C40004BFC00E000BF386C01F046FC7B6C1846A2
:100C50004837BD4680BD00BF65F2001009F40010A2
:100C600001F6001095F60010A1FC001045FD0010E3
:100C700083FC001065FC00108DF8001089FA00104C
:100C80001FED0010F5EC00105FEF001041B20010F6
:100C9000DDB10010F82D012080B586B000AF78607E
:100CA0007B68002B02D16FF015031CE07B68DB6EC4
:100CB000184601F06DFC7B681B68184600F07EFD4D
:100CC0007B681B6D184601F007FC7B689B6D18461E
:100CD00001F002FC7B681B6C184601F0FDFB786894
:100CE00001F0FAFB002318461837BD4680BD80B4DA
:100CF00083B000AF78603960002318460C37BD46DA
:100D000080BC704780B5ADF5067D00AF07F5067372
:100D1000A3F50373186007F50673A3F50473196050
:100D200007F50673A3F505731A6007F50673A3F5B7
:100D3000057307F114001A6808490EF0A3FB034677
:100D4000C7F8143207F11403194605480DF0F2FFF5
:100D50000023184607F50677BD4680BDB4CE0210C5
:100D6000D8CE021080B58AB000AF786039603B6899
:100D70001B783B733B685B683B6101233B754FF419
:100D8000E133BB6103233B7700237B770023BB77F1
:100D90003B685B693B623B689B697B6207F10C03C4
:100DA00019467868FAF7A8F9034618462837BD4669
:100DB00080BD84B080B592B000AF786007F1540078
:100DC00080E80E0000237B64D7F88830BB631421D1
:100DD000012001F073FB78637B6B002B02D16FF075
:100DE0000B0316E1D7F88C207B6BDA60D7F89020E4
:100DF0007B6B1A6107F1540303F1180207F1080332
:100E000011461846FFF7AEFFF863FB6B002BC0F2EC
:100E1000DC8007F1540303F1180207F108031146BF
:100E20001846FFF764FFF863FB6B002BC0F2D98014
:100E3000BA687B6B1A6000233B73BB683B613B6EF7
:100E40001821184601F03AFB78647B6C002B03D123
:100E50006FF00B03FB63C7E000233B6490E0F96D88
:100E60003A6C13465B001344DB0019443A6C13469A
:100E70005B001344DB001A467B6C13440A681A605B
:100E8000F96D3A6C13465B001344DB0019443A6C6D
:100E900013465B001344DB001A467B6C13444A681C
:100EA0005A60F96D3A6C13465B001344DB00194439
:100EB0003A6C13465B001344DB001A467B6C134408
:100EC0008A689A60F96D3A6C13465B001344DB0044
:100ED00019443A6C13465B001344DB001A467B6CE2
:100EE00013444A695A61F96D3A6C13465B00134426
:100EF000DB000B44DB68002B08D0F96D3A6C13461D
:100F00005B001344DB000B44DB6807E0F96D3A6CCF
:100F100013465B001344DB000B441B693B633B6BD4
:100F2000002B16D03A6C13465B001344DB001A46C4
:100F30007B6C13443A6B5268DA603A6C13465B0080
:100F40001344DB001A467B6C13443A6B12681A6137
:100F500013E03A6C13465B001344DB001A467B6CCB
:100F600013440022DA603A6C13465B001344DB0042
:100F70001A467B6C134400221A613B6C01333B64BC
:100F80003B6E3A6C9A42FFF46AAF7B6C3B623B6EFD
:100F90007B627B6EBB62BB6EFB627B6DBB61BB6DBC
:100FA000FB617B6B083307F10C0211461846FFF713
:100FB00037FDF863FB6B002B15DB786C01F08CFAC6
:100FC0007B687A6B1A60002323E000BF07F15403AB
:100FD00003F1180207F1080311461846FFF7C2FE95
:100FE00002E000BF00E000BF786C01F075FA786B9A
:100FF00001F072FA07F1540303F1180107F1080335
:10100000FA6B1846FFF77EFEBB681846FAF7B8F889
:10101000FB6B18464837BD46BDE8804004B07047BA
:1010200080B584B000AF78607B689B681846FEF797
:101030002FFFF860FB68002B0ED0FB6813F10B0F3D
:101040000AD0FB6813F1800F06D0FB686FF4FA62D8
:10105000934201D0FB680EE07B68DB68002BE3D095
:101060007B68DB687A68126910469847F860FB680D
:10107000002BD9D0FB6818461037BD4680BD80B51F
:1010800084B000AF78607B681B68002B0AD07B6857
:101090001B681846FAF774F8F860FB68002B01D05B
:1010A000FB680EE07B689B681846FFF7F5FDF8606B
:1010B000FB68002B01D0FB6803E0786801F00CFAB4
:1010C000002318461037BD4680BD000080B584B0AF
:1010D00000AF786039607B68002B02D16FF0150398
:1010E00024E00023FB601CE0124AFB6852F8233026
:1010F000DB00114A1344BB60BB681B681946786863
:101100000EF0A2FA0346002B08D10A4AFB6852F8F7
:101110002330DAB23B681A70002307E0FB68013322
:10112000FB60FB680D2BDFD96FF0150318461037F5
:10113000BD4680BDA0CF02105413002080B586B0FC
:1011400000AFF860B9607A607A6807F11403194655
:10115000F8680FF031FF0246BB681A60BB681B6875
:10116000002B06D17B691B78002B02D06FF0150392
:1011700000E0002318461837BD4680BD80B586B014
:1011800000AFF860B9607A60FB68002B02D16FF0A5
:10119000150340E0BB680C330A221946F868FFF7D4
:1011A000CDFF78617B69002B01DA7B6933E07A68D7
:1011B0001B4900200FF08CFDF860FB68002B02D16A
:1011C0006FF0150327E0BB68043310221946F86856
:1011D000FFF7B4FF78617B69002B01DA7B691AE0C5
:1011E000BB6800221A767A680D4900200FF070FD66
:1011F000F860FB68002B0DD00A49F8680EF024FA5D
:101200000346002B03D1BB6801221A7602E06FF07F
:10121000150300E0002318461837BD4680BD00BF07
:10122000401300206CCF021080B584B000AFF8608E
:10123000B9607A60FB68002B02D16FF015031DE0E6
:101240001049F8680EF000FA0346002B02D06FF048
:10125000150313E07A680C4900200FF039FDF8609F
:10126000FB68002B02D16FF0150307E0BB68143355
:101270000A221946F868FFF761FF0346184610373F
:10128000BD4680BD74CF02104013002080B586B0EB
:1012900000AFF860B9607A60BB68042283F8D92196
:1012A000FB68002B1FD000237B6119E0494A7B6952
:1012B00052F823301946F8680EF0C6F90346002BA1
:1012C0000BD17A68444900200FF002FDF8607B6979
:1012D000DAB2BB6883F8D92105E07B6901337B6111
:1012E0007B69032BE2DDBB6893F8D931032B04D073
:1012F000BB6893F8D931022B12D1FB68002B02D1C5
:101300006FF0150361E0BB6859334022F968184655
:101310000EF024FC7A68304900200FF0D9FCF86008
:10132000BB681B78082B3BD1FB68002B02D16FF008
:1013300015034AE0FB681B782F2B14D9FB681B7838
:10134000392B10D8BB6899334FF4807200211846AE
:101350000DF08AFCBB6810330A221946F868FFF7C3
:10136000EDFE034631E0BB6899334FF48072F968B3
:1013700018460EF0F3FB7A68174900200FF0A8FC1E
:10138000F860FB68002B02D16FF015031DE0BB680D
:1013900010330A221946F868FFF7D0FE034614E01E
:1013A000FB68002B08D0BB6899334FF48072F96852
:1013B00018460EF0D3FB07E0BB6899334FF48072F8
:1013C000002118460DF050FC002318461837BD4682
:1013D00080BD00BF441300204013002080B586B0BC
:1013E00000AFF860B9607A607A684749F8680FF032
:1013F0006FFC7861B9687869FFF768FE38613B690E
:10140000002B01DA3B697AE07A683F4900200FF04F
:101410005FFC7861BB681B78032B02DC002B03DACE
:101420000DE0042B02D00AE0002368E0BB6808331B
:101430000A2219467869FFF781FE03465FE0BB6820
:1014400019334022796918460EF088FB7A682E49D4
:1014500000200FF03DFC7861BB681B78053B082B32
:101460004AD801A252F823F0911401108D140110F2
:101470009F1401109F140110AD140110AD14011040
:101480008D140110BF140110EB140110002336E07D
:101490007A68B9687869FFF771FE03462FE07A68C9
:1014A000B9687869FFF7F2FE034628E0BB6810339D
:1014B0000A2219467869FFF741FE03461FE07B695F
:1014C000002B08D0BB6803F29913402279691846B3
:1014D0000EF044FB07E0BB6803F2991340220021A1
:1014E00018460DF0C1FB002309E07A68B9687869F5
:1014F000FFF79AFE034602E000BF6FF0150318469F
:101500001837BD4680BD00BF4013002080B485B0B1
:1015100000AFF860B9607A603B606FF01503184661
:101520001437BD4680BC704780B483B000AF78608C
:1015300039606FF0150318460C37BD4680BC704704
:1015400080B485B000AFF860B9607A603B606FF03E
:10155000150318461437BD4680BC704780B485B06B
:1015600000AFF860B9607A603B606FF01503184611
:101570001437BD4680BC704780B485B000AFF860BA
:10158000B9607A603B606FF0150318461437BD46AA
:1015900080BC704780B483B000AF786039606FF072
:1015A000150318460C37BD4680BC704780B485B023
:1015B00000AFF860B9607A606FF015031846143711
:1015C000BD4680BC7047000080B483B000AF786037
:1015D00039603B685B68002B03D03B681B68002BBD
:1015E00002D16FF0150380E03B685A687B685A604F
:1015F0003B681A687B681A603B689B68002B02D0C6
:101600003B689B6800E03B4B7A6893603B68DB6813
:10161000002B02D03B68DB6800E0374B7A68D36070
:101620003B681B69002B02D03B681B6900E0334B11
:101630007A6813613B689B69002B02D03B689B6909
:1016400000E02F4B7A6893613B681B6A002B02D045
:101650003B681B6A00E02B4B7A6813623B685B6A4D
:10166000002B02D03B685B6A00E0264B7A6853622D
:101670003B689B6A002B02D03B689B6A00E01F4BD3
:101680007A6893623B68DB6A002B02D03B68DB6AB6
:1016900000E01B4B7A68D3623B681B6B002B02D0C7
:1016A0003B681B6B00E0184B7A6813633B685B6B0D
:1016B000002B02D03B685B6B00E0144B7A685363ED
:1016C0003B685B69002B02D03B685B6900E00A4B1A
:1016D0007A6853613B68DB69002B02D03B68DB69A9
:1016E00000E0054B7A68D361002318460C37BD46ED
:1016F00080BC70470D150110291501105D150110F2
:10170000791501104115011095150110AD15011045
:1017100080B584B000AF786039607B68002B06D05C
:101720003B68002B03D03B681B68002B02D16FF095
:1017300015033FE04FF4D85101200CF0C5FE0346DD
:10174000FB60FB68002B02D16FF00B0332E0FB68FB
:1017500003F5D55318333A68126811461846FFF757
:1017600033FFB860BB68002B04DAF8680CF030FF78
:10177000BB681FE03B689B68FA6802F58052C2F8BC
:10178000F43A3B68DB68FA6802F58052C2F8F83A2E
:101790003B685B68FA6802F58052C2F8F03A3B6831
:1017A0001A7CFB6803F5805383F8FC2A7B68FA688F
:1017B0001A60002318461037BD4680BD80B582B040
:1017C00000AF786078680CF003FF00BF0837BD46B3
:1017D00080BD80B582B000AF78607B6808334FF47D
:1017E000EE72002118460DF03FFA7B6803F5F273A4
:1017F0001422002118460DF037FA7B6803F5227396
:101800000C22002118460DF02FFA7B680022C3F845
:10181000EC217B680022C3F8F0217B680022C3F82A
:101820007C227B68002283F8F82100BF0837BD4680
:1018300080BD80B586B000AFF860B9607A60FB68A3
:10184000002B02D07B68002B02D16FF015033CE027
:1018500000237B6134E0FA687B694FF42B7101FB54
:1018600003F3134404331B7883F00103DBB2002B32
:1018700023D07B694FF42B7202FB03F3FA68134405
:101880003B614FF42B72002138690DF0EDF93B6993
:1018900001221A71BB681A683B691A60BB685A68F2
:1018A0003B69C3F88022BB689A683B69C3F884220D
:1018B0007B687A691A60002307E07B6901337B61EA
:1018C0007B69092BC7D96FF00F0318461837BD463F
:1018D00080BD0000F0B587B002AFF860B9607A60F3
:1018E000BB681B780D2B65D801A252F823F000BF0E
:1018F00029190110B5190110B5190110B5190110F8
:101900002F1901104119011063190110B5190110A7
:10191000B5190110B5190110B5190110B51901104B
:10192000751901109F1901106FF0150345E0FB6850
:101930001B6BBA68926811467868984703463CE08A
:10194000FB689C68BB6803F11901BB68DA68BB6877
:101950005868BB681B7E009303467868A04703461F
:101960002BE0FB68DB68BA68193211467868984743
:10197000034622E0FB68DC6ABB6803F11905BB681B
:1019800003F29916BB6803F2991318460EF038F863
:101990000346324629467868A04703460DE0FB68B7
:1019A0005B6BBA6802F11901BA68526978689847A6
:1019B000034602E000BF6FF0150318461437BD461A
:1019C000F0BD00BF80B58AB000AFF860B9607A6042
:1019D000FB70FB6803F58053D3F8F03A7B61BB687A
:1019E0001B68BB617B689A687B685B68D31A3B6243
:1019F0003B6A002B33D07B681A687B685B681344B2
:101A0000FB61FB7803F00103002B0BD0FB6803F5AF
:101A10008053D3F8B83A3A6A07F11400F969984745
:101A200078620AE0FB6803F58053D3F8BC3A3A6A5F
:101A300007F11400F969984778627B6A002B01DA94
:101A40007B6A28E07B685A687B6A1A447B685A6024
:101A50007A6A3B6A9A4202DA6FF00A031BE0FB786B
:101A600003F00203002B15D0FB6803F58053D3F875
:101A7000B83A07F1140001220949984778627B6A55
:101A8000002B01DA7B6A06E07B6A012B02D06FF043
:101A90000A0300E0002318462837BD4680BD00BF7A
:101AA00084CF021090B589B000AF786039607B6850
:101AB00003F58053D3F8F03AFB603B681B683B6149
:101AC0003B68D3F880223B68C3F888223B689A6958
:101AD0003B68D3F88432934228BF1346FB61FA690E
:101AE0003B68D3F89032D31ABB617B6803F580530F
:101AF000D3F8C84A3B6803F121013B68D3F8882238
:101B00003B68D3F890321A4407F10C00BB69A04738
:101B100078617B69002B01DA7B6928E03B68D3F8A8
:101B200090227B691A443B68C3F890223B68D3F843
:101B300090223B689B699A4202D26FF00A0316E03A
:101B40003B6803F52272012339687868FFF73AFF92
:101B500078617B69002B01DA7B6908E03B68002231
:101B6000C3F890223B680022C3F88C220023184659
:101B70002437BD4690BD90B589B000AF786039601C
:101B80007B6803F5805393F8FC3A022B05D1396842
:101B90007868FFF787FF034665E07B6803F58053AD
:101BA000D3F8F02A3B681B683A617B613B68D3F845
:101BB0009032002B2DD13B68D3F880223B68C3F8CC
:101BC00088223B689A693B68D3F88432934228BFE5
:101BD0001346FB617B6803F58053D3F8C84A3B6822
:101BE00003F121013B68D3F88822FB6907F110005B
:101BF000A047B861BB69002B01DABB6933E0BB6960
